:020000021000EC
:1060000000600020D5B801001DB901001FB90100D2
:106010000000000000000000000000000000000080
:1060200000000000000000000000000021B9010095
:10603000000000000000000023B9010025B90100A4
:1060400027B9010027B9010071A9010027B9010092
:1060500027B90100000000001DB2010027B90100AE
:1060600027B9010027B9010027B9010027B90100AC
:1060700027B9010027B9010027B9010027B901009C
:1060800027B9010019A1010027B9010027B90100B2
:1060900065A1010027B90100F190010027B90100B5
:1060A00027B9010027B9010000000000000000002E
:1060B00000000000000000000000000000000000E0
:1060C00010B5064C2378002B07D1054B002B02D0CE
:1060D000044800E000BF0123237010BDD828002031
:1060E000000000007434020008B5084B002B03D0F8
:1060F0000748084900E000BF07480368002B03D0A9
:10610000064B002B00D0984708BDC0460000000099
:1061100074340200DC280020D42800200000000095
:10612000164B002B00D1144B9D46402292029A1A26
:10613000924600218B460F461348144A121A05F066
:1061400069FC0F4B002B00D098470E4B002B00D062
:1061500098470020002104000D000D48002802D0BF
:106160000C4807F0C9F805F0EFFB2000290000F00B
:1061700095FE05F0D9FBC046000008000060002035
:106180000000000000000000D8280020942D00200E
:10619000F9D2010091E3010080B500AFBFF34F8F4A
:1061A000024B034ADA60BFF34F8FFEE700ED00E0D9
:1061B0000400FA0570DF7047181CC04671DF704795
:1061C000181CC04672DF7047181CC04673DF70474A
:1061D000181CC04674DF7047181CC04675DF704736
:1061E000181CC04676DF7047181CC04677DF704722
:1061F000181CC04678DF7047181CC04679DF70470E
:10620000181CC0467ADF7047181CC0467BDF7047F9
:10621000181CC0467CDF7047181CC0467DDF7047E5
:10622000181CC0467EDF7047181CC0467FDF7047D1
:10623000181CC04680DF7047181CC04681DF7047BD
:10624000181CC04682DF7047181CC04683DF7047A9
:10625000181CC04684DF7047181CC046B0DF70476A
:10626000181CC046B1DF7047181CC046B2DF70472B
:10627000181CC04690DF7047181CC04691DF70475D
:10628000181CC04692DF7047181CC04693DF704749
:10629000181CC04694DF7047181CC04695DF704735
:1062A000181CC04696DF7047181CC04697DF704721
:1062B000181CC04698DF7047181CC046A0DF704706
:1062C000181CC046A1DF7047181CC046A2DF7047EB
:1062D000181CC046A3DF7047181CC046A4DF7047D7
:1062E000181CC046A5DF7047181CC046A6DF7047C3
:1062F000181CC046A7DF7047181CC046A8DF7047AF
:10630000181CC046A9DF7047181CC046AADF70479A
:10631000181CC04660DF7047181CC04661DF70471C
:10632000181CC04662DF7047181CC04663DF704708
:10633000181CC04664DF7047181CC04665DF7047F4
:10634000181CC04666DF7047181CC04667DF7047E0
:10635000181CC04668DF7047181CC04669DF7047CC
:10636000181CC04623DF7047181CC04624DF704746
:10637000181CC04625DF7047181CC04626DF704732
:10638000181CC04627DF7047181CC04628DF70471E
:10639000181CC04629DF7047181CC0462ADF70470A
:1063A000181CC0462BDF7047181CC0462CDF7047F6
:1063B000181CC0462DDF7047181CC0462EDF7047E2
:1063C000181CC0462FDF7047181CC04630DF7047CE
:1063D000181CC04631DF7047181CC04632DF7047BA
:1063E000181CC04635DF7047181CC04636DF7047A2
:1063F000181CC04633DF7047181CC04634DF704796
:10640000181CC04637DF7047181CC04638DF70477D
:10641000181CC04639DF7047181CC0463ADF704769
:10642000181CC0463BDF7047181CC0463CDF704755
:10643000181CC0463DDF7047181CC0463EDF704741
:10644000181CC0463FDF7047181CC04641DF70472C
:10645000181CC04642DF7047181CC04643DF704717
:10646000181CC04640DF7047181CC04644DF704708
:10647000181CC04645DF7047181CC04646DF7047F1
:10648000181CC04647DF7047181CC04648DF7047DD
:10649000181CC04649DF7047181CC0464ADF7047C9
:1064A000181CC0464BDF7047181CC0464CDF7047B5
:1064B000181CC0464DDF7047181CC04651DF70479E
:1064C000181CC04652DF7047181CC04621DF7047B9
:1064D000181CC04620DF7047181CC04622DF7047DA
:1064E000181CC0464EDF7047181CC0464FDF70476F
:1064F000181CC04650DF7047181CC04610DF70479C
:10650000181CC04611DF7047181CC04612DF7047C8
:10651000181CC04613DF7047181CC04680B582B0F7
:1065200000AF7860A023DB057A68C132FF329200A9
:106530000321D150BD4602B080BDC04680B582B0B7
:1065400000AF7860FB1C1970BB1C1A70A023DB0520
:10655000BA1C12781204111CFA1C12789200114312
:106560007A68C132FF329200D150BD4602B080BD80
:1065700080B582B000AF7860A023DA057B68012186
:106580009940A123DB00D150BD4602B080BDC0467A
:1065900080B582B000AF7860A023DA057B68012166
:1065A0009940024BD150BD4602B080BD0C050000A1
:1065B00080B584B000AFF860B9607A60FFF7ECFD99
:1065C000BD4604B080BDC04680B582B000AF021C9D
:1065D0003960BB1D1A80BB1D1A8805493B68081C21
:1065E000111C1A1CFFF7E4FFBD4602B080BDC04677
:1065F000EFBEADDE80B500AF1220FFF78FFF132096
:10660000FFF78CFFBD4680BD80B584B002AF0C4B58
:106610000022009200200221052203F0A9FD031CA4
:106620007B607B683B603B68002B06D03A68054B7B
:10663000101CAB211A1CFFF7BBFFBD4602B080BD8A
:106640001C290020142E020080B586B000AF3B1C30
:106650001A780F218A4301210A431A703B1C1978CA
:106660000F220A4010210A431A703A1C1D4B101CBD
:10667000191C0722FFF7CEFD031C7B617B693B6180
:106680003B69002B06D03A69174B101CBF211A1C1E
:10669000FFF78EFF3B1D181C0021082205F0BAF9F8
:1066A0003B1D07221A803B1D3C225A803B1D0022C5
:1066B0009A803B1DC8225200DA803B1D181CFFF750
:1066C000A1FD031C7B617B69FB60FB68002B06D08E
:1066D000FA68054B101CC9211A1CFFF769FFBD465B
:1066E00006B080BD202E0200142E020080B5A6B098
:1066F00000AFFB1D05221A703A1C2C4B111C1A1CF2
:106700000423081C111C1A1C05F042F93B1C083319
:10671000181C0021382205F07DF93B1C08330222A9
:106720001A703B1C083300229A703B1C083301226C
:106730009A803B1C0833FA1D9A603B1C08330122E7
:106740001A833B1C08333A1CDA613B1C0833181CC3
:10675000002101F02DFE031C9420C0190360391C98
:106760004031134A9420C0190368081C502105F0D9
:10677000D1F93B1C4033181C00F0C6FA9422D21900
:1067800013689020C01903609022D2191368002B5F
:1067900008D09023DB191A68064B101CEE211A1C36
:1067A000FFF706FFBD4626B080BDC046342E02006E
:1067B000282E0200142E020080B586B000AFF860CB
:1067C000B960BB1D1A8000237B6109E07B69BA6850
:1067D000D3181B78181C04F017FB7B6901337B610D
:1067E000BB1D1A887B699A42F0DC0A2004F00CFB7E
:1067F000BD4606B080BDC04680B584B000AF3B1D2D
:10680000181C0021042205F005F90E4B7B600E4A8E
:106810003B1D101C191C00F055FF031CFB60FB689E
:10682000BB60BB68002B09D0B96810231A1CFF326B
:10683000064B081C111C1A1CFFF7BAFEBD4604B01B
:1068400080BDC046B9670100FC280020142E02005C
:1068500080B500AF104B1E221A800F4B9A78012191
:106860000A439A700C4B9A7802218A439A700A4B19
:106870009A781C218A430C210A439A70064B9A7815
:1068800020218A439A70044B0722DA70024B1022AF
:106890001A71BD4680BDC046F428002080B584B082
:1068A00000AF78607B681B78002B16D10C4B1B88DF
:1068B000181C3B21FFF796FC031CFB60FB68BB60C8
:1068C000BB68002B09D0B96834231A1CFF32054B72
:1068D000081C111C1A1CFFF76BFEBD4604B080BDDE
:1068E00004200020142E020080B582B000AF786032
:1068F00079689F235A00044B081C111C1A1CFFF7CF
:1069000057FEBD4602B080BD142E020080B58AB08D
:1069100000AF3B1D181C00211C2205F07BF83B1D1D
:1069200000221A603B1DA02292025A603B1DF022F9
:1069300012039A603B1D03221A733B1D0022DA8169
:106940003B1D00221A743B1D0E4A5A613B1D0E4A24
:106950009A613B1D181C01F011FF031C7B627B6ACE
:106960003B623B6A002B09D0396A56231A1CFF325E
:10697000064B081C111C1A1CFFF71AFEBD460AB074
:1069800080BDC0469D680100E9680100142E020028
:1069900080B588B000AF3B1D181C0021142205F003
:1069A00039F83B1D00221A703B1D00225A603B1D26
:1069B00000221A723B1D40221A823B1DB4225A82C9
:1069C0003B1D181CFFF702FC031CFB61FB69BB614C
:1069D000BB69002B08D0B969B5235A00054B081CC8
:1069E000111C1A1CFFF7E4FD1220FFF7C1FDBD4684
:1069F00008B080BD142E020080B58AB000AF786068
:106A00006E4B181C00F080F97B681B88132B29D073
:106A100007DC102B11D0112B1AD0012B00D1BEE0B6
:106A2000C9E0172B52D002DC142B5AD0C3E0192B2B
:106A300000D193E0522B2FD0BDE01320FFF798FD3B
:106A40001220FFF7A5FD7B689A885D4B1A80B2E0A3
:106A50001320FFF79DFD5A4B012252421A80FFF787
:106A600097FFA8E0564B1A88564B101C00211A1CA1
:106A7000FFF7DCFB031C7B627B6A3B623B6A002BFB
:106A800009D0396AC8235A004F4B081C111C1A1C24
:106A9000FFF78EFD8FE08EE0494B1B88181C00210C
:106AA0000022FFF72FFC031C7B627B6AFB61FB6902
:106AB000002B0AD0F96996231A1CFF32424B081C9E
:106AC000111C1A1CFFF774FD75E074E03F497A68E9
:106AD0000623D2183223081C111C1A1C04F058FF7C
:106AE00069E03B4BBB61BB691A887B68DB899A42D2
:106AF0001AD1334B1A88BB69101C191C0022FFF7EE
:106B00009DFB031C7B627B6A7B617B69002B0AD047
:106B10007969A2231A1CFF322B4B081C111C1A1C6A
:106B2000FFF746FD19E018E0254B1B88181C0021D3
:106B30000022FFF783FB031C7B627B6A3B613B699E
:106B4000002B0AD03969A8231A1CFF321E4B081CDF
:106B5000111C1A1CFFF72CFD2DE02CE07B689B79A3
:106B6000002B1BD11220FFF713FD1020032103225D
:106B7000FFF7E4FCFFF742FC031C7B627B6AFB60CF
:106B8000FB68002B0AD0F968B8231A1CFF320E4BA1
:106B9000081C111C1A1CFFF70BFD0CE00BE00D4B41
:106BA0001B7801225340DBB2002B03D00A4B012299
:106BB0001A70FFE7C046BD460AB080BD382E0200FD
:106BC00004200020F4280020142E0200342B002082
:106BD0003A2B0020062000201829002080B582B022
:106BE00000AF78607B68181C01F026FF064A7B68BE
:106BF000101C191C00F038FD7B68181CFFF7FCFE08
:106C0000BD4602B080BDC046FC28002080B586B0DD
:106C100000AF274B0820191C5022002302F0E6F990
:106C2000031C7B617B693B613B69002B08D03969A0
:106C3000EF235A001F4B081C111C1A1CFFF7B8FC4D
:106C40003B1C181C0021012204F0E4FE3B1C1A78B6
:106C500001218A431A703B1C181CFFF75BFB031CC5
:106C6000FB60FB68BB60BB68002B09D0B968E623FA
:106C70001A1CFF320F4B081C111C1A1CFFF798FC42
:106C80000D4B181C02F00CFA031CFB60FB687B60C8
:106C90007B68002B09D07968EA231A1CFF32054B68
:106CA000081C111C1A1CFFF783FCBD4606B080BDF2
:106CB000682B0020142E0200DD6B010080B500AFB0
:106CC000102003210322FFF739FCBD4680BDC046DA
:106CD00080B582B000AFFFF7C5FB031C7B607B680B
:106CE0003B603B68002B09D03968FC231A1CFF323B
:106CF000044B081C111C1A1CFFF75AFCBD4602B0BD
:106D000080BDC046142E020080B586B000AF78600A
:106D10007B68181C04F032FF021C3B1C16331A70EF
:106D20003B1C173300221A701EE03B1C17331B78E4
:106D30007A68D3181B78181C04F066F8031C3B61B2
:106D40003B69FB60FB68002B07D0F9680C4A0D4BD0
:106D5000081C111C1A1CFFF72BFC3B1C17331A785C
:106D60003B1C173301321A703A1C17323B1C163386
:106D700012781B789A42D8D3BD4606B080BDC04673
:106D800009020000142E020080B582B000AF7860C6
:106D90007B681B78032B04D0042B04D0002B04D079
:106DA00004E0C04602E0C04600E0C046BD4602B076
:106DB00080BDC04680B58AB002AF3B1C16330022AE
:106DC0001A803B1D144A1A603B1D20225A603B1D4D
:106DD000124A9A603B1D2022DA6011493A1D114B7C
:106DE000381C16300090081C111C1A1C032303F0D9
:106DF00093FE031CFB61FB69BB61BB69002B07D0E1
:106E0000B969094A094B081C111C1A1CFFF7D0FB71
:106E1000BD4608B080BDC046B82B0020D82B00204E
:106E2000082E0200896D01003A020000142E0200B3
:106E300080B584B000AF78600A1CFB1C1A70FB1C84
:106E40001B789BB211497A68081C111C1A1C00F0AF
:106E5000A5FC031CFB60FA680D4B9A4201D100238C
:106E600010E0FB68082B0CD0FB68BB60BB68002BF4
:106E700007D0B968074A084B081C111C1A1CFFF7F9
:106E800097FB0123181CBD4604B080BDFC280020E0
:106E9000043000004A020000142E020080B582B0C7
:106EA00000AFFFF7A7FBFFF7AFFBFFF707FFFFF709
:106EB00081FF304B181CFFF727FFFFF7A7FEFFF7F6
:106EC000C3FBFFF799FCFFF711FCFFF71FFDFFF76E
:106ED000BFFC294B181CFFF717FFFFF759FD274B85
:106EE000181CFFF711FF264B1B78002B26D0FB1D2B
:106EF000181C03F077FF031C002B1FD1214B1B78BC
:106F00005A1CD1B21F4A1170FA1D11781E4AD15471
:106F10001C4B1B78132B11D91A4B1B781A4A101CC7
:106F2000191CFFF785FF031C1A1C154B1A70144B14
:106F30001B78002B02D0134B00221A70134B1B78C6
:106F4000002B14D0114B00221A700E4B1B780E4AE6
:106F5000101C191CFFF76CFF031C1A1C084B1A703D
:106F6000074B1B78002B02D0064B00221A70FFF74C
:106F7000AFFEB8E7442E02004C2E0200582E02004D
:106F800006200020F82B0020FC2B002018290020D0
:106F900070DF7047181CC04671DF7047181CC04670
:106FA00072DF7047181CC04673DF7047181CC0465C
:106FB00074DF7047181CC04675DF7047181CC04648
:106FC00076DF7047181CC04677DF7047181CC04634
:106FD00078DF7047181CC04679DF7047181CC04620
:106FE0007ADF7047181CC0467BDF7047181CC0460C
:106FF0007CDF7047181CC0467DDF7047181CC046F8
:107000007EDF7047181CC0467FDF7047181CC046E3
:1070100080DF7047181CC04681DF7047181CC046CF
:1070200082DF7047181CC04683DF7047181CC046BB
:1070300084DF7047181CC04680B584B000AF78600C
:1070400039603B1C0F3300221A703B1C0F331B7836
:107050003A1C0F32591C11707A68D3183A681278AA
:107060001A703B1C0F331B783A1C0F32591C1170DD
:107070007A68D3183A6852781A703B1C0E333A1C5F
:107080000F321278023A51424A411A703B1C0E33B9
:107090001B7801225340DBB2002B05D0064B0020A9
:1070A00020211A1CFFF784FA3B1C0F331B78181C95
:1070B000BD4604B080BDC046642E020080B582B0DB
:1070C00000AF786039603B68181C04F057FD031C62
:1070D0009AB27B681A807B683A685A60BD4602B0F3
:1070E00080BDC04670DF7047181CC04671DF704716
:1070F000181CC04672DF7047181CC04673DF70470B
:10710000181CC04674DF7047181CC04675DF7047F6
:10711000181CC04676DF7047181CC04677DF7047E2
:10712000181CC04678DF7047181CC04679DF7047CE
:10713000181CC0467ADF7047181CC0467BDF7047BA
:10714000181CC0467CDF7047181CC0467DDF7047A6
:10715000181CC0467EDF7047181CC0467FDF704792
:10716000181CC04680DF7047181CC04681DF70477E
:10717000181CC04682DF7047181CC04683DF70476A
:10718000181CC04684DF7047181CC046B0DF70472B
:10719000181CC046B1DF7047181CC046B2DF7047EC
:1071A000181CC04690DF7047181CC04691DF70471E
:1071B000181CC04692DF7047181CC04693DF70470A
:1071C000181CC04694DF7047181CC04695DF7047F6
:1071D000181CC04696DF7047181CC04697DF7047E2
:1071E000181CC04698DF7047181CC046A0DF7047C7
:1071F000181CC046A1DF7047181CC046A2DF7047AC
:10720000181CC046A3DF7047181CC046A4DF704797
:10721000181CC046A5DF7047181CC046A6DF704783
:10722000181CC046A7DF7047181CC046A8DF70476F
:10723000181CC046A9DF7047181CC046AADF70475B
:10724000181CC04660DF7047181CC04661DF7047DD
:10725000181CC04662DF7047181CC04663DF7047C9
:10726000181CC04664DF7047181CC04665DF7047B5
:10727000181CC04666DF7047181CC04667DF7047A1
:10728000181CC04668DF7047181CC04669DF70478D
:10729000181CC04680B582B000AF78607B681B7850
:1072A0001A1C7B6801331B781B029BB213439BB2F1
:1072B0009BB2181CBD4602B080BDC04690B585B0DB
:1072C00000AF78603C1C0E347B68181CFFF7E2FFAF
:1072D000031C23803B1C0E331A88012313405A1EC3
:1072E0009341DBB2181CBD4605B090BD80B582B09D
:1072F00000AF786039603B689A887B689A82BD46A7
:1073000002B080BD80B582B000AF786039607B6824
:10731000012252429A82BD4602B080BD80B584B03F
:1073200000AF786039603B680633FB60FB681A8801
:107330007B681B8A9A4213D1FB681B8B022B0FD1EF
:10734000FB681A33181CFFF7B9FF031C002B03D08E
:107350007B6801229A7516E07B6800229A7512E01C
:10736000FB681A887B689B889A420CD17B689B6972
:10737000002B08D07B689B69FA68111C1A31FA68E7
:10738000128B78689847BD4604B080BD80B592B036
:1073900000AF786039603B1C2833181C00210322A1
:1073A00004F038FB3B1C28331A780F218A43012153
:1073B0000A431A703B1C283319780F220A40102107
:1073C0000A431A703B1C28335A780F218A43012143
:1073D0000A435A703B1C283359780F220A40102167
:1073E0000A435A703B1C28339A7806218A430221AB
:1073F0000A439A703B1C2C33181C00211C2204F0F9
:1074000009FB3B1C2C331A7810210A431A703B1CD1
:107410002C3300225A603B1C2C330022DA603B1CC8
:107420002C3300221A613B1C2C333A1C28325A613F
:107430003B1C2C3300229A617B681A783B1C10336A
:107440009A703B1C103303221A803B1C0C33181C0F
:107450000021032204F0DEFA3B1C0C331A780F21C2
:107460008A4301210A431A703B1C0C3319780F22FE
:107470000A4010210A431A703B1C0C335A780F2122
:107480008A4301210A435A703B1C0C3359780F225E
:107490000A4010210A435A703B1C0C339A7806218B
:1074A0008A4302210A439A703B1C0C339A780821C4
:1074B0008A439A703B1C0C339A7810218A439A7045
:1074C0003B1C0C339A7801210A439A703B1C1433FD
:1074D000181C0021142204F09DFA3B1C14333A1CA2
:1074E00010321A603B1C14333A1C0C325A603B1C9D
:1074F000143301221A813B1C143300225A813B1C95
:10750000143314229A817B6858887B680C33391CA9
:107510002C313A1C1432FFF771FE031C181CBD46B7
:1075200012B080BD80B590B000AF786039603B1C70
:107530002433181C00211C2204F06CFA3B1C243359
:107540001A7808210A431A703B1C24331A78042144
:107550000A431A703B1C243300225A603B1C24331C
:107560000022DA603B1C243300221A613B1C2433C6
:1075700000225A613B1C243300229A617B681A78EE
:107580003B1C0C339A703B1C0C3302221A803B1CB0
:107590000833181C0021032204F03CFA3B1C08337A
:1075A0001A780F218A4301210A431A703B1C0833C1
:1075B00019780F220A4010210A431A703B1C083325
:1075C0005A780F218A4301210A435A703B1C083321
:1075D00059780F220A4010210A435A703B1C083385
:1075E0009A7806218A4302210A439A703B1C083389
:1075F0009A7808218A439A703B1C08339A781021A4
:107600008A439A703B1C08339A7801210A439A7086
:107610003B1C1033181C0021142204F0FBF93B1C06
:1076200010333A1C0C321A603B1C10333A1C0832DF
:107630005A603B1C103301221A813B1C103300227C
:107640005A813B1C103314229A817B6858887B68CE
:107650000433391C24313A1C1032FFF7CFFD031CD0
:10766000181CBD4610B080BD80B582B000AF7860F8
:1076700039607B68002B02D03B68002B00D11DE0F5
:107680003B681B88112B0BD0502B10D0102B00D037
:1076900014E07A683B68101C191CFFF727FE0DE008
:1076A0007A683B68101C191CFFF72CFE06E07A680C
:1076B0003B68101C191CFFF731FEC046BD4602B0E6
:1076C00080BDC04680B588B000AF786039603A1C94
:1076D0000832314B111C1A1C1023081C111C1A1CD7
:1076E00004F056F97B68002B02D03B68002B01D1D7
:1076F0000E234CE07B68012252429A823B681A6852
:107700007B689A617B6800229A757B683A1C083214
:10771000101C191CFFF7A2FD031CFB61FB69002B69
:1077200001D0FB6933E07B681A783B1C18339A70F0
:107730003B1C183301221A807B6802333A1C183232
:107740000120111C1A1CFFF751FD031CFB61FB6992
:10775000002B01D0FB691AE07A683B68101C191CE9
:10776000FFF714FE031CFB61FB69002B01D0FB69D2
:107770000DE07A683B68101C191CFFF7D3FE031C50
:10778000FB61FB69002B01D0FB6900E00023181CA2
:10779000BD4608B080BDC046B02E020080B588B09E
:1077A00000AFF860B960BB1D1A80FB68002B01D1E7
:1077B0000E2334E0FB689A8A1B4B9A4206D0FB6882
:1077C0009B7D01225340DBB2002B01D0082326E031
:1077D000BB1D1B88142B01D9072320E03B1C103351
:1077E000181C0021102204F015F9FB689A893B1C33
:1077F00010331A803B1C1033BA68DA603B1C10331C
:10780000BA1D9A603B1C103301229A70FB689A8A59
:107810003B1C1033101C191CFFF700FD031C181C27
:10782000BD4608B080BDC046FFFF000070DF704756
:10783000181CC04671DF7047181CC04672DF7047C5
:10784000181CC04673DF7047181CC04674DF7047B1
:10785000181CC04675DF7047181CC04676DF70479D
:10786000181CC04677DF7047181CC04678DF704789
:10787000181CC04679DF7047181CC0467ADF704775
:10788000181CC0467BDF7047181CC0467CDF704761
:10789000181CC0467DDF7047181CC0467EDF70474D
:1078A000181CC0467FDF7047181CC04680DF704739
:1078B000181CC04681DF7047181CC04682DF704725
:1078C000181CC04683DF7047181CC04684DF704711
:1078D000181CC046B0DF7047181CC046B1DF7047A7
:1078E000181CC046B2DF7047181CC04690DF7047B6
:1078F000181CC04691DF7047181CC04692DF7047C5
:10790000181CC04693DF7047181CC04694DF7047B0
:10791000181CC04695DF7047181CC04696DF70479C
:10792000181CC04697DF7047181CC04698DF704788
:10793000181CC046A0DF7047181CC046A1DF704766
:10794000181CC046A2DF7047181CC046A3DF704752
:10795000181CC046A4DF7047181CC046A5DF70473E
:10796000181CC046A6DF7047181CC046A7DF70472A
:10797000181CC046A8DF7047181CC046A9DF704716
:10798000181CC046AADF7047181CC04660DF70474D
:10799000181CC04661DF7047181CC04662DF704784
:1079A000181CC04663DF7047181CC04664DF704770
:1079B000181CC04665DF7047181CC04666DF70475C
:1079C000181CC04667DF7047181CC04668DF704748
:1079D000181CC04669DF7047181CC04680B582B0CD
:1079E00000AF021C3960BB1D1A80BB1D1B88DAB2B8
:1079F0003B681A703B680133BA1D1288120A92B2B2
:107A0000D2B21A700223181CBD4602B080BDC04617
:107A100080B588B000AFF860B9607A603B1C1C3359
:107A20007A6812781A703B1C1C331B7802331F2BA8
:107A300004DCFB685B7802331F2B01DD0C237DE047
:107A40003B1C1C331B789AB23B1C1E331D218A1A27
:107A50001A803B1C16333A1C1E3212881A803B1CBB
:107A60001C331B780233BA68D2183B1C1633101C27
:107A7000191CFFF70FFF031CBB61BB69002B01D072
:107A8000BB695BE0FB681B78022B12D13B1C1633F1
:107A90001B883A1C1E3212889A420AD33B1C1D33A3
:107AA00009221A703B1C1E333A1C163212881A80A7
:107AB0001AE03B1C1D3308221A70FB685B78002B10
:107AC0000CD0FB685B783A1C1E3212889A4205D3B0
:107AD000FB685A783B1C1E331A8005E03B1C1E33A2
:107AE0003A1C163212881A803B1C1C331B783A1C35
:107AF0001C32591C1170BA68D3183A1C1E321288F5
:107B0000D2B20132D2B21A703B1C1C331B783A1C21
:107B10001C32591C1170BA68D3183A1C1D321278E5
:107B20001A707B681A783B1C1E331B88DBB2D31893
:107B3000DBB20233DAB27B681A700023181CBD4630
:107B400008B080BD90B585B000AF786039603B6803
:107B50001B7804331F2B01DD0C2332E03B1C0A335E
:107B6000181CFFF787FE031CFB60FB68002B01D08D
:107B7000FB6826E03B681B785A1CD1B23A6811704A
:107B80007A68D31803221A703B681B785A1CD1B24A
:107B90003A6811707A68D31819221A703B681C78F9
:107BA0003B1C0A331A883B681B787968CB18101C79
:107BB000191CFFF713FF031CE318DAB23B681A70B5
:107BC0000023181CBD4605B090BDC04680B584B0EA
:107BD00000AFF8607A603B603B1C0B330A1C1A70E4
:107BE000FB685B68002B01D107233AE03B681B78F8
:107BF0009A1CFB681B88D3181F2B01DD0C2330E077
:107C00003B681B785A1CD1B23A6811707A68D31855
:107C1000FA681288D2B20132D2B21A703B681B786D
:107C20005A1CD1B23A6811707A68D3183A1C0B32D8
:107C300012781A703B681B787A68D118FB685A680A
:107C4000FB681B88081C111C1A1C03F0A1FE3B6872
:107C50001A78FB681B88DBB2D318DAB23B681A705B
:107C60000023181CBD4604B080BDC04680B584B05A
:107C700000AFB9607A603B1C0F33021C1A707B683E
:107C80001B7803331F2B01DD0C2320E07B681B785E
:107C90005A1CD1B27A681170BA68D31802221A70CD
:107CA0007B681B785A1CD1B27A681170BA68D318F5
:107CB0000A221A707B681B785A1CD1B27A6811703C
:107CC000BA68D3183A1C0F3212781A700023181CA5
:107CD000BD4604B080BDC04680B58AB000AFF86034
:107CE0007B603B1C0B3319703B1C0A331A703B1C26
:107CF000233300221A703B1C22333A6B12781A701D
:107D000000237B627EE0FB685A687B6A9B00D31885
:107D10003A1C1432111C1A1C0423081C111C1A1CB6
:107D200003F036FE3A1C14323B1C1A33101C191C8B
:107D30000022FFF73FFE031CFB61FB69002B01D013
:107D4000FB697BE03B1C1A331B783A1C0A32127821
:107D50009A4254D13B1C23331B78002B01D00023C3
:107D600000E002233A1C1B3213703B6B1B781A1C79
:107D70003B1C1A331B78D2183B1C1B331B78D318BF
:107D80001F2B01DD0C2359E03B1C23331B78012200
:107D90005340DBB2002B15D03B6B1B780133DAB2BA
:107DA0003B6B1A703B6B1B785A1CD1B23A6B11704B
:107DB0007A68D3183A1C0B3212781A703B1C2333A2
:107DC00001221A703B6B1B787A68D318391C143166
:107DD0003A1C1A32081C111C1A1CFFF7EBFD031C7D
:107DE000FB61FB69002B01D0FB6927E03B6B1A7834
:107DF0003B1C1A331B78D318DAB23B6B1A707B6AC0
:107E000001337B62FB681B881A1C7B6A9A4200DD87
:107E100079E73B1C23331B78002B0ED03B1C22330D
:107E20001B787A68D3183A6B11783A1C2232127890
:107E30008A1AD2B2013AD2B21A700023181CBD4677
:107E40000AB080BD80B588B002AFF8607B603B1C93
:107E50000B3319703B1C0A331A70F9683B1C0B3347
:107E60001A787B68386A0090081C111C0222FFF700
:107E700033FF031C7B617B69002B01D07B6913E01E
:107E8000F9683B1C0A331A787B68386A0090081C32
:107E9000111C1022FFF720FF031C7B617B69002B64
:107EA00001D07B6900E00023181CBD4606B080BDF0
:107EB00080B582B000AF78607B681B88052B0AD93B
:107EC0007B681A88C8231B019A4206D97B681A88E6
:107ED000164B9A4201D0072323E07B685B88052B71
:107EE0000AD97B685A88C8231B019A4206D97B6845
:107EF0005A880E4B9A4201D0072312E07B681A88F9
:107F00000A4B9A420CD07B685A88084B9A4207D099
:107F10007B681A887B685B889A4201D9072300E056
:107F20000023181CBD4602B080BDC046FFFF000004
:107F300090B587B000AFF860B9607A607B681B7855
:107F400006331F2B01D90C2341E0FB68181CFFF7F7
:107F5000AFFF031C7B617B69002B01D07B6936E09E
:107F60007B681B785A1CD1B27A681170BA68D31832
:107F700005221A707B681B785A1CD1B27A6811707E
:107F8000BA68D31812221A707B681C78FB681A88AA
:107F90007B681B78B968CB18101C191CFFF71EFDF5
:107FA000031CE318DAB27B681A707B681C78FB68E4
:107FB0005A887B681B78B968CB18101C191CFFF70E
:107FC0000DFD031CE318DAB27B681A700023181C3D
:107FD000BD4607B090BDC04690B587B000AFF86011
:107FE000B9607A60FB689B88DAB23B1C17330232B7
:107FF0001A707B681B789A1C3B1C17331B78D318AC
:108000001F2B01DD0C2349E07B681B785A1CD1B281
:108010007A681170BA68D3183A1C17321278013294
:10802000D2B21A707B681B785A1CD1B27A68117070
:10803000BA68D318FF221A707B681C78FB681A880C
:108040007B681B78B968CB18101C191CFFF7C6FC9D
:10805000031CE318DAB27B681A70FB689B88002B5C
:108060001BD0FB689B68002B01D1072316E07B68BF
:108070001B78BA68D118FB689A68FB689B88081C53
:10808000111C1A1C03F084FC7B681A78FB689B881F
:10809000DBB2D318DAB27B681A700023181CBD4615
:1080A00007B090BD90B589B000AFF860B9607A6054
:1080B000FB681B6B002B01D107236FE03B1C1F33B8
:1080C00000221A7061E0FB68196B3B1C1F331A78A1
:1080D000131C5B009B189B00CB18BB61BB699B8882
:1080E000DAB23B1C173302321A707B681B785A1CB9
:1080F000D1B27A681170BA68D3183A1C1732127864
:108100000132D2B21A707B681B785A1CD1B27A68DD
:108110001170BA68D31816221A707B681C78BB6974
:108120001A887B681B78B968CB18101C191CFFF7DC
:1081300055FC031CE318DAB27B681A70BB699B8894
:10814000002B1BD0BB699B68002B01D1072325E0C6
:108150007B681B78BA68D118BB699A68BB699B8831
:10816000081C111C1A1C03F013FC7B681A78BB69ED
:108170009B88DBB2D318DAB27B681A703B1C1F33C2
:108180001A783B1C1F3301321A70FA683423D35C0F
:108190003A1C1F3212789A4295D30023181CBD4610
:1081A00009B090BD80B588B002AFF860B9607A6060
:1081B00000237B617B6800221A70FB681B78002B10
:1081C0000ED0F968BA687B68081C111C1A1CFFF7EE
:1081D0001FFC031C7B617B69002B01D07B69B8E02D
:1081E000FB689B78002B0CD0BA687B68101C191CAC
:1081F000FFF7A8FC031C7B617B69002B01D07B6926
:10820000A7E0FB689B88002B0ED0FB68191DBA689D
:108210007B68081C0121FFF7D9FC031C7B617B698B
:10822000002B01D07B6994E0FB68DB68002B11D048
:10823000FB68DB681B7859B2BA687B68081C111CA4
:108240001A1CFFF713FD031C7B617B69002B01D017
:108250007B697EE0FB681B8A002B11D0FB681A1C2F
:108260001032BB6879680091101C02210622FFF7CA
:10827000E9FD031C7B617B69002B01D07B6968E011
:10828000FB681B8B002B11D0FB681A1C1832BB68D3
:1082900079680091101C03210722FFF7D3FD031C0E
:1082A0007B617B69002B01D07B6952E0FB681B8CF2
:1082B000002B11D0FB681A1C2032BB687968009132
:1082C000101C14211522FFF7BDFD031C7B617B6987
:1082D000002B01D07B693CE0FB689B6A002B0FD030
:1082E000FB68996ABA687B68081C111C1A1CFFF7A6
:1082F0001FFE031C7B617B69002B01D07B6928E09A
:10830000FB68DB6A002B0FD0FB68D96ABA687B6810
:10831000081C111C1A1CFFF75FFE031C7B617B69A4
:10832000002B01D07B6914E0FA683423D35C002B66
:108330000ED0F968BA687B68081C111C1A1CFFF77C
:10834000B1FE031C7B617B69002B01D07B6900E0DF
:108350007B69181CBD4606B080BDC04680B582B0A2
:1083600000AF78607B689B88002B0AD07B689B6895
:10837000002B06D07B689B681B781A1C04231340D3
:1083800001D1072300E00023181CBD4602B080BDC8
:1083900080B582B000AF78607B689B88002B01D0ED
:1083A000072300E00023181CBD4602B080BDC04674
:1083B00080B596B000AF786039603B1C4B3300222B
:1083C0001A703B1C4A3300221A707B68002B1FD0A6
:1083D0007B68181CFFF7C2FF031CFB64FB6C002BBF
:1083E00001D0FB6C46E079683A1C28323B1C4B33C9
:1083F000081C111C1A1CFFF7D5FE031CFB64FB6C48
:10840000002B01D0FB6C35E03B1C28337B6501E081
:1084100000237B653B68002B1FD03B68181CFFF7CF
:10842000B7FF031CFB64FB6C002B01D0FB6C21E04D
:1084300039683A1C08323B1C4A33081C111C1A1CB0
:10844000FFF7B0FE031CFB64FB6C002B01D0FB6C40
:1084500010E03B1C08333B6501E000233B653B1CFF
:108460004B3319783B1C4A331B78786D3A6DFFF714
:10847000E5F9031C181CBD4616B080BD70DF7047BF
:10848000181CC04671DF7047181CC04672DF704769
:10849000181CC04673DF7047181CC04674DF704755
:1084A000181CC04675DF7047181CC04676DF704741
:1084B000181CC04677DF7047181CC04678DF70472D
:1084C000181CC04679DF7047181CC0467ADF704719
:1084D000181CC0467BDF7047181CC0467CDF704705
:1084E000181CC0467DDF7047181CC0467EDF7047F1
:1084F000181CC0467FDF7047181CC04680DF7047DD
:10850000181CC04681DF7047181CC04682DF7047C8
:10851000181CC04683DF7047181CC04684DF7047B4
:10852000181CC046B0DF7047181CC046B1DF70474A
:10853000181CC046B2DF7047181CC04690DF704759
:10854000181CC04691DF7047181CC04692DF704768
:10855000181CC04693DF7047181CC04694DF704754
:10856000181CC04695DF7047181CC04696DF704740
:10857000181CC04697DF7047181CC04698DF70472C
:10858000181CC046A0DF7047181CC046A1DF70470A
:10859000181CC046A2DF7047181CC046A3DF7047F6
:1085A000181CC046A4DF7047181CC046A5DF7047E2
:1085B000181CC046A6DF7047181CC046A7DF7047CE
:1085C000181CC046A8DF7047181CC046A9DF7047BA
:1085D000181CC046AADF7047181CC04660DF7047F1
:1085E000181CC04661DF7047181CC04662DF704728
:1085F000181CC04663DF7047181CC04664DF704714
:10860000181CC04665DF7047181CC04666DF7047FF
:10861000181CC04667DF7047181CC04668DF7047EB
:10862000181CC04669DF7047181CC04680B582B070
:1086300000AF78607B681B781A1C7B6801331B785D
:108640001B029BB213439BB29BB2181CBD4602B0E7
:1086500080BDC04690B585B000AF78603C1C0E343C
:108660007B68181CFFF7E2FF031C23803B1C0E33C2
:108670001A88012313405A1E9341DBB2181CBD46D1
:1086800005B090BD80B582B000AF78607B685A8835
:10869000084B1B889A4207D37B685A88054B5B8836
:1086A0009A4201D8012300E00023181CBD4602B005
:1086B00080BDC0462C2C002080B586B000AF78600D
:1086C000294B1A88294B9A424BD0294B1B780133EE
:1086D000DAB2274B1A70274B1A7B254B1B789A422C
:1086E00016D3214B1A88244B101C191CFFF7DAFEF5
:1086F000031C7B617B69002B09D01E4B9B69002BFF
:1087000005D01C4B9B697A69101C984729E028E02A
:10871000174B00221A70174B1B7C002B13D0124BE7
:108720001B88181C3B21FFF7C1FE031C3B613B6902
:10873000002B08D00F4B9B69002B04D00D4B9B697D
:108740003A69101C98470B4B5B69002B09D03B1C06
:108750000C3300221A70074B5B693A1C0C32101C58
:108760009847BD4606B080BD362C0020FFFF0000B4
:10877000342C0020102C00202C2C002090B585B02B
:1087800000AF7860214B7A6813CA13C313CA13C3AE
:1087900012681A601E4B00221A707B681B68002B3F
:1087A00015D07B681B681B4A111C1A1C0823081C67
:1087B000111C1A1C03F0ECF8164B181CFFF786FE70
:1087C000031CFB60FB68002B0CD0FB6819E0114B0D
:1087D000181CFFF77FFE031CFB60FB68002B01D019
:1087E000FB680EE00C4B012252421A800B4B002218
:1087F0001A700B4A0B4B101C00211A1C01F070FD63
:10880000031C181CBD4605B090BDC046102C0020AE
:10881000442C00202C2C0020362C0020342C00204E
:10882000402C0020B986010080B500AF044B1B68C6
:10883000181C01F013FE031C181CBD4680BDC04669
:10884000402C002080B584B000AF284B181CFFF7E7
:1088500019FF031C01225340DBB2002B33D0244B01
:108860001B78002B0CD0234B5B69002B2AD03B1DBF
:1088700000221A701F4B5B693A1D101C98472EE0AE
:108880001D4B1B78002B03D11A4B5B68FB6002E089
:10889000184B9B68FB60194B1A68FB68101C191C6D
:1088A000002201F095FD031CBB60BB68002B09D0C2
:1088B000104B9B69002B05D00E4B9B69BA68101CAE
:1088C00098470CE00BE00B4B5B69002B07D03B1C7F
:1088D00001221A70074B5B693A1C101C9847044B25
:1088E00000221A70BD4604B080BDC046382C00205E
:1088F000442C0020102C0020342C0020402C002080
:1089000080B582B000AF78607B689A880B4B1A8084
:108910000B497A680E23D2180823081C111C1A1C54
:1089200003F036F8074B00221A70074BDB89002B47
:1089300001D1FFF787FFBD4602B080BD362C002075
:10894000382C0020342C0020102C002080B584B05E
:1089500000AF78600E4B012252421A800D4B00226C
:108960001A700D4B1B68181C01F078FD031CFB608E
:10897000FB68002B08D0094B9B69002B04D0074BE8
:108980009B69FA68101C9847BD4604B080BDC0467C
:10899000362C0020342C0020402C0020102C0020ED
:1089A00080B584B000AF78607B680633FB60FB68FD
:1089B0001A88144BDB899A4221D1FB681B8B022B4E
:1089C0001DD1FB681A33181CFFF744FE031C002B53
:1089D00002D0FFF737FF12E00B4B1B68181C01F0A9
:1089E0003DFD031CBB60BB68002B08D0054B9B6999
:1089F000002B04D0034B9B69BA68101C9847BD46F6
:108A000004B080BD102C0020402C002080B582B026
:108A100000AF786007497A680623D2180823081C3B
:108A2000111C1A1C02F0B4FFFFF70CFFBD4602B088
:108A300080BDC046382C002080B582B000AF786081
:108A40007B681B88112B0DD002DC102B05D018E0A1
:108A5000122B11D0502B0AD013E07B68181CFFF7A3
:108A60004FFF0EE07B68181CFFF770FF09E07B6882
:108A7000181CFFF795FF04E07B68181CFFF7C6FF82
:108A8000C046BD4602B080BD80B584B000AF7860FE
:108A9000204A7B68111C1A1C0823081C111C1A1C74
:108AA00002F076FF1B4B181CFFF710FD031CFB6048
:108AB000FB68002B29D1184B181CFFF7E3FD031CA2
:108AC00001225340DBB2002B0FD0144B01221A704D
:108AD000134B1A880F4B101C191CFFF7E3FC031CE7
:108AE000FB60104B01221A700FE00F4B5B69002BEB
:108AF00009D03B1C083301221A700B4B5B693A1CEE
:108B00000832101C98470023FB60FB68181CBD4608
:108B100004B080BD2C2C0020382C0020442C0020D8
:108B2000362C0020342C0020102C002023DF70472E
:108B3000181CC04624DF7047181CC04625DF70474C
:108B4000181CC04626DF7047181CC04627DF704738
:108B5000181CC04628DF7047181CC04629DF704724
:108B6000181CC0462ADF7047181CC0462BDF704710
:108B7000181CC0462CDF7047181CC0462DDF7047FC
:108B8000181CC0462EDF7047181CC0462FDF7047E8
:108B9000181CC04630DF7047181CC04631DF7047D4
:108BA000181CC04632DF7047181CC04635DF7047BE
:108BB000181CC04636DF7047181CC04633DF7047AC
:108BC000181CC04634DF7047181CC04637DF70479A
:108BD000181CC04638DF7047181CC04639DF704784
:108BE000181CC0463ADF7047181CC0463BDF704770
:108BF000181CC0463CDF7047181CC0463DDF70475C
:108C0000181CC0463EDF7047181CC0463FDF704747
:108C1000181CC04641DF7047181CC04642DF704731
:108C2000181CC04643DF7047181CC04640DF704721
:108C3000181CC04644DF7047181CC04645DF70470B
:108C4000181CC04646DF7047181CC04647DF7047F7
:108C5000181CC04648DF7047181CC04649DF7047E3
:108C6000181CC0464ADF7047181CC0464BDF7047CF
:108C7000181CC0464CDF7047181CC0464DDF7047BB
:108C8000181CC04651DF7047181CC04652DF7047A1
:108C9000181CC04621DF7047181CC04620DF7047F3
:108CA000181CC04622DF7047181CC0464EDF7047B4
:108CB000181CC0464FDF7047181CC04650DF704775
:108CC000181CC04610DF7047181CC04611DF7047E3
:108CD000181CC04612DF7047181CC04613DF7047CF
:108CE000181CC04680B582B000AF78607A68032354
:108CF00013405A425341DBB2181CBD4602B080BD3E
:108D000070DF7047181CC04671DF7047181CC046E2
:108D100072DF7047181CC04673DF7047181CC046CE
:108D200074DF7047181CC04675DF7047181CC046BA
:108D300076DF7047181CC04677DF7047181CC046A6
:108D400078DF7047181CC04679DF7047181CC04692
:108D50007ADF7047181CC0467BDF7047181CC0467E
:108D60007CDF7047181CC0467DDF7047181CC0466A
:108D70007EDF7047181CC0467FDF7047181CC04656
:108D800080DF7047181CC04681DF7047181CC04642
:108D900082DF7047181CC04683DF7047181CC0462E
:108DA00084DF7047181CC046B0DF7047181CC046EF
:108DB000B1DF7047181CC046B2DF7047181CC046B0
:108DC00090DF7047181CC04691DF7047181CC046E2
:108DD00092DF7047181CC04693DF7047181CC046CE
:108DE00094DF7047181CC04695DF7047181CC046BA
:108DF00096DF7047181CC04697DF7047181CC046A6
:108E000098DF7047181CC046A0DF7047181CC0468A
:108E1000A1DF7047181CC046A2DF7047181CC0466F
:108E2000A3DF7047181CC046A4DF7047181CC0465B
:108E3000A5DF7047181CC046A6DF7047181CC04647
:108E4000A7DF7047181CC046A8DF7047181CC04633
:108E5000A9DF7047181CC046AADF7047181CC0461F
:108E600060DF7047181CC04661DF7047181CC046A1
:108E700062DF7047181CC04663DF7047181CC0468D
:108E800064DF7047181CC04665DF7047181CC04679
:108E900066DF7047181CC04667DF7047181CC04665
:108EA00068DF7047181CC04669DF7047181CC04651
:108EB00080B584B000AFF8607A603B1C0A330A1CAE
:108EC0001A803B1C0A331A887B68101C191CFDF79A
:108ED0007BFBBD4604B080BD80B584B000AF3D4B88
:108EE0001B78DBB201225340DBB2002B00D06DE0D7
:108EF000394B1A683B1C0F3351424A411A70374BA9
:108F00001A683B1C0E3351424A411A703B1C0F3306
:108F10001B7801225340DBB2002B1DD03B1D181CD7
:108F2000FFF7B0FE031CBB60BB68052B04D13B1CE4
:108F30000F3301221A700FE0BB68002B07D0BA680C
:108F4000274B101C69211A1CFDF732FB04E0224B51
:108F50001B687A68101C98473B1C0E331B78012253
:108F60005340DBB2002B25D01E4B1A88BB1C1A8045
:108F70001D4B1A68BB1C101C191CFFF775FF031C46
:108F8000BB60BB68052B04D13B1C0E3301221A7059
:108F900010E0BB68002B07D0BA68114B101C802171
:108FA0001A1CFDF705FB05E00C4B1A680E4B1B68FD
:108FB000181C90473B1C0F331B78002B05D03B1C23
:108FC0000E331B78002B00D000E09FE7BD4604B0B5
:108FD00080BDC046522C0020582C0020542C00206C
:108FE000C02E0200502C00204C2C002080B586B0F2
:108FF00000AFF860B9603B60BB1D1A80BB68002BF6
:1090000001D1072329E0BB68181CFFF76BFE031C86
:1090100001225340DBB2002B01D007231DE0114B8E
:10902000BA681A60104BBA1D12881A800F4B3A6842
:109030001A60FA680E4B101C191CFFF743FE031C44
:109040007B617B69002B01D07B6906E0094B012223
:109050001A701620FFF776FD031C181CBD4606B0DB
:1090600080BDC0464C2C0020502C0020482C0020F5
:10907000B18E0100522C002080B582B000AFFFF706
:1090800025FE031C7B607B685A1E9341DAB2034BBA
:109090001A707B68181CBD4602B080BD522C00209F
:1090A00080B582B000AF78607B68002B01D10E23C1
:1090B00003E0044B7A681A600023181CBD4602B016
:1090C00080BDC046542C002080B582B000AF7860CF
:1090D0007B68002B01D10E2303E0044B7A681A60F1
:1090E0000023181CBD4602B080BDC046582C00208D
:1090F00080B582B000AF0F4B1B68002B14D00D4B16
:109100001B689847031C7B607B683B603B68002BB7
:1091100009D0396899235A00074B081C111C1A1CE6
:10912000FDF746FA02E001E0FFF7D6FEBD4602B0C9
:1091300080BDC046482C0020C02E020080B582B001
:1091400000AF78607A68032313405A425341DBB280
:10915000181CBD4602B080BD80B582B000AF021CB5
:10916000FB1D1A70064BFA1D1278111C1F220A40B3
:109170000121081C9040021C1A60BD4602B080BD4F
:1091800000E100E080B582B000AF021CFB1D1A7048
:10919000074AFB1D1B78191C1F230B400121081CCB
:1091A0009840031C191C8023D150BD4602B080BDDD
:1091B00000E100E080B582B000AF021CFB1D1A7018
:1091C000084AFB1D1B78191C1F230B400121081C9A
:1091D0009840031C191C80235B00D150BD4602B08F
:1091E00080BDC04600E100E080B582B000AF021C47
:1091F000FB1D1A70084AFB1D1B78191C1F230B400E
:109200000121081C9840031C191CC0235B00D1508D
:10921000BD4602B080BDC04600E100E0B0B582B0FE
:1092200000AF021C3960FB1D1A70FB1D1B787F2BE1
:1092300032D93049FB1D1B781A1C0F231340083B01
:1092400098082C4AFB1D1B781C1C0F232340083B4D
:109250009B0806339B00D3185B68FA1D1278141C18
:1092600003222240D200FF24251C95402A1CD24311
:109270001A403B689C01FF231C40FB1D1B781D1CF2
:1092800003232B40DB00251C9D402B1C1A43831D10
:109290009B00CB185A6029E0174BFA1D127852B286
:1092A00092081549F81D007840B28008C03080004F
:1092B0004158F81D0078041C03202040C000FF2402
:1092C000251C8540281CC043084039688C01FF21BB
:1092D0000C40F91D09780D1C03212940C900251CEB
:1092E0008D40291C0143C0329200D150BD4602B0CE
:1092F000B0BDC04600ED00E000E100E080B582B006
:1093000000AF021CFB1D1A70FB1D1B787F2B16D9AA
:10931000164AFB1D1B78191C0F230B40083B9B08AA
:1093200006339B00D3185A68FB1D1B78191C0323B6
:109330000B40DB00DA40FF2313409B0911E00C4B8C
:10934000FA1D127852B29208C0329200D258FB1D18
:109350001B78191C03230B40DB00DA40FF2313406A
:109360009B09181CBD4602B080BDC04600ED00E060
:1093700000E100E023DF7047181CC04624DF70477F
:10938000181CC04625DF7047181CC04626DF7047F2
:10939000181CC04627DF7047181CC04628DF7047DE
:1093A000181CC04629DF7047181CC0462ADF7047CA
:1093B000181CC0462BDF7047181CC0462CDF7047B6
:1093C000181CC0462DDF7047181CC0462EDF7047A2
:1093D000181CC0462FDF7047181CC04630DF70478E
:1093E000181CC04631DF7047181CC04632DF70477A
:1093F000181CC04635DF7047181CC04636DF704762
:10940000181CC04633DF7047181CC04634DF704755
:10941000181CC04637DF7047181CC04638DF70473D
:10942000181CC04639DF7047181CC0463ADF704729
:10943000181CC0463BDF7047181CC0463CDF704715
:10944000181CC0463DDF7047181CC0463EDF704701
:10945000181CC0463FDF7047181CC04641DF7047EC
:10946000181CC04642DF7047181CC04643DF7047D7
:10947000181CC04640DF7047181CC04644DF7047C8
:10948000181CC04645DF7047181CC04646DF7047B1
:10949000181CC04647DF7047181CC04648DF70479D
:1094A000181CC04649DF7047181CC0464ADF704789
:1094B000181CC0464BDF7047181CC0464CDF704775
:1094C000181CC0464DDF7047181CC04651DF70475E
:1094D000181CC04652DF7047181CC04621DF704779
:1094E000181CC04620DF7047181CC04622DF70479A
:1094F000181CC0464EDF7047181CC0464FDF70472F
:10950000181CC04650DF7047181CC04680B582B09A
:1095100000AF7860C046C046C046C046C046C046A0
:10952000C046C046C046C046C046C046C046C0460B
:109530007B68013B7B60002BECD1BD4602B080BD57
:1095400080B582B000AF0C4B5B68DB05DB0D7B6048
:109550007B68002B0BD07B68103B3B603B68DBB229
:109560005BB2181CFFF7CAFE031CDBB200E0042349
:10957000181CBD4602B080BD00ED00E080B582B091
:1095800000AF7860054AA123DB007968D150112033
:109590000321FFF743FEBD4602B080BD001001402D
:1095A00080B500AF0E4AD1239B0080214902D150E3
:1095B0000B4AC1239B0080214902D1501120FFF7A3
:1095C00013FE1120FFF7C8FD054B01221A602F2062
:1095D000FFF79CFF034B01221A70BD4680BDC046B9
:1095E00000100140842C002080B500AF1120FFF74F
:1095F000C9FD104AD2239B0080214902D1500D4A57
:10960000C2239B0080214902D1500A4B01225A609B
:109610002F20FFF77BFF074B01229A60064B0022A9
:109620001A602F20FFF772FF044B00221A70BD460C
:1096300080BDC04600100140702C0020842C00200A
:1096400080B500AF024A034BD358181CBD4680BDFD
:10965000001001400405000080B582B000AF7860C2
:1096600039607A683B68D31A1B021B0A181CBD4676
:1096700002B080BD80B582B000AF7860034AA823F5
:10968000DB007968D150BD4602B080BD00100140BA
:1096900080B586B000AF78604C4B19687A68131CAF
:1096A000DB009B189B00CB18BB60494B1B68013348
:1096B00003D1474B7A681A6084E0BB685968434B12
:1096C0001868434B1A68131CDB009B189B00C318D7
:1096D0005B6899421ED83D4B19683D4B1A68131CB4
:1096E000DB009B189B00CA18384B1868384B196868
:1096F0000B1CDB005B189B00C3185968BB685B68D8
:10970000CB1A5360324B1A68BB681A62304B7A68C6
:109710001A6057E0BB685B68FB602D4B1B687B6180
:109720002B4B1B683B6117E0284B19683A69131CE7
:10973000DB009B189B00CB185B68FA68D31AFB60B0
:109740003B697B61214B19683A69131CDB009B184C
:109750009B00CB181B6A3B613B6901330BD01B4B51
:1097600019683A69131CDB009B189B00CB185A68D8
:10977000FB689A42D8D33B69013313D0134B196865
:109780003A69131CDB009B189B00CA180F4B186822
:1097900039690B1CDB005B189B00C3185968FB6818
:1097A000CB1A5360BB68FA685A60BB683A691A62A0
:1097B000064B19687A69131CDB009B189B00CB18B9
:1097C0007A681A62BD4606B080BDC046602C002093
:1097D0006C2C002080B586B000AF7860394B1B68D8
:1097E0007B617B693B6110E03A697B689A4200D1FA
:1097F0000EE03B697B61344B19683A69131CDB004E
:109800009B189B00CB181B6A3B613B690133EBD172
:109810003B69013300D152E07A693B699A4211D128
:10982000294B1968274B1A68131CDB009B189B00F7
:10983000CB181A6A234B1A60224B1B68013301D1E3
:10984000FFF7D2FE204B19683A69131CDB009B1806
:109850009B00CB185B68FB601B4B19687A69131C73
:10986000DB009B189B00CA18174B186839690B1C42
:10987000DB005B189B00C3181B6A1362124B19684C
:109880007A69131CDB009B189B00CB181B6A3B6199
:109890003B69013313D00C4B19683A69131CDB0088
:1098A0009B189B00CA18084B186839690B1CDB0011
:1098B0005B189B00C3185968FB68CB185360BD4602
:1098C00006B080BD6C2C0020602C002080B500AF5D
:1098D0001120FFF76FFCBD4680BDC04680B500AFCC
:1098E0001420FFF767FCBD4680BDC04680B584B03C
:1098F00000AF7860144B1B68002B1BD0124B1A680A
:109900007B6899697B68DB69081C191C9047031CFC
:10991000FB60FB68BB60BB68002B0AD0B96864239E
:109920001A1CFF32094B081C111C1A1CFCF740FEC4
:1099300006E005E07B689A697B68DB69181C904744
:10994000BD4604B080BDC046802C0020082F020018
:1099500080B584B000AF2B4B1B6801334FD0002380
:109960007B60FFF76DFE021C274B1B68101C191C47
:10997000FFF772FE031CBB60224B1B68FB601FE0FD
:10998000224B1968FA68131CDB009B189B00CB184C
:109990003B603B685A68BB689A4200D913E03B6859
:1099A0005B68BA68D31ABB603B685B687A68D31897
:1099B0007B603B681B6AFB603B68181CFFF796FFE7
:1099C000FB680133DCD1124B1A78124B1B789A4298
:1099D0000CD1104B1B780133DAB20E4B1A700D4BC1
:1099E0001B78022B02D10B4B00221A70094B1B78FB
:1099F0001A1C094B92007968D150FFF76FFFBD46E2
:109A000004B080BD6C2C0020702C0020602C002045
:109A10007C2C00207D2C0020742C002080B582B08E
:109A200000AF7860184B1A78184B1B789A4223D0F5
:109A3000154B1B780133DAB2134B1A70124B1B789B
:109A4000022B02D1104B00221A700F4B1B781A1CEC
:109A50000F4B9200D2587B681A607B681A680D4BD6
:109A60001B68D2180B4B1A600A4B1B681B021A0AA0
:109A7000084B1A60012303E07B6800221A60002370
:109A8000181CBD4602B080BD7C2C00207D2C00201F
:109A9000742C0020702C002080B586B000AF434BA2
:109AA0001B683B613B1C1733414A12781A7068E00F
:109AB000404B1A683B1C17331B78DB00D318FB6044
:109AC0003B1C1633FA6812781A7053E0FB68596829
:109AD0003B1C16331A78131C5B009B18DB00CB1859
:109AE000BB603B1C16331A783B1C163301321A70CC
:109AF000FB689B783A1C163212789A4203D13B1CC1
:109B0000163300221A70BB681B78022B02D0032B7D
:109B10002AD02FE0284B1968BB685A68131CDB0059
:109B20009B189B00CB187B607B681B7D002B08D0AB
:109B3000BB685B68181CFFF74DFE7B6800221A7536
:109B400018E017E01C4B1968184B1A68131CDB004F
:109B50009B189B00CB183B603B6800221A753B6842
:109B60001A6A124B1A6000E0C046104B1B680133A2
:109B7000E8D1C046FB685B783A1C163212789A42EC
:109B8000A4D13B1C17331B783A1C1732591E117095
:109B9000002B8DD1054B1A683B69D31A5A1E93418D
:109BA000DBB2181CBD4606B080BDC0466C2C002040
:109BB000642C0020682C0020602C002080B588B028
:109BC00000AFF860B9607A600023FB6142E0254B8A
:109BD0001968254B1A68131CDB009B189B00CB18D7
:109BE000BB61BB695A68FB689A4206D9BB695A686F
:109BF000FB68D21ABB695A6030E0BB695B68FA68DF
:109C0000D31AFB60BB695B68FA69D318FB61BB6957
:109C100000225A60BB6900221A75134B1B687B61D6
:109C2000BB691A6A104B1A60BB691B69002B11D003
:109C3000BA68FB69D3181B021A0ABB699A60BB6930
:109C40001A69BB69DA607B681A68BB691A627B684B
:109C50007A691A60044B1B680133B8D1BD4608B05D
:109C600080BDC046602C00206C2C002080B58AB0DE
:109C700000AF7860624B1B68BB613B1C2733614AB5
:109C800012781A70A7E0604B1A683B1C27331B78C8
:109C9000DB00D3187B6193E07B6801330ED07B68D7
:109CA0003B625A4B19683A6A131CDB009B189B00F5
:109CB000CB18FB61FB691B6A7B603EE07B695968DE
:109CC0007B691B781A1C131C5B009B18DB00CB18EC
:109CD0003B617B691B780133DAB27B691A707B695F
:109CE0001A787B699B789A4202D17B6900221A70AC
:109CF0003B695B683B62454B19683A6A131CDB00A1
:109D00009B189B00CB18FB613B691B78012B03D18F
:109D1000FB691B7D002B00D052E03B699A68FB6910
:109D20009A603B69DA68FB69DA603B691A69FB692A
:109D30001A613B695A69FB69DA61FB699A68344BBD
:109D40001B68D31A1B021A0A324B9A420ED8FB69BF
:109D50009A682F4B1B68101C191CFFF77DFC021C16
:109D6000FB69DB68D218FB695A6018E0284B1A6857
:109D7000FB699B68101C191CFFF76EFC031CFB6041
:109D8000FB69DA68FB689A4206D9FB69DA68FB6806
:109D9000D21AFB695A6002E0FB6900225A60FB6933
:109DA00000229A60FB690022DA60FB6901221A75C1
:109DB000FB69012252421A623B6A181CFFF768FCD9
:109DC0007B68013300D067E77B691A787B695B7831
:109DD0009A4200D060E73B1C27331B783A1C27329D
:109DE000591E1170002B00D04DE7054B1A68BB6956
:109DF000D31A5A1E9341DBB2181CBD460AB080BD6F
:109E00006C2C0020642C0020682C0020602C00208A
:109E1000702C0020FEFF7F0090B589B000AF786005
:109E20002A4B1B6801334CD0294B1968274B1A6801
:109E3000131CDB009B189B00CB185B68FB61FFF7D2
:109E4000FFFB031CBB61234B1B687B61BA697B6909
:109E5000101C191CFFF700FC031C03333B611E4B55
:109E60001B7801225340DBB2002B01D0FFF798FB97
:109E7000FA693B69934200D2131C7A69D3187B615B
:109E80007B691B021B0A7B617B69181CFFF7F2FBD5
:109E9000FFF7D6FB031CFB60FA68BB69101C191C9A
:109EA000FFF7DAFB031CDC1C7A69BB69101C191C68
:109EB000FFF7D2FB031C9C4202D9FFF707FD02E02B
:109EC00001E0FFF791FBBD4609B090BD6C2C00206E
:109ED000602C0020702C0020842C002090B587B0CE
:109EE00000AF01235B427B601D4B1B683B611D4B38
:109EF0001B68FB603C1C0B343B1C181CFFF78EFDE1
:109F0000031C23703C1C1734FFF7C6FD031C237091
:109F10003B1C0B331B78002B0BD039683A693B1D77
:109F2000081C111C1A1CFFF749FE3B1C17330122A9
:109F30001A707B68181CFFF799FE031C002B03D0D6
:109F40003B1C173301221A703B1C17331B78002B64
:109F500003D0FB68181CFFF75FFFBD4607B090BD3C
:109F6000702C00206C2C002080B582B000AF78608F
:109F700039603B68DAB27B685A70BD4602B080BD7A
:109F800080B584B000AF786039607B685B7801335E
:109F9000FB607B689B781A1CFB689A4201D1002306
:109FA000FB607B681B781A1CFB689A4201D1002376
:109FB0000EE03B68FA681A607B6859687B685B78DA
:109FC0001A1C131C5B009B18DB00CB18BB60BB6822
:109FD000181CBD4604B080BD80B586B000AFF860E7
:109FE000B9607A603B601B4B1A68FB68DB00D218D3
:109FF0003B1C1033101C191CFFF7C2FF031C7B61B4
:10A000007B69002B01D1042320E07B6901221A70B7
:10A010007B69BA685A60FFF713FB021C7B699A6080
:10A020007B697A68DA607B693A681A617B693A6AA7
:10A030005A61084B1A68FB68DB00D2183B69101C98
:10A04000191CFFF791FFFFF749FC0023181CBD46C0
:10A0500006B080BD682C002080B584B000AF786069
:10A060003960144B1A687B68DB00D2183B1C08333C
:10A07000101C191CFFF784FF031CFB60FB68002BFE
:10A0800001D1042312E0FB6802221A70FB683A68CF
:10A090005A60084B1A687B68DB00D218BB68101C3A
:10A0A000191CFFF761FFFFF719FC0023181CBD46C0
:10A0B00004B080BD682C002080B584B000AF78600B
:10A0C000144B1A687B68DB00D2183B1C0833101C49
:10A0D000191CFFF755FF031CFB60FB68002B01D127
:10A0E000042313E0FB6803221A70FB68012252422A
:10A0F0005A60084B1A687B68DB00D218BB68101CDA
:10A10000191CFFF731FFFFF7E9FB0023181CBD46C0
:10A1100004B080BD682C002080B500AF104AA02399
:10A120005B000021D1500E4AA2235B000021D150D8
:10A130000B4AA4235B000021D150094AA6235B00EF
:10A140000021D150064A80235B000021D150044AEF
:10A1500082235B000021D150FFF7FAFBBD4680BD92
:10A160000010014080B500AFFFF7B8FEBD4680BDCE
:10A1700080B586B000AFF8607B603B1C0B33197074
:10A180003B1C0A331A707B68181CFEF7D7FF031CB0
:10A1900001225340DBB2002B01D0072389E07B680A
:10A1A000002B01D1072384E0FFF71EFA434B3A6AE4
:10A1B0001A60434B3A1C0B3212781A70414B7A6882
:10A1C0001A6000237B6116E03E4B19687A69131C04
:10A1D000DB009B189B00CB1800221A70394B1968C2
:10A1E0007A69131CDB009B189B00CB1800221A75A0
:10A1F0007B6901337B613B1C0B331A787B699A4284
:10A20000E2DC3B1C0B331A78131CDB009B189B0011
:10A210007A68D3187B602C4B03221A702B4B7A6818
:10A220001A607B6818337B6000237B6120E0274B3A
:10A230001A687B69DB00D3183B613B6900221A7006
:10A240003B6900225A703B693A1C0A3212789A70B4
:10A250003B697A685A603B1C0A331A78131C5B000E
:10A260009B18DB007A68D3187B607B6901337B61C4
:10A270007B69022BDBDD164B012252421A60154B23
:10A2800000221A70144B00221A701420FEF7ACFF43
:10A2900014200321FEF7C2FF1420FEF75DFFFB68C8
:10A2A000181CFFF76BF9FFF7CBF9021C0B4B1A6078
:10A2B0000023181CBD4606B080BDC046802C00207F
:10A2C0005C2C0020602C0020642C0020682C0020D6
:10A2D0006C2C00207C2C00207D2C0020702C002079
:10A2E00080B586B000AFF8607A603B1C0B330A1C67
:10A2F0001A70284B1B68002B01D1082346E07B68AD
:10A30000002B01D1072341E0FB68002B01D107237B
:10A310003CE000237B6132E01E4B19687A69131C14
:10A32000DB009B189B00CB181B78002B24D1194B0A
:10A3300019687A69131CDB009B189B00CB1801225B
:10A340001A70144B19687A69131CDB009B189B0068
:10A35000CB183A1C0B3212785A700E4B19687A6976
:10A36000131CDB009B189B00CB187A689A617A69F2
:10A37000FB681A60002309E07B6901337B61064BAF
:10A380001B781A1C7B699A42C6DC0423181CBD4644
:10A3900006B080BD602C00205C2C002080B582B00F
:10A3A00000AFFFF7CDF8031C012B02D0032B03D025
:10A3B00005E000237B6005E001237B6002E00223CF
:10A3C0007B60C0467B68181CBD4602B080BDC0469D
:10A3D00090B589B002AFF860B9607A601D4B1B6818
:10A3E000002B01D1082330E01B4B1B781A1CFB68A3
:10A3F0009A4202D9BB68042B01D8072325E0154BEC
:10A400001968FA68131CDB009B189B00CB181B789B
:10A41000012B01D0082318E00E4B1968FA68131CB1
:10A42000DB009B189B00CB185B78012B01D1BB682C
:10A4300000E000237B61FFF7B1FFF968BA687B6930
:10A440007C680094FFF7C8FD031C181CBD4607B0CC
:10A4500090BDC046602C00205C2C002080B582B0EE
:10A4600000AF7860134B1B68002B01D108231DE05F
:10A47000114B1B781A1C7B689A4201D8072315E000
:10A480000C4B19687A68131CDB009B189B00CB18D7
:10A490001B78012B01D0082308E0FFF77FFF021C87
:10A4A0007B68101C191CFFF7D7FD031C181CBD4648
:10A4B00002B080BD602C00205C2C002080B500AF75
:10A4C000074B1B68002B01D1082306E0FFF766FF4E
:10A4D000031C181CFFF7F0FD031C181CBD4680BDB3
:10A4E000602C002080B582B000AF7860FFF7A8F83C
:10A4F000021C7B681A600023181CBD4602B080BD98
:10A5000080B584B000AFF860B9607A60FA68BB6863
:10A51000101C191CFFF7A0F8021C7B681A600023AE
:10A52000181CBD4604B080BD80B582B000AF021CCF
:10A53000FB1D1A70064BFA1D1278111C1F220A40CF
:10A540000121081C9040021C1A60BD4602B080BD6B
:10A5500000E100E080B582B000AF021CFB1D1A7064
:10A56000084AFB1D1B78191C1F230B400121081CE6
:10A570009840031C191CC0235B00D150BD4602B09B
:10A5800080BDC04600E100E0B0B582B000AF021C63
:10A590003960FB1D1A70FB1D1B787F2B32D93049A7
:10A5A000FB1D1B781A1C0F231340083B98082C4AEC
:10A5B000FB1D1B781C1C0F232340083B9B08063304
:10A5C0009B00D3185B68FA1D1278141C03222240EA
:10A5D000D200FF24251C95402A1CD2431A403B6818
:10A5E0009C01FF231C40FB1D1B781D1C03232B40DB
:10A5F000DB00251C9D402B1C1A43831D9B00CB18A0
:10A600005A6029E0174BFA1D127852B29208154988
:10A61000F81D007840B28008C03080004158F81D15
:10A620000078041C03202040C000FF24251C854026
:10A63000281CC043084039688C01FF210C40F91DDB
:10A6400009780D1C03212940C900251C8D40291CB7
:10A650000143C0329200D150BD4602B0B0BDC046E9
:10A6600000ED00E000E100E080B582B000AF78606E
:10A67000A023DB057A68C132FF3292000321D1505A
:10A68000BD4602B080BDC04680B582B000AF7860E4
:10A690000A1CFB1C1A70A023DB05FA1C127892001E
:10A6A000111C7A68C132FF329200D150BD4602B00F
:10A6B00080BDC04680B582B000AF7860FB1C1970C9
:10A6C000BB1C1A70A023DB05BA1C12781204111CE3
:10A6D000FA1C1278920011437A68C132FF3292005C
:10A6E000D150BD4602B080BD80B500AF074B0022FF
:10A6F0001A70074B0122DA60054B01225A60044AA6
:10A70000A023DB000021D150BD4680BDB42C002029
:10A710000020004080B582B000AF084B0122DA6013
:10A72000074B01221A703B1C03221A70054B1B6851
:10A730003A1C101C9847BD4602B080BD0020004066
:10A74000B42C0020B02C002080B582B000AF154B97
:10A750001B78DBB2022B02D0134B01229A60134A02
:10A76000FB1D101C191C00F025FC031C002B02D043
:10A77000FFF7D0FF12E00C4AC2239B008021D1508A
:10A78000094AFB1D1B78191C094BD150054B0222AD
:10A790001A70054AC1239B008021D150BD4602B0EA
:10A7A00080BDC046B42C002000200040982C002022
:10A7B0001C05000080B500AF064BDA68054B9B68AE
:10A7C0009A4202D0FFF7C0FF01E0FFF7A3FFBD46AA
:10A7D00080BDC046982C002080B500AF084B1B7888
:10A7E000DBB2012B02D0022B03D006E0FFF77CFF87
:10A7F00003E0034B03221A70C046BD4680BDC0462D
:10A80000B42C002080B500AF114B1B78DBB2002BBD
:10A8100002D0032B15D018E00E4AA023DB00042140
:10A82000D1500C4B01221A600B4BDA680A4B9B6823
:10A830009A4202D0FFF788FF07E0054B01221A7009
:10A8400003E0034B02221A70C046BD4680BDC046DD
:10A85000B42C002000200040982C002080B500AFD0
:10A86000094B1B78DBB2012B0ADB022B05DD032B26
:10A8700000D005E0FFF738FF03E0FFF79BFF00E0A3
:10A88000C046BD4680BDC046B42C002080B500AF98
:10A89000044B1B78DBB2012B01D1FFF755FFBD46FE
:10A8A00080BDC046B42C002080B500AFFFF71CFF70
:10A8B000BD4680BD80B582B000AF021CFB1D1A7082
:10A8C000FB1D1B78042B13D89A000B4BD3181B6865
:10A8D0009F46FFF781FF0CE0FFF794FF09E0FFF7C9
:10A8E000BDFF06E0FFF7D2FF03E0FFF7DDFF00E06A
:10A8F000C046BD4602B080BD482F020080B584B07E
:10A9000000AF786039603B687A681A40164B1B6864
:10A91000134015D0154B1A783B1C0833101C191C1A
:10A9200000F0EEFE031CFB60FB68002B19D1BA6837
:10A930007B6813407B60BB68DA433B6813403B6035
:10A94000094B1B683A68134003D00120FFF7B2FFA0
:10A9500007E0054B1B687A68134002D00020FFF720
:10A96000A9FFBD4604B080BDAC2C0020A82C00205F
:10A9700080B586B000AF304A84235B00D358002BEB
:10A9800028D02D4A84235B000021D1502B4BDA685C
:10A990002A4B9B68D21A294B9B889A421AD8264A7E
:10A9A000A323DB00D358DBB2244A101C191C00F08F
:10A9B000D9FA224BDA68214B9B68D31A012B09D1B3
:10A9C0003B1C0C3300221A701D4B1B683A1C0C32C6
:10A9D000101C9847184A8E235B00D358002B07D0D1
:10A9E000154A8E235B000021D1500320FFF762FF40
:10A9F000114A92235B00D358002B19D00E4A9223A0
:10AA00005B000021D1500C4A9023DB00D3587B61BE
:10AA1000094A9023DB007969D1503B1D02221A704C
:10AA20003B1D7A695A60064B1B683A1D101C9847FB
:10AA3000BD4606B080BDC04600200040882C0020E6
:10AA4000B02C002080B500AF164AA023DB00042103
:10AA5000D150144A84235B000021D150114A8E2327
:10AA60005B000021D1500F4A0E490F4BCB580121FA
:10AA7000181C8843011C0C4BD1500A4AA123DB004F
:10AA800001214942D150074AA223DB00012149425A
:10AA9000D150044B01229A60024B01221A60BD463C
:10AAA00080BDC046002000406C05000080B582B02B
:10AAB00000AF7860164AA023DB000421D150144A6D
:10AAC00084235B000021D150114A8E235B000021BA
:10AAD000D1500F4A0E490F4BCB58012119430D4B52
:10AAE000D1500B4A7B68DB78191CA223DB00D150C4
:10AAF000074A7B689B78191CA123DB00D150044BCB
:10AB000001229A60024B01221A60BD4602B080BD4C
:10AB1000002000406C05000080B588B000AFF860F0
:10AB2000B9607A601A1CFB1C1A700023FB610023B9
:10AB3000BB619E4B00221A709D4B7A681A60BB68FD
:10AB4000002B01D107232DE1BB681A68BB685B6845
:10AB50009BB29849081C111C1A1C00F0D5F9031C63
:10AB60007B617B69002B01D07B691BE1BB689A6824
:10AB7000BB68DB689BB29049081C111C1A1C00F0D2
:10AB8000C3F9031C7B617B69002B01D07B6909E160
:10AB9000FB685B78181CFFF767FDFB681B78181CC7
:10ABA0000021FFF771FD854AFB685B78191C844B17
:10ABB000D150824AFB681B78191C824BD1507F4AC6
:10ABC000FB689968804BD150FB685B79002B04D0FF
:10ABD0007A4A7E4B0E21D15003E0784A7B4B00210C
:10ABE000D150FB681B79022B00D097E0FB689B7863
:10ABF000181CFFF739FDA023DA05FB689B780121BB
:10AC0000081C9840031C191C714BD1506B4AA2239D
:10AC1000DB0001214942D150684AFB689B78191C2E
:10AC2000A123DB00D150654A6449684BCB58012110
:10AC30001943664BD150FB68DB780122111C994007
:10AC40000B1C1A1C634B1A60FB68DB78181C002174
:10AC50000322FFF72FFDFB68DB780122101C9840D0
:10AC6000031CFB61FB68DB780122111C99400B1C63
:10AC7000BB61BB6A1B88002B17D15748F969BA69B9
:10AC8000564B00F0F1FB031C7B617B69002B01D06C
:10AC90007B6987E0504B1B781B029BB2FF2213435A
:10ACA0009BB29AB2BB6A1A800CE0BB6A1B88FE2B6F
:10ACB00001D8072376E0BB6A1B881B0A9BB2DAB275
:10ACC000454B1A70444B1A783B1C1033101C191C4E
:10ACD00000F016FD031C7B617B69002B01D07B69B2
:10ACE00060E03D4B1B78181C00F022FC031C7B61CC
:10ACF0007B69002B01D07B6954E0FB68DB78012283
:10AD0000101C9840031C3A69134003D10120FFF73F
:10AD1000D1FD2EE00020FFF7CDFD2AE0FB681B7976
:10AD2000012B14D1BB6A1B88002B08D12C4B1B783C
:10AD30005A1CD1B22A4A11701A1CBB6A1A80FB68CD
:10AD4000181CFFF7B3FE194B01221A7011E0BB6A01
:10AD50001B88002B08D1224B1B785A1CD1B2204AE9
:10AD600011701A1CBB6A1A80FFF76CFE0F4B012290
:10AD70001A70124AC2239B0001214942D1500F4A46
:10AD8000C1239B00A1218900D1500220FFF7E2FBE3
:10AD9000FB1C1B780220191CFFF7F6FB0220FFF7B3
:10ADA000C3FB0023181CBD4608B080BDB42C002096
:10ADB000B02C0020882C0020982C0020002000407F
:10ADC0000C05000014050000240500006C050000BF
:10ADD00004050000AC2C0020A82C0020FDA80100D8
:10ADE0000820002080B582B000AF7860054A7B68FB
:10ADF000101C191C00F0DEF8031C181CBD4602B024
:10AE000080BDC046882C002080B584B000AF021CF5
:10AE1000FB1D1A70094AFB1D1B78101C191C00F041
:10AE2000A1F8031CFB60FB68002B02D10220FFF796
:10AE300041FDFB68181CBD4604B080BD982C002065
:10AE400080B582B000AF0D4B181C00F0D5F8031C84
:10AE50007B607B68002B01D07B680BE0084B181CE3
:10AE600000F0CAF8031C7B607B68002B01D07B6874
:10AE700000E00023181CBD4602B080BD882C0020D5
:10AE8000982C002080B582B000AF7860064B1B780C
:10AE9000DBB25A1E9341DBB21A1C7B681A70002386
:10AEA000181CBD4602B080BDB42C002080B584B013
:10AEB00000AF021CBB1D1A80BB1D1B88FE2B04D8D3
:10AEC0000420FFF7F7FC002317E03B1C0E33BA1DEC
:10AED0001288120A1A800B4B1B783A1C0E32128809
:10AEE0009A4201D0072308E00420FFF7E3FC054B5A
:10AEF0001B78181C00F0C8FB031C181CBD4604B0CE
:10AF000080BDC046A82C002080B584B000AFF8609A
:10AF1000B960BB1D1A80BB68002B01D10E231CE059
:10AF2000BB1D1B88002B06D0BB1D1B88013BBA1D17
:10AF30001288134001D009230FE0FB68BA681A6039
:10AF4000BB1D1B88013B9AB2FB689A80FB680022FC
:10AF50009A60FB680022DA600023181CBD4604B02A
:10AF600080BDC04680B582B000AF78600A1CFB1C73
:10AF70001A707B68DA687B689B68D21A7B689B884A
:10AF80009A4211D87B681A687B68DB68796889887F
:10AF90000B40D318FA1C12781A707B68DB685A1CB5
:10AFA0007B68DA60002300E00423181CBD4602B071
:10AFB00080BDC04680B582B000AF786039607B68E4
:10AFC000DA687B689B689A4211D07B681A687B6854
:10AFD0009B68796889880B40D3181A783B681A7087
:10AFE0007B689B685A1C7B689A60002300E00523FD
:10AFF000181CBD4602B080BD80B582B000AF78603D
:10B000007B68DA687B689A600023181CBD4602B032
:10B0100080BDC04680B582B000AF021CFB1D1A7017
:10B02000064BFA1D1278111C1F220A400121081C30
:10B030009040021C1A60BD4602B080BD00E100E0F5
:10B0400080B582B000AF021CFB1D1A70084AFB1DC0
:10B050001B78191C1F230B400121081C9840031C5E
:10B06000191CC0235B00D150BD4602B080BDC04654
:10B0700000E100E0B0B582B000AF021C3960FB1DFA
:10B080001A70FB1D1B787F2B32D93049FB1D1B78B2
:10B090001A1C0F231340083B98082C4AFB1D1B78F1
:10B0A0001C1C0F232340083B9B0806339B00D3182E
:10B0B0005B68FA1D1278141C03222240D200FF2480
:10B0C000251C95402A1CD2431A403B689C01FF2353
:10B0D0001C40FB1D1B781D1C03232B40DB00251C83
:10B0E0009D402B1C1A43831D9B00CB185A6029E0FE
:10B0F000174BFA1D127852B292081549F81D0078C4
:10B1000040B28008C03080004158F81D0078041C0F
:10B1100003202040C000FF24251C8540281CC0437C
:10B12000084039688C01FF210C40F91D09780D1C7D
:10B1300003212940C900251C8D40291C0143C03230
:10B140009200D150BD4602B0B0BDC04600ED00E057
:10B1500000E100E080B582B000AF78607A68032338
:10B1600013405A425341DBB2181CBD4602B080BDA9
:10B1700080B586B000AF7860396000237B6145E020
:10B180007B690122111C99400B1CFB603B68FA682B
:10B19000134038D07B68DB68FA68134009D18023FC
:10B1A0009B023B617B68DA68FB681A437B68DA6064
:10B1B00009E0C0239B023B617B68DB68FA68D243ED
:10B1C0001A407B68DA60A023DB05A022D2057969EA
:10B1D000C131FF31890089580F4A11407A69C13263
:10B1E000FF329200D150A023DB05A022D20579695D
:10B1F000C131FF31890089583A6911437A69C132F6
:10B20000FF329200D1507B6901337B617B691F2B38
:10B21000B6D9BD4606B080BDFFFFFCFF80B588B043
:10B2200000AFA023DA05A223DB00D358BB613E4A5E
:10B23000BE235B000021D1503B1C1F3300221A703B
:10B2400068E03A4B19683B1C1F331A78131C9B00AB
:10B250009B189B00CB183B613B1C1F331B780122C2
:10B26000111C99400B1C1A1C314B1B6813404AD00F
:10B270003B69DB68DA43BB695A403B691B68134092
:10B280007B613A697B69101C191CFFF771FFA023D1
:10B29000DA05A223DB00D258BB695340FB60FB6890
:10B2A000002B16D0BA69FB681343BB613B69DB68AE
:10B2B000DA43BB695A403B691B681340BB603A697B
:10B2C000BB68101C191CFFF753FF7A69BB68134356
:10B2D0007B61BB69DA433B699B6813407A69134021
:10B2E0007B603B695B68BA6913407A6913403B60D5
:10B2F0003A687B68134306D03B691B6939687A68F2
:10B30000081C111C98473B1C1F331A783B1C1F3329
:10B3100001321A70074B1B783A1C1F3212789A427E
:10B320008FD3BD4608B080BD00600040C02C002017
:10B33000B82C0020BD2C002080B584B000AF021CCA
:10B34000FB1D1A700023FB6031E01C4B1968FB1DCC
:10B350001A78131C9B009B189B00CB181B68FA687B
:10B360000121081C9040021C13401DD0A023DB05C6
:10B37000A022D205F968C131FF3189008958104AED
:10B380001140FA68C132FF329200D150A023DB0590
:10B39000A022D205F968C131FF3189008958FA68C5
:10B3A000C132FF329200D150FB680133FB60FB6871
:10B3B0001F2BCAD9BD4604B080BDC046C02C00209A
:10B3C000FFFFFCFF80B582B000AF021C3960FB1D9F
:10B3D0001A703B68002B01D1072337E03B68181C2B
:10B3E000FFF7B8FE031C01225340DBB2002B01D053
:10B3F00007232BE0174B3A681A60174BFA1D127897
:10B400001A70164B00221A70154B00221A60114B4D
:10B410001968114B1B781A1C131C9B009B189B006E
:10B42000081C00211A1C00F0F5FA0E4AC2239B00EA
:10B4300001214942D1500620FFF702FE06200121DA
:10B44000FFF718FE0620FFF7E5FD0023181CBD4698
:10B4500002B080BDC02C0020BC2C0020BD2C0020E0
:10B46000B82C00200060004080B584B000AFF860C8
:10B47000B9607A603B602B4B1B68002B01D108231D
:10B480004CE03B68002B01D1072347E0264B1A789C
:10B49000264B1B789A4201D304233FE0214B1968C5
:10B4A000214B1B781A1C131C9B009B189B00CB186C
:10B4B000B9687A680A431A601A4B19681A4B1B78E4
:10B4C0001A1C131C9B009B189B00CB18BA685A606F
:10B4D000144B1968144B1B781A1C131C9B009B18E7
:10B4E0009B00CB187A689A600E4B19680E4B1B783C
:10B4F0001A1C131C9B009B189B00CB183A681A61FE
:10B50000094B1B785A1CD1B2074A1170FA681370A4
:10B51000FB681B78181CFFF70FFF0023181CBD46A3
:10B5200004B080BDC02C0020BD2C0020BC2C00200D
:10B5300080B586B000AF021CFB1D1A704D4B1B6816
:10B54000002B01D1082391E04B4B1B78FA1D127898
:10B550009A4201D3072389E0484ABE235B000021B9
:10B56000D150A023DA05A223DB00D358FB60444B63
:10B570001B68002B05D1414AC1239B00802109068D
:10B58000D150FB1D1B780122111C99400B1C1A1C69
:10B590003B4B1B681A433A4B1A60364B1968FB1D2C
:10B5A0001A78131C9B009B189B00CB180022DA60B2
:10B5B00000237B6156E07B690122111C99400B1C22
:10B5C000BB602C4B1968FB1D1A78131C9B009B1841
:10B5D0009B00CB181B68BA68134040D0FB68BA6860
:10B5E000134003D0C0239B023B6118E080239B02E1
:10B5F0003B61204B1968FB1D1A78131C9B009B189C
:10B600009B00CA181B4B1868FB1D19780B1C9B006C
:10B610005B189B00C318D968BB680B43D360A02399
:10B62000DB05A022D2057969C131FF318900895833
:10B63000144A11407A69C132FF329200D150A023DE
:10B64000DB05A022D2057969C131FF318900895813
:10B650003A6911437A69C132FF329200D1507B6955
:10B6600001337B617B691F2BA5D90023181CBD46C4
:10B6700006B080BDC02C0020BD2C00200060004022
:10B68000B82C0020FFFFFCFF80B582B000AF021C89
:10B69000FB1D1A70164B1B68002B01D1082323E0F9
:10B6A000144B1B78FA1D12789A4201D307231BE032
:10B6B000FB1D1B78181CFFF73FFEFB1D1B780122AA
:10B6C000111C99400B1CDA430B4B1B681A400A4BA8
:10B6D0001A60094B1B68002B05D1084AC2239B0046
:10B6E00080210906D1500023181CBD4602B080BD40
:10B6F000C02C0020BD2C0020B82C00200060004091
:10B7000080B584B000AF021C3960FB1D1A70134B6A
:10B710001B68002B01D108231CE0114B1B78FA1D7C
:10B7200012789A4201D3072314E00C4B1968FB1DD1
:10B730001A78131C9B009B189B00CB18FB60A0235E
:10B74000DA05A223DB00D258FB681B681A403B686D
:10B750001A600023181CBD4604B080BDC02C002018
:10B76000BD2C002080B584B000AFF860B9607A606D
:10B770000B4A7B68101C191C7F2200F007FA084A4C
:10B780007F230021D154BB689AB2064B1A80064B26
:10B79000FA681A60034B1B88034B1B6872B6FEE7FE
:10B7A000C42C0020442D0020482D002080B500AF7F
:10B7B000024B034A1A60BD4680BDC0460C200020E3
:10B7C0000024F40080B500AF00F01EF8031C002B2D
:10B7D00006D00A4B0A4A1A600A4B802212021A60EB
:10B7E00000F052F8031C002B05D08023DA05C1239A
:10B7F000DB000121D150BD4680BDC046040500409C
:10B80000DFFF07C0186C004080B500AF1A4B1A6804
:10B81000FF231340012B2AD1184B1A680F23134022
:10B8200025D1174B1A68F023134006D1154B1A681F
:10B83000F023134001D101231AE0114B1A68F023C1
:10B840001340102B06D10F4B1A68F023134001D17F
:10B8500001230DE00A4B1A68F0231340302B06D168
:10B86000084B1A68F023134001D1012300E00023A4
:10B87000181CBD4680BDC046E00F00F0E40F00F08C
:10B88000E80F00F0EC0F00F080B500AF0D4B1A6828
:10B89000FF231340012B11D10B4B1A680F231340C8
:10B8A0000CD10A4B1A68F0231340402B06D1084BE9
:10B8B0001A68F023134001D1012300E00023181C73
:10B8C000BD4680BDE00F00F0E40F00F0E80F00F08F
:10B8D000EC0F00F003210A4802680A43026009489D
:10B8E00002680A4302600849084A094B9B1A03DDB3
:10B8F000043BC858D050FBDC064880470648004748
:10B90000240500405405004080340200002000203F
:10B91000D8280020C5B7010021610100FEE7FEE73D
:10B92000FEE7FEE7FEE7FEE710B50021041C01F08C
:10B9300057FC044B1868C36B002B00D09847201CA1
:10B9400007F054FA602F020070B50D4E0D4D002423
:10B95000AD1BAD1005D0A300F35801349847A542A4
:10B96000F9D107F045FA084E084D0024AD1BAD1083
:10B9700005D0A300F35801349847A542F9D170BD12
:10B98000C8280020C8280020C8280020D02800206F
:10B99000F0B50F2A35D9031C0B439C0735D1161C73
:10B9A000103E36093501451910350C1C031C27685B
:10B9B0001F6067685F60A7689F60E7681034DF609A
:10B9C0001033AB42F3D1731C1B01C518C9180F23E8
:10B9D0001340032B1BD91C1FA4080134A40000230F
:10B9E000CE58EE500433A342FAD1ED18C918032300
:10B9F0001A4005D00023CC5CEC5401339342FAD1B9
:10BA0000F0BD051C002AF5D1FAE7051CF2E71A1C67
:10BA1000F8E7C046F0B5830746D0541E002A42D04E
:10BA2000CEB2031C032503E0621E002C3BD0141C85
:10BA300001335A1E16702B42F6D1032C2BD9FF2549
:10BA40000D402A0215432A0415430F2C15D9271C33
:10BA5000103F3F091E1C3A011036B6181A1C15601B
:10BA600055609560D5601032B242F8D101373F0180
:10BA70000F22DB191440032C0DD9271FBF08BA0071
:10BA80001E1DB6181A1C20C2B242FCD10137BF00DD
:10BA90000322DB191440002C05D01C19C9B21970FF
:10BAA0000133A342FBD1F0BD141C031CC5E7C04603
:10BAB00008B470B5061C9DB0151E25DB822302ACB0
:10BAC0009B00A381029121610023002A17D1A3606A
:10BAD000636101235B42E381219A22AB301C211C6C
:10BAE000019300F08DF8421C0BDB002D02D0029A6E
:10BAF000002313701DB070BC08BC01B01847531E62
:10BB0000E5E78B223260F0E78B230360012040429F
:10BB1000F0E7C0460CB430B5174B9DB00C1C1D6847
:10BB200024D4822302A99B008B8102900861002308
:10BB3000002C16D18B604B6101235B42CB81209A94
:10BB400021AB281C019300F05BF8421C0BDB002C9E
:10BB500002D0029A002313701DB030BC08BC02B0A2
:10BB60001847631EE6E78B232B60F0E78B23012049
:10BB70002B604042F0E7C046382400200023C25C1E
:10BB80000133002AFBD1581E7047C046031C0B43EB
:10BB9000F0B5041C9D0701D1032A15D8002A12D044
:10BBA0000D78013A631C4E1C2570002D1BD0311CF2
:10BBB00007E00C7801335D1E013A2C700131002C36
:10BBC00011D0002AF5D1F0BD0B4E0B680B4FDD19DB
:10BBD0009D433542E2D10434251F043A04312B60E1
:10BBE000032AF2D8DAE79C180021002AEBD019705A
:10BBF0000133A342FBD1E6E780808080FFFEFEFE9A
:10BC0000F0B544465F4656464D46F0B4C7B014936F
:10BC10000B9190460D9002F005FC00681A90FFF71A
:10BC2000ADFF0B9C1D90A3891D0604D5206900283B
:10BC300001D101F0A1F836AC002529AF0023099409
:10BC400029940024BB607B6019951B941C9536AE2B
:10BC50001F941E951194C3465D462B785C46002BBD
:10BC60001BD0252B02D118E0252B3AD001342378A4
:10BC7000002BF9D15846251A002D0ED0B8685A4627
:10BC80002B18BB607B683260013375607B60072BCB
:10BC900034DC08361199491911912378002B36D0DC
:10BCA000621C8725934600236D4401222B7052426B
:10BCB0000025637800240C92109410220A954024E9
:10BCC0008025914600212020A446AA465A460132EA
:10BCD0001C1C203C582C00D9CAE2C74DA4002C598A
:10BCE000A7465946651AC7E7109D14946D421095F2
:10BCF0000A9C04231C430A941378E8E70D980B99D7
:10BD00003A1C03F051FB002809D136AEC2E7B868EF
:10BD1000002804D00D980B993A1C03F045FB0B9CAE
:10BD20001198A3895D0601D50120404247B03CBC73
:10BD300090469946A246AB46F0BD13782B21C6E744
:10BD40001378551CA8462A2B01D101F0F0F91C1CD0
:10BD5000303C0022092C01D901F05FF92B1C8846E8
:10BD600091008A1852000133A2185C1E21780C1C25
:10BD7000303C092CF4D91C1C0B1C4146A046002A5F
:10BD800001DA01F067F80C924246A1E70A9C554699
:10BD90002C430A9413789AE70A9C1793102387255B
:10BDA0001C436D440A9429700A9D9346AD0600D445
:10BDB00070E1149A072307329A43141C53681268DF
:10BDC0000834149412921393002B00DA70E1872543
:10BDD0006D442D78129A1398A846012302430C9CB7
:10BDE000002C03DB0A9D80218D430A95002A00D098
:10BDF00068E30C9C002C00D064E3002B01D000F021
:10BE0000C1FC0A9DED0701D400F0BCFC6D46D7359E
:10BE10003023099C2B70641B0F9415950F9B0C9D70
:10BE2000AB4200DA2B1C00240E9318944546002DDB
:10BE300002D00E9C01340E940A9D02231D40AA4696
:10BE400002D00E9C02340E940A9D84231D40A94604
:10BE500000D017E2109D0E982C1A002C00DC11E285
:10BE6000BA687B68102C01DC00F0F0FF634D311CD8
:10BE7000A8464646102503E0103C0831102C15DD7D
:10BE8000103201330E604D60BA607B60072BF3DD2A
:10BE90000D980B993A1C03F087FA002800D03EE772
:10BEA000103CBA687B6836A9102CE9DCB0460E1C41
:10BEB000404674600133A4183060BC607B60072B7F
:10BEC00001DD00F0B6FC8721694409780836884610
:10BED000D9E1179387236B441970149B934607335A
:10BEE000072293431D1C083514951C681B945B683E
:10BEF0001B981C931C9903F00BFA012801D000F049
:10BF0000CFFD1B981C993B4B394A04F013FD0028C8
:10BF100001D000F0F0FF87256D442D78A846179CCE
:10BF2000472C01DC00F024FF354C15940A9D80233A
:10BF30009D4303240A950E9403250F9500240025A4
:10BF40000C94189572E7002410941C1C303C0023BC
:10BF500088469900CB185B0001321B19541E2178CA
:10BF60000C1C303C092CF4D910930B1C4146AFE655
:10BF70000A9D08231D430A951378A8E60A9C179387
:10BF800010231C430A940A9D9346AD0600D45FE13A
:10BF9000149B0722073393431C1C083414941C6819
:10BFA0005D6812941395221C00232A4387240021E4
:10BFB0006C442170884612E70A9C179310231C4397
:10BFC0000A940A9D9346AD0600D42BE1149B0722E8
:10BFD000073393431C1C083414941C685D68221CAE
:10BFE0001294139501232A43E0E7C046C046C04699
:10BFF0000000000000000000642F02001C3102005D
:10C00000DC3002009346BC4C87220A9D6A44179399
:10C0100011701F94AD0600D4A1E0149B07220733D2
:10C0200093431C1C083414941C685D681294139587
:10C030000A9DED0701D400F00CFC129A139802231C
:10C040000243B3D00A9D179C22A930201D430870DB
:10C050004C700A95AAE7149C1793149B04341B6830
:10C0600093462CAD1494012487202B706844002340
:10C070000E940F940024037098460C941894159510
:10C08000DAE687200A9D6844179393460170AD064F
:10C0900000D58EE60A9DED0601D400F040FD149C0B
:10C0A000236804341293DB171393149400D48EE6A0
:10C0B00012981399002544428D4187212D2369440C
:10C0C000221C0B7098461294139501232A4386E68E
:10C0D00087250A9C6D4493462970A40601D400F07C
:10C0E000F9FC149D119C2B68E21704351C605A6002
:10C0F0001495B1E5149B149D1B680A9C129304359A
:10C1000002231C43934622AB302214957B4D1A70B8
:10C11000002078220A9478245A7013901F950223E5
:10C120001794129A42E70A9C65462C430A941378A6
:10C13000CDE51378141C6C2B01D100F07FFD0A9C17
:10C140004D462C430A94C2E587256D4429706B4CFB
:10C150000A9D179393461F94AD0600D55DE70A9D8F
:10C16000ED0601D400F0CDFC1498149C0068002169
:10C1700004341290139114945AE70A9C04430A94CD
:10C180001378A4E5149D149C2D68872017936844A8
:10C1900000239346043415950370002D01D100F05F
:10C1A00091FE0C9D1598002D01DA00F043FE002150
:10C1B0002A1C02F0D1FB002801D100F0F3FE159DEE
:10C1C000401B0C9D0F90A84200DD0F9587200F9D0E
:10C1D00068440078EB43DB1780461D400E951494AD
:10C1E000002500240C94189520E60A9D01231D4388
:10C1F0000A9513786BE5149D149C2D6804341095F2
:10C20000002D00DA70E51378149460E513780029A6
:10C2100000D05CE520215AE50A9D17939346AD06B0
:10C2200000D5D3E60A9DED0601D400F09DFC1498DC
:10C23000149C00680021043412901391149401237B
:10C24000021CB3E60A9D17939346AD0600D59FE600
:10C250000A9DED0601D400F072FC1498149C00684D
:10C26000002104341290139114940023021C9DE6C3
:10C2700087256D44179393462970002B00D146E51E
:10C280002CADF0E6BC684346002B0DD00123736053
:10C290007B6887256D44013401333560BC607B6069
:10C2A000072B00DD1AE20836504600280CD022ABDE
:10C2B0003360022373607B6802340133BC607B60AF
:10C2C000072B00DD22E208364946802900D17DE1B6
:10C2D0000C9A0F9BD51A002D3EDD7B68102D01DCDA
:10C2E00000F052FC0649102289469246211C321C5D
:10C2F0000D9C2E1C4D4609E0E8300200FC30020087
:10C30000C8300200103E0832102E16DD50461031A3
:10C31000013315605060B9607B60072BF2DD201C93
:10C320000B993A1C03F040F8002800D0F7E4103EC7
:10C33000B9687B6836AA102EE8DCA9460C1C351CAF
:10C34000161C49466419013331607560BC607B601E
:10C35000072B00DDB6E108360A9DED0500D5D8E0D3
:10C36000159D7B6835600F9D013364197560BC6055
:10C370007B60072B00DD9AE008360A9D6D0743D5E8
:10C3800010980E99451A002D3EDD7B68102D01DCBA
:10C3900000F0ADFDDA4810218946321C211C2E1C0C
:10C3A00080460D9C0B9D03E0103E0832102E17DDD9
:10C3B000D34810311060013348465060B9607B604B
:10C3C000072BF1DD201C291C3A1C02F0EDFF002890
:10C3D00000D0A4E4103EB9687B6836AA102EE7DCD2
:10C3E000351C0C1C161C41466419013322C6BC6066
:10C3F0007B60072B08DD0D980B993A1C02F0D4FFE7
:10C40000002800D08BE4BC680E9B109DAB4200DA84
:10C410002B1C119DED181195002C00D025E1002357
:10C420007B6036AEFFF718FC199D012D00DCEFE2B2
:10C43000012373607B68159D013401333560BC6056
:10C440007B60072B00DD04E308361A9D013335605D
:10C450001D9D984664197560BC607B60072B00DDEC
:10C4600004E308361B981C99A44BA34A04F05CFA19
:10C47000002800D0F3E1199B159D0121013B884460
:10C480000135E418424635607360BC607A60072A63
:10C4900000DDDCE0083625AB1E9D336043466419A1
:10C4A00001337560BC607B60072B00DC64E70D988E
:10C4B0000B993A1C02F078FF002800D02FE4BC68EA
:10C4C00036AE5AE7012B00D12CE1022B00D0D6E08A
:10C4D0001F9D6B46D7330F21A946B4461C1C129AE8
:10C4E000139B201C0C1C14404D462C5D1E07150987
:10C4F000321C04702A431C09231C151C441E1D43B6
:10C50000EFD1099C1590241A1292139366460F944A
:10C5100084E4179D652D87DD1B981C99774B764A1F
:10C5200004F002FA002800D132E1764B0134336086
:10C53000012373607B68BC6001337B60072B00DDE7
:10C5400026E308362398199DA84203DB0A9DED07D0
:10C5500000D412E71A9D7B6835601D9D0133641974
:10C560007560BC607B60072B00DD6EE30836199DAB
:10C57000013D002D00DC00E77B68102D01DC00F0A0
:10C58000CEFD6149102289469046211C321C0D9C2B
:10C590002E1C4D4604E00832103E102E00DCADE1AA
:10C5A00040461031013315605060B9607B60072B45
:10C5B000F1DD201C0B993A1C02F0F6FE002801D098
:10C5C000FFF7ADFBB9687B6836AAE5E7109A0E9BCA
:10C5D000D51A002D00DC7BE67B68102D01DC00F015
:10C5E000B7FC4949102289469246211C321C0D9CF9
:10C5F0002E1C4D4603E0103E0832102E17DD50462B
:10C600001031013315605060B9607B60072BF2DD9B
:10C61000201C0B993A1C02F0C7FE002801D0FFF73E
:10C620007EFB103EB9687B6836AA102EE7DCA9466F
:10C630000C1C351C161C49466419013331607560A9
:10C64000BC607B60072B00DD1EE2083640E60D98DB
:10C650000B993A1C02F0A8FE002801D0FFF75FFBFF
:10C660007B68BC68984636AE15E70D980B993A1C66
:10C6700002F09AFE002800D1D1E6FFF750FB6B468E
:10C68000D7330720B446129C139D021C224030323F
:10C69000191C1A706B079946E6084C46EB083443A0
:10C6A0001D1C261C4B1E2E43EFD1129413950A9C81
:10C6B00015916646E40700D52FE1099D6D1A0F9587
:10C6C000FFF7ACFB0D980B993A1C02F06DFE0028A9
:10C6D00001D0FFF724FBBC6836AE3DE60D980B9900
:10C6E0003A1C02F061FE002801D0FFF718FBBC687D
:10C6F00036AED9E5C046C04600000000000000008C
:10C700001C31020018310200C83002000D980B994C
:10C710003A1C02F049FE002801D0FFF700FBBC687C
:10C7200036AED1E51398002802D11299092923D9F0
:10C730006B46D733B146129C139D1E1C201C291C2E
:10C740000A22002304F01EF930323270201C0A2223
:10C750000023291C04F016F9021C041C0D1C731E76
:10C760000A43EAD1159612941395099D159C4E46DD
:10C770002D1B0F95FFF752FB6D460B1CD735303341
:10C78000FFF747FB002536AC0F951594FFF746FBE6
:10C79000239B002B00DC07E215981999189A45187D
:10C7A000281A8046904200DD9046404600280BDD66
:10C7B0007B6815994444013331607060BC607B60D4
:10C7C000072B00DD4AE308364246D343DB171898AF
:10C7D0001340C01A8046002800DCBBE07B681028AC
:10C7E00001DC00F0A0FCDE4A10209146211C321C26
:10C7F00044468246A8464E460D9D04E00832103C51
:10C80000102C00DC95E0504610310133166050606A
:10C81000B9607B60072BF1DD281C0B993A1C02F0F4
:10C82000C3FD002801D0FFF77AFAB9687B6836AA01
:10C83000E5E70D980B993A1C02F0B6FD002801D0EF
:10C84000FFF76DFA87226A441278BC68904636AECC
:10C8500019E5129A139802230243FFF7A7FB199DCB
:10C86000013D002D00DC16E6102D01DC00F040FC3F
:10C87000BB49102289469246211C321C43462E1C7D
:10C880000D9C4D4603E0103E0832102E17DD504639
:10C890001031013315605060B9607B60072BF2DD09
:10C8A000201C0B993A1C02F07FFD002801D0FFF7F5
:10C8B00036FA103EB9687B6836AA102EE7DCA94626
:10C8C0000C1C351C9846161C0122904449466419DC
:10C8D000434631607560BC607B60072B00DCD9E5A6
:10C8E0000D980B993A1C02F05FFD002801D0FFF76C
:10C8F00016FA7D68BC68A84636AECCE5A9460C1C85
:10C90000351C161C49466419013331607560BC60E2
:10C910007B60072B00DC2FE5C9E5302A03D0159397
:10C92000013930230B70099C159D641B0F94FFF790
:10C9300075FA4546B146A046161C0C1C49464246AF
:10C940004444013331607260BC607B60072B00DDC2
:10C95000ACE20836159B19989846189B9844239B7F
:10C96000834247DB0A99C90744D441466A1A199D94
:10C97000EB1A1D1E954200DD151C002D0BDD7A689B
:10C9800040466419013230607560BC607A60072AE5
:10C9900000DD7CE20836EA43D21715405D1B002D0E
:10C9A00000DCEAE47B68102D00DCD1E36C4A102047
:10C9B0009146211C321C80462E1C0D9C4D4603E0E6
:10C9C0000832103E102E99DD4046103101331560BB
:10C9D0005060B9607B60072BF2DD201C0B993A1C7C
:10C9E00002F0E2FC002801D0FFF799F9B9687B68F2
:10C9F00036AAE6E71A9A1D9832607A68241801323E
:10CA00007060BC607A60072A00DD33E20836ACE76C
:10CA10000A9D01232B4200D00AE57868159D8046C7
:10CA2000012080440134414635607360BC60796008
:10CA3000072900DC2EE50D980B993A1C02F0B4FC96
:10CA4000002801D0FFF76BF97A68BC68904636AED3
:10CA500021E50D980B993A1C02F0A6FC002801D0A4
:10CA6000FFF75DF9BC687B6836AEEEE40D980B9974
:10CA70003A1C02F099FC002801D0FFF750F97868C1
:10CA8000BC68804636AEEDE40D980B993A1C02F076
:10CA90008BFC002801D0FFF742F9BC6836AE17E4E2
:10CAA0001B981C9902F034FC002800D0D9E0179C98
:10CAB000472C00DC6EE12B4C159487200A9D6844BE
:10CAC000802300789D4303240A9580460E94032515
:10CAD000FFF733FA0A9DED060BD40A9C640608D5CD
:10CAE000149D119C2D682C80149D04351495FFF71E
:10CAF000B3F8149C119D236804341D601494FFF74F
:10CB0000ABF80A9D6D0600D46FE1149C00252488C3
:10CB100013951294149C04341494FFF789FA0A9D17
:10CB2000149C6D0601D4FFF7BBFA0023E35E149D4D
:10CB300012930435DB1713931495FFF745F90A9DFB
:10CB40006D0600D439E1149C0025248813951294B5
:10CB5000149C002304341494129AFFF727FAC04659
:10CB6000C8300200E43002000A9D6D0600D430E1B6
:10CB7000149C0025248813951294149C01230434DA
:10CB80001494129AFFF712FAE1488146FFF7D9FB95
:10CB90000D980B993A1C02F007FC002801D0FFF712
:10CBA000BEF8BC6836AECDE4DA4A01343260012208
:10CBB00072607A68BC6001327A60072A00DDECE0BE
:10CBC0000836181C002807D1199D002D04D10A9D94
:10CBD000ED0701D4FFF7D1FB1A9D7B6835601D9DE1
:10CBE000013361197560B9607B60072B00DD19E2C4
:10CBF000321C08324442002C00DC0CE1102C00DC1A
:10CC0000C6E2C34D102604E00832103C102C00DCB4
:10CC1000F5E01031013315605660B9607B60072B79
:10CC2000F2DD0D980B993A1C02F0BEFB002801D0F2
:10CC3000FFF775F8B9687B6836AAE6E70A9D013206
:10CC400005430A956378FFF742F80D980B993A1C53
:10CC500002F0AAFB002801D0FFF761F8BC6836AEED
:10CC600085E4179D20230C9C9D43A946013400D1E7
:10CC7000A0E0472D00D1C9E180230A9C5B001C4342
:10CC80001C9D1C9B1694A846002B00DAE7E10024AB
:10CC90000E94179D662D00D15EE1462D00D15BE11B
:10CCA0004B460C9C453B5A425341E41802230093E7
:10CCB00023AB029324AB039327AB049301940D9809
:10CCC0001B9A434600F0C8FBA2461590672D01D081
:10CCD000472D03D10A9DED0700D4E0E115984946A0
:10CCE000041C5444462900D148E1884B864A1B98CD
:10CCF000414603F019FE221C00280BD1279B1A1C69
:10CD00009C4207D930215A1C27921970279B9C42BC
:10CD1000F9D81A1C159C4D46121B1992472D00D1AB
:10CD20000EE1179C652C00DC38E2179C662C00D1C4
:10CD3000A8E1239D1895199C189DAC4200DD7FE168
:10CD40000A9CE40700D5D7E1EB43DB172B400F9596
:10CD5000672517950E9D002D00D0E5E087206844DB
:10CD60000078169C80460E930A940C95FFF75EF8A7
:10CD7000694D1595FFF7DAF80D98402101F066FB33
:10CD800020602061002800D10DE20B9D40236B61E3
:10CD9000FEF751FF614D15958FE60D980B993A1CE2
:10CDA00002F002FB002801D0FEF7B9FF2398BC680F
:10CDB00036AE07E706240C945EE7149D149C2D689C
:10CDC0000020043412951390149400232A1CFFF7BA
:10CDD000EDF8149D149C2D680020043412951390D6
:10CDE000149401232A1CFFF7E1F8149D149C2D686C
:10CDF00000200434129513901494FFF719F9A946F2
:10CE000048460919013310605460B9607B60072BF4
:10CE100000DD2AE10832159C199D146001334C197C
:10CE20005560BC607B60072B01DDFFF740FB161CE3
:10CE3000FFF7A2FAFEF7A2FE0F90C34387206844D3
:10CE40000078DB1780460F9DFFF7C7F93449884605
:10CE5000FFF72EF801225242FEF795FF0D980B992D
:10CE60003A1C02F0A1FA002801D0FEF758FFBC6876
:10CE700036AEA9E40D980B993A1C02F095FA0028F9
:10CE800001D0FEF74CFF239BBC6836AE6DE50D98D4
:10CE90000B993A1C02F088FA002801D0FEF73FFFF8
:10CEA000199C239836AE231ABC6874E50D980B992B
:10CEB0003A1C02F079FA002801D0FEF730FFBC6876
:10CEC00036AE47E50C9B062B00D906230F930F9D2A
:10CED000DB43DB17149400241D400C94114C0E9579
:10CEE00000200025804618951594FEF7A5FF0C4AF2
:10CEF0009046FFF778FA87202D2368440370984600
:10CF0000FFF70DF8C046C04600000000000000001A
:10CF1000C830020018310200D8300200E0300200B0
:10CF20001C31020010310200169C87202D2268441B
:10CF30000A94002402700E9390460C94FEF779FF39
:10CF4000239CE01C36DB0C9DA54233DB1894F2E6F3
:10CF50009B488146FFF76FFB0323009323AB0C9C98
:10CF6000029324AB039327AB049301940D981B9A6F
:10CF7000434600F071FAA2461590AFE60378302BD5
:10CF800002D0239BE418B0E61B9841468B4B8A4A9B
:10CF900003F0CAFC0028F4D1012350461B1A239346
:10CFA000E418A2E68720684400780E958046149421
:10CFB000FEF7C3FF179D023D1795179825AD013C5D
:10CFC0002394A8462870002C00DAD4E06B462B226C
:10CFD00095331A70092C64DC6B469633302230345A
:10CFE0001A705C7026AB4446199D1C1B2D191E94AB
:10CFF000199C0F95012C00DCB7E00F9C01340F94B5
:10D00000E343DB17002523401895A3E60C9C002C76
:10D0100000D031E601250C952EE600242A1C0C9444
:10D02000FEF756FE0D980B993A1C02F0BDF9002848
:10D0300001D0FEF774FE2398B9687B6836AAD9E55B
:10D04000189C0123002C00DCA5E0199D5B190F93AF
:10D050000F9CDB43DB176725234017957AE6802575
:10D060002D062D24A8440E9413E60D980B993A1C16
:10D0700002F09AF9002801D0FEF751FEB9687B68EA
:10D0800036AAC8E6239C0C9D1894002C64DD002D64
:10D090003BD10A9CE40738D4189B0F935AE6279A91
:10D0A00038E6A221694489460B1C201C0A211D1C5C
:10D0B00003F01EFC30312970201C0A2103F0C2FB52
:10D0C0006B1E041E092CF0DC30346A46E4B2A33235
:10D0D0001C70934264D20D3A01E05C780133147005
:10D0E00001329945F9D196227B1B6A44D3187AE71D
:10D0F00033488146FFF7E8FB189C67250134E3437A
:10D10000DB170F942340179524E60C9B189D0133E1
:10D11000EB180F930F9CDB43DB1723401AE62848DC
:10D120008146FFF7EFFB26498946FFF707FC149D70
:10D13000149C2D68043453780C9514944246002DA9
:10D1400001DBFEF7C4FD012464420C94FEF7BFFD31
:10D150001B498946FFF7D6FB002D12D10A9CE40734
:10D160000FD4012401230F94F4E50A9DED0700D5A7
:10D1700043E70F9C44E76B462D22953364421A70B7
:10D1800028E70C9D0235EB43DB170F952B40E1E5BB
:10D190000B48814634E602231B1B56E7239C0CE711
:10D1A0006B4696331FE70D9C0C2301202360404201
:10D1B000FEF7BCFDC046C0460000000000000000B5
:10D1C000C8300200C046C04608B5034B002B02D051
:10D1D000024800F091F808BD0000000091E3010052
:10D1E000F0B55F4656464D464446F0B4404B85B0D8
:10D1F0001B68029001934933FF3303930F1C01987E
:10D20000A421490042589046002A4AD003988146FA
:10D2100041464E68741E41D44546A3008835ED183A
:10D22000C620C42301365B004000B6009B46824600
:10D230004644C344C24408E02B1C80331B68BB42F5
:10D2400005D0043D043E013C28D3002FF4D14146D3
:10D250004A683368013AA2422CD000223260002B87
:10D26000EFD040465946406801220968A24000902C
:10D2700011421DD05046006810421DD10298296805
:10D28000984741464968009A9142B8D14A46126887
:10D290004245B4D1043D043E013CD6D2154A002A91
:10D2A0000DD105B03CBC90469946A246AB46F0BDB8
:10D2B0009847E6E74C60D2E728689847E1E743469D
:10D2C0005B684046002B0DD10368002B0ED0494609
:10D2D0000B6000E000BF4B461A68904641460029AB
:10D2E00096D1DEE70368C1469846F7E70023FAE7E0
:10D2F000602F02000000000008B5011C0022002081
:10D30000002302F049FE08BDF0B544465F4656468C
:10D310004D46F0B480468B460C694146096985B09C
:10D3200000208C4200DD90E05D46013C1435A300F6
:10D3300002954746ED1814372968FB180131186823
:10D34000039303F031FA061E42D000218A46029B65
:10D350003A1CAC46B9465546071C0E1CA24602CBE9
:10D360000804000C7843090C79433018040C641845
:10D37000116800040904090C4D19000C281A1568DD
:10D38000260C2404290C240C0514091B491900043B
:10D390000D14000C0904014302C29C45DFD203991D
:10D3A0003E1C096865464F465446002910D1039B30
:10D3B000043B9F420AD21A68002A03D006E019688B
:10D3C000002903D1043B013C9F42F8D3424614613B
:10D3D0004046594601F08CFD002835DB0021894686
:10D3E0000136211C029BB4464C463A1C2E1C894631
:10D3F000116820CB0804000C04192804000C201A22
:10D40000090C2D0C0414491B091900040C14000C00
:10D410000904014302C29E42EAD24C46A300FB1813
:10D420001A686646002A0FD1043B9F420AD21D6843
:10D43000002D03D006E01968002903D1043B013C0C
:10D440009F42F8D342461461301C05B03CBC904664
:10D450009946A246AB46F0BDF0B556464D465F46EE
:10D460004446F0B4016C9DB08246299D029203931C
:10D47000002909D0436C01229A404B608A6001F078
:10D48000D9FA002351460B64039E002E34DB00239F
:10D490002B601F4B321C1A409A421AD0029C039DEB
:10D4A0001A4B194A201C291C03F03EFA002837D0D9
:10D4B000289C2A9D01232360002D00D13AE21548C3
:10D4C000286001381DB03CBC90469946A246AB4648
:10D4D000F0BD114B289C029D2360002D00D10CE271
:10D4E0000E482A9C002CEDD0C278C31C002A00D024
:10D4F00005332A9D2B60E5E77600012376082B6033
:10D500000396C6E7C046C0460000000000000000C9
:10D510000000F07F193102000F27000038310200AF
:10D520001BAB00931AAB019350462B1C221C01F03D
:10D53000E7FD330D834600D1E4E1201CBC4C2A03F7
:10D54000120B211C1143BB4A00241A9F9E181394EE
:10D55000A84BA74A04F082FCA74AA84B04F0EEF9B6
:10D56000A74AA84B03F064FA041C301C0D1C04F0FD
:10D57000D3FFA54AA54B04F0E1F9021C0B1C201CAB
:10D58000291C03F055FA041C0D1C04F091FFA04A5D
:10D59000A04B0890291C201C03F0CCF9002800D0D7
:10D5A000BBE2089D01241194162D0FD8A24AEB006E
:10D5B000D31818685968029A039B03F0CFF9002822
:10D5C00000D1CDE3013D0024089511940024BE1B39
:10D5D0000994013EB14600D5ACE2089C002C00DA6B
:10D5E00092E20025A1440D940B95269C092C00D9AC
:10D5F000A2E10125052C02DD043C26940025269C91
:10D60000032C01D100F0FFFC01DC00F07FFC269C24
:10D61000042C01D100F0FDFB01241094269C052C64
:10D6200000D08BE1279C08996418129401340A9465
:10D63000002C01DC00F037FC00235246536400212B
:10D64000172C0AD9012204235B00181C1430111C6A
:10D650000132A042F8D953465964504601F0C2F94C
:10D6600051460C9008640E2C00D978E1002D00D1B1
:10D6700075E1089D002D01DC00F002FD2A1C0F233E
:10D680006D491A40D2008A180899146855680E111D
:10D69000F20601D400F0C3FC1E40684B02980399C7
:10D6A0001A6A5B6A03F0E0FC0E900F910323984620
:10D6B000002E12D0614F201C291C44460123334206
:10D6C00004D03A687B68013404F038F976100837E2
:10D6D000002EF3D1A0460D1C041C0E980F99221C9D
:10D6E0002B1C03F0C1FC061C0F1C119D002D09D042
:10D6F000301C391C484A494B03F01CF9002801D062
:10D7000000F0A9FD404604F007FF021C0B1C301C72
:10D71000391C04F013F9424A424B03F089F90E9088
:10D720000F910F9B464C0A9D1C190F94002D01D19F
:10D7300000F044FC089C0A9D1894A846109C002CFC
:10D7400001D100F0DEFC43463B4A013BDB00D3182D
:10D750001A685B683448354903F086FC0E9A0F9BC3
:10D7600004F07CFB14901591391C301C04F0A0FED1
:10D77000041C04F0D1FE021C0B1C301C391C04F0EC
:10D780006DFB271C30370C9D0E900F910E9A0F9B4E
:10D79000149815990C9EFFB22F70013603F0DEF835
:10D7A000002801D000F097FD0E9A0F9B1A481B49E4
:10D7B00004F054FB021C0B1C1498159903F0CEF8CE
:10D7C000002801D000F0C3FD4146012900DCC6E07D
:10D7D0004C46199452465C46A8441694B1460E9C99
:10D7E0000F9D149E159F0E923EE0C046C046C04657
:10D7F000000000000000F83F61436F63A787D23F3D
:10D80000B3C8608B288AC63FFB799F501344D33F2F
:10D810000000000000000000000000000000F03FD9
:10D820000000000000001C40000000000000E03F7D
:10D830000000F03F01FCFFFF4831020010320200FF
:10D840000000C0FC221C2B1CBE49BD4804F006FB96
:10D85000321C3B1C03F06EF8002801D000F053FD91
:10D86000C14501D100F05BFD301C391CB64AB74BF5
:10D8700004F064F8B44AB54B061C0F1C201C291C8C
:10D8800004F05CF80D1C041C04F012FE824604F047
:10D8900043FE021C0B1C201C291C04F0DFFA0D1C8B
:10D8A00001210123494299448B4653463033CB44EE
:10D8B000DBB25A46041C13709A46201C291C321CE9
:10D8C0003B1C03F037F80028BCD00E9C169BA246E8
:10D8D000189C9B464E4608945046594601F0AAF8BB
:10D8E00000233370089B289C2A9D01332360002D60
:10D8F00000D108E32E600C98E4E5360300D0EFE594
:10D900009548EEE51A9F1B99944B7D189D4200DACD
:10D9100020E29348934A401B029C8640AB18301C7F
:10D92000DC40204304F036FE8F4A012489186E1E25
:10D9300013940DE68D48C5E5002426940023554632
:10D9400000216B64504601F04DF80126764200211B
:10D9500001240C9028640A961296279110941B9B20
:10D96000002B00DAB2E0089D0E2D00DDAEE0804A0B
:10D97000EB00D3181C685D6804940595279D002D65
:10D9800000DA50E2029C039D049A059B201C291C8E
:10D9900003F06AFB04F08CFD804604F0BDFD049AA0
:10D9A000059B03F0CBFF021C0B1C201C291C04F060
:10D9B00055FA43460C9A30330C9E13700A9B041C94
:10D9C0000D1C0136012B53D05F4A604B03F0B6FFAC
:10D9D0005F4A604B041C0D1C02F0A6FF002800D01B
:10D9E0007AE70C990C9F89460A99023752465B46A2
:10D9F000BA46894402930792049E059F12E0101CC8
:10DA0000191C514A514B03F099FF514A514B0D1CBF
:10DA1000041C01218A44201C291C02F085FF0028D7
:10DA200000D0B2E2321C3B1C201C291C03F01CFB62
:10DA300004F03EFD804604F06FFD321C3B1C03F0F9
:10DA40007DFF021C0B1C201C291C04F007FA021C81
:10DA50000B1C041C0D1C4046514601393030D34686
:10DA60000870CA45CBD1029A079B564693469A4600
:10DA7000221C2B1C201C291C02F0DAFF041C0D1C8C
:10DA8000221C049805992B1C02F054FF00280CD18D
:10DA900004980599221C2B1C02F046FF002800D197
:10DAA0001AE74346DB0700D416E7741E27780C9B61
:10DAB00006E0A34200D1CAE2023E3778261C013CB0
:10DAC000392FF6D00137FFB2277005E7109C002CE4
:10DAD00050D0269D012D00DCCCE10A9C0B9D013C21
:10DAE000A54200DA93E22C1B0A9D002D00DA99E38F
:10DAF000099E0A9B099D5046ED18012109959944FC
:10DB000001F08EF8071C38E0089D099C641B0994FD
:10DB10006C4200250B940D9567E5089804F0FCFC19
:10DB20002B1C221C02F000FF089D43424341ED1ACA
:10DB3000089536E54D466D420995A1464DE5C0462E
:10DB4000000000000000F03F000000000000244042
:10DB500000000000000000002C310200EFFBFFFF7E
:10DB60000EFCFFFF12040000000010FE183102003E
:10DB7000483102000B9C099E0027002E0DD049461B
:10DB800000290ADD4B46B14500DD40E1099D4946CB
:10DB9000ED1AC91A0995F61A89460B9D002D1ADD52
:10DBA000109D002D00D127E2002C10DD391C221C15
:10DBB000504601F0E1F8071C5A46391C504601F066
:10DBC00039F85946051C504600F034FFAB460B9D12
:10DBD0002A1B00D048E15046012101F021F80D9C9C
:10DBE0008046002C05DD41465046221C01F0C4F859
:10DBF0008046269D0024012D00DC8EE10D9D012331
:10DC0000002D00D074E14B441F22134000D19FE04F
:10DC10002022D21A042A00DC9FE31C22D31A099D79
:10DC2000F618ED1809959944099D002D05DD594612
:10DC300050462A1C01F0FCF883464946002905DDC0
:10DC4000414650464A4601F0F3F88046119D002DAA
:10DC500000D02EE10A9D002D00DC71E1109D002D09
:10DC600000D180E0002E05DD391C5046321C01F049
:10DC7000DFF8071CB946002C00D02EE20C9C0A9D50
:10DC8000231C013B5B19029D0D9301231D4042465D
:10DC90000295A0465D46079254460799281CFFF757
:10DCA00033FB031C30330A90391C281C099301F004
:10DCB0001FF9079982464A46201C01F035F9C168D0
:10DCC000061C002900D0E4E0281C311C01F010F9EA
:10DCD0008346311C201C00F0ADFE26995B460B43A9
:10DCE000514603D1029A002A00D1F8E2002900DA55
:10DCF00062E2269953460B4303D1029A002A00D1CF
:10DD0000FAE25946002900DD76E2099A41460A7096
:10DD10000D9946460136884500D17CE2291C0A222D
:10DD20000023201C00F090FE391C051C0A22201C38
:10DD300000234F4500D1A6E000F086FE4946071CAF
:10DD40000A22201C002300F07FFEB0468146A4E793
:10DD50001C2364E7C6480299401B8140081CE1E58A
:10DD60000025119532E40C9AB946002447460A9ED4
:10DD70005D46904606E0291C50460A22002300F02A
:10DD800063FE051C391C281CFFF7BEFA031C303348
:10DD900041460B550134A642EDDC0A9EB846099374
:10DDA000AB464F46002E00DC40E20C9C0025A61935
:10DDB00059465046012201F03BF84146834601F0A6
:10DDC00097F8002800DC32E1741E23780C9A06E0F4
:10DDD000A24200D1D2E0023E3378261C013C392B0E
:10DDE000F6D0013323705046414600F023FE002F49
:10DDF00000D171E5002D05D0BD4203D05046291C4D
:10DE000000F018FE5046391C00F014FE64E5331C87
:10DE1000BCE601241094279900293DDD0C1C1291C9
:10DE20000A91FFF709FC0A9C002C00DDAAE500D04E
:10DE300085E28C4B8A4A0498059903F07FFD029A8B
:10DE4000039B02F095FD002800D1FCE000229046E3
:10DE50000027279C0C9EE44308945046414600F05E
:10DE6000E9FD002FCED137E55946504600F084FF3A
:10DE70008346B0E6139C002C00D1D9E17D4D0B9C6C
:10DE80005B19099E36E600F0DFFDB046071C8146AF
:10DE900003E7012293461CE701230121012201240B
:10DEA00012930A912792514600234B640021FFF7F9
:10DEB000D4FB5846414601F01BF8002800DBC9E6B8
:10DEC000089D5946013D50460A220023089500F05E
:10DED000BBFD129D83460A95109D002D00D1B9E629
:10DEE000391C50460A22002300F0AEFD071CB1E6A3
:10DEF00041460B6903339B004344586800F044FEDD
:10DF000020231B1A7FE60C98FFF7DCFA00241094FC
:10DF1000269C022C00D17EE710E50299002900D052
:10DF20006CE6039A130300D068E6534B134200D10A
:10DF300064E6099C012501340994A94401245DE6A5
:10DF4000269D022D00DC89E60A9C002C81D14146E9
:10DF500050460522002300F077FD80464146584692
:10DF600000F0C6FF002800DC73E7089D0C9E0C9CA7
:10DF7000312301350136237008956EE7089C312363
:10DF8000013408940C9C23702DE70299079A5E4691
:10DF900092468B46A0E4404604F0BEFA021C0B1CDD
:10DFA000301C391C03F0CAFC2F4A304B02F040FDF4
:10DFB0000E900F910F99314A8A180F92294B284AD7
:10DFC000301C391C03F04AFF0E9A0F9B041C0D1CD9
:10DFD00002F0C4FC002836D1201C291C0F9C80258F
:10DFE0002D060E9A631902F0A5FC002800D1B6E4B4
:10DFF0000025A84600272CE7594650460B9A00F00A
:10E00000BBFE8346E7E500241094FFF70BFB0B9D56
:10E010000B94631B0D9D0024ED180D9564E502998A
:10E02000039A0E910F9202229046FFF741FB0028BF
:10E0300004D1099CE40701D5C6E61E1C731E1A789C
:10E04000302AFAD0CFE60025A84600278DE7089DA4
:10E050003023013508950C9D31272B7027703BE448
:10E0600000000000000014400000000000001C4000
:10E07000EEFBFFFF330400000000F07F0000C0FC57
:10E08000089D6C42002C00D1D8E00F232340BC4AED
:10E09000DB00D318029803991A685B6803F04EFC02
:10E0A0002411061C0F1C002C00D14CE102218846D3
:10E0B000B44D301C391C46460122224204D02A6845
:10E0C0006B68013603F03AFC64100835002CF3D17C
:10E0D000B0460F1C061CFFF708FB7968504600F09D
:10E0E00081FC3A69391C0232041C92000C310C305C
:10E0F000FDF74EFC5046211C012200F099FE81469E
:10E10000BCE54546013D9E4AEB00D31818685968A6
:10E110000E9A0F9B149503F011FC16901791391C61
:10E12000301C04F0C5F90E9004F0F6F90B1C021C2B
:10E13000391C301C03F092FE0E9F0D1C0C9E0C9996
:10E1400030370F70013641444346041C371C0E9192
:10E15000012B1ED0B046201C291C844B824A03F0A0
:10E16000EDFB041C0D1C04F0A3F9061C04F0D4F90B
:10E17000021C0B1C201C291C03F070FE30360E9C68
:10E180003E700137A742E8D10D1C14994646041C85
:10E190007618774A774B1698179902F049FC221C9B
:10E1A0002B1C02F0C7FB002800D180E0189D741ED4
:10E1B000277808950C9B83E4079A5E46A246AB46F7
:10E1C00044469046002E11DD59465046012200F08B
:10E1D0002FFE4146834600F08BFE002800DCA6E0BF
:10E1E000099D392D30D00A9D31350995099D661C50
:10E1F00025703D1C4F46F6E5AB46079A099DA246A1
:10E2000044469046392D1FD0099B3D1C0133661CA6
:10E2100023704F46E7E5AB46079DA246A8463D1C46
:10E220004F46C5E5099900234E1B63E40126BCE572
:10E230001A9936235B1A0B9C099E5BE40223029E0B
:10E24000039F9846FFF751FA39233D1C661C237043
:10E250004F460C9AC3E50A9C002C00D19BE6129D08
:10E26000002D01DCFFF77BFB089C404B3E4A301C35
:10E27000391C013C189403F061FB061C4046013038
:10E280000F1C04F049F9021C0B1C301C391C03F054
:10E2900055FB394A394B02F0CBFB0E900F910F9D85
:10E2A0003949129A69180F919046FFF747FA169A62
:10E2B000179B2F482F4903F0D1FD221C2B1C02F085
:10E2C0004DFB002801D1FFF74AFB00E01E1C731E26
:10E2D0001A78302AFAD0189D0895FFF7FDFAAB4658
:10E2E000079A099DA246029144469046392DABD02B
:10E2F000002900DD77E779E7079B5E46A246AB463B
:10E30000444698465EE70E9D57461699AA46189DC4
:10E310005C464E468B4608950C9BFFF7D1FB199A3D
:10E32000169B0E9C91469B46A246FFF718FB0028C1
:10E3300000D05BE7099DED0700D457E750E70021C7
:10E340008846002785E50224A046FFF7CEF9189CF1
:10E3500008940C9C231CFFF7B3FB042A00D163E450
:10E360003C22D31A5BE4C0460000000000002440B9
:10E37000000000000000E03F0000000000001C4022
:10E3800048310200103202000000C0FCC046C04606
:10E3900038B5094B094DED1AAD1009D0013DAC005F
:10E3A000E41800E0013D23689847043C002DF9D1B2
:10E3B00004F024FD38BDC046D0280020D428002019
:10E3C00038B5141E05D0101C0B4900F0E3FF0028DF
:10E3D00002D10A4D281C38BD084D201C291C00F014
:10E3E000D9FF0028F6D0201C054900F0D3FF434296
:10E3F000584140422840EEE73C3102005C2F0200C9
:10E40000F83002000048704794240020014B18683F
:10E410007047C046B4240020004870473C240020C8
:10E4200000207047004870475C24002008B50A1C93
:10E430000349031C0868191CFFF7C2FF08BDC0464A
:10E4400038240020004870475C240020F0B5564670
:10E4500044465F464D46F0B40C1C0B3483B0061C9A
:10E46000162C2BD907239C432BD4A14229D8301C2E
:10E4700000F0B4FAF823FF339C4226D8E208CA4DD4
:10E48000D300EB18DF689F4200D1BBE1786803231B
:10E49000FA68B96898433B18CA60916059680122CC
:10E4A0000A43301C5A6000F09BFA381C083003B055
:10E4B0003CBC90469946A246AB46F0BD1024A14212
:10E4C000D5D90C2333600020F1E7630A00D18EE038
:10E4D000042B00D93DE1A30938339C465900B24DC5
:10E4E00089006918CF68B94215D07A6803239A4326
:10E4F000101B0F2800DD8DE000287CDA032007E0E8
:10E500007A688243131B0F2B00DD83E0002B72DA45
:10E51000FF68B942F4D1012294442B1C2F690833BF
:10E520009F4200D163E1786803229043021C011BE3
:10E530000F2900DD4AE16B612B6100295FDA9B4BFB
:10E54000984200D90FE1C3089A100121DB00EB18B3
:10E55000914068680A1C99680243FB60B9606A6070
:10E560009F60CF6061468B1001219940914255D840
:10E5700011420DD1032360469843031C0433490024
:10E580009C46114204D1042349009C441142FAD014
:10E59000032080466246D3005B199A46181CE14668
:10E5A000C768B84207D124E1002B00DB33E1FF68E4
:10E5B000B84200D11DE17A6843469A43131B0F2BE2
:10E5C000F2DD01213A190C437C60F868BC6808351B
:10E5D000E06019438460EA60AA60301CD5609560F1
:10E5E0005160D35000F0FCF9381C08305FE73F223F
:10E5F0007E21944673E7FB68B968CB609960BA18CE
:10E60000516801230B43301C536000F0E9F9381CBA
:10E6100008304CE70120404284447CE7AF68032384
:10E62000786898438146A04203D3031B0F2B00DD7B
:10E6300081E05F4A5F4B49461B6810687918019179
:10E64000E3189346013000D147E15B495B181B0B8F
:10E650001B030093301C009900F08AFE021C8046C8
:10E6600001325DD0019B834200D9EBE05348009911
:10E67000026882468B1801990360414500D135E15B
:10E680005A461268013200D143E1019841460A1A04
:10E690009B1851460B6007234246134000D104E10A
:10E6A000D21A08329046464AD31A0098021C4244B5
:10E6B0001205120D9A1A111C301C934600F058FED8
:10E6C000411C00D121E14246801A584401231843DD
:10E6D000524611680B1C5B444146A96013604860B8
:10E6E000AF4213D04A460F2A00D8E9E04A4678687C
:10E6F00007210C3A8A43012101401143796005202A
:10E70000B918486088600F2A00D906E12D4A1068C0
:10E71000834200D913602C4A11688B4200D91360E0
:10E72000AF6803237A689A43131B944200D9AEE082
:10E730000F2B00DCABE00122211C11433C191343D9
:10E740007960301CAC60636000F04AF9381C083016
:10E75000ADE6142B6ED9542B00D99DE0230B6E33FC
:10E760009C465900BBE6430A042B67D9142B00D9F9
:10E77000B6E0191C5B31480080004019836881466F
:10E78000834200D194E00321884659684046814382
:10E790008A4202D29B689945F7D1D9686A68F960C4
:10E7A000BB608F60DF60DDE6B8240020FF01000061
:10E7B000C4280020602D00200F100000642D0020D0
:10E7C000081000005C2D0020582D002001203A196F
:10E7D000044308437C606A612A615060D36093609F
:10E7E000301C515000F0FCF8381C08305FE66A68B5
:10E7F000B8E60122914443464A460830134200D00D
:10E80000CEE62CE03B1C7F69023208339446BB42C3
:10E8100000D182E63AE6BA185068012303435360F8
:10E82000FB68BA68301CD3609A6000F0D9F8381CD5
:10E8300008303CE65B339C46590050E6810938318C
:10E84000480099E7AF4200D06AE70FE753461868DF
:10E8500001225242083B94448246984277D1434673
:10E8600060460342F2D16B688B436B60490099426A
:10E8700000D9D3E6002900D1D0E6CC46194200D019
:10E8800088E60422490094441942FAD082E6301CFA
:10E8900000F0A6F800200AE6AA225200934214D8FB
:10E8A000E30B77339C46590019E680235B01FCE6B5
:10E8B0008910686801228A4002436A60191C6EE769
:10E8C00001234B60474600222EE7224A934218D884
:10E8D000A30C7C339C46590001E610330093B9E643
:10E8E000542B22D8010B6E31480045E70A0500D0B1
:10E8F000C6E60099AA68081C4844012101435160FA
:10E9000004E77E23FC219C46E9E5002301209B4689
:10E91000DEE6434658460360BDE6391C0831301C2C
:10E9200001F01AFC51460B68F0E6AA2149008B421F
:10E9300003D8C10B773148001EE706498B4203D844
:10E94000810C7C31480017E7FC207E2114E76B68BE
:10E950008CE7C04654050000F0B5CCB2830737D031
:10E96000531E002A1FD00278A2421DD0032505E0C5
:10E97000002B18D00278013BA24215D0013028426A
:10E98000F6D1032B11D8002B0DD00278A2420BD068
:10E99000421CC31804E00132511E0978A14203D081
:10E9A000101E9842F7D10020F0BDFF2631400E0224
:10E9B00031430E04074D0E430268074F7240D119D0
:10E9C00091432942DFD1043B0430032BF4D8DAE72A
:10E9D000131CD6E780808080FFFEFEFE7047C04695
:10E9E0007047C046C36C70B5041C0D1C002B0AD0C8
:10E9F000AA009A18106800280ED00368136000223D
:10EA00000261C26070BD0421212201F025FBE06497
:10EA1000031EEDD10020F5E70126AE40721D9200E5
:10EA2000201C012101F018FB0028F3D0456086600E
:10EA3000E5E7C046002906D04A689300C26CD318A7
:10EA40001A680A6019607047F8B54D4644465F463B
:10EA5000564698460B69F0B40D1C83468A46994683
:10EA6000143500242E68013437043F0C5743360C0C
:10EA7000564347443B0C9E193F04310C3F0C36046F
:10EA8000F619884640C5A145ECDC00290DD0524658
:10EA90009268914510DA4B4604339B00534442463A
:10EAA0005A604B46013351460B6150463CBC904680
:10EAB0009946A246AB46F8BD5346596858460131BF
:10EAC000FFF790FF53461A6951460232041C0C317D
:10EAD00092000C30FCF75CFF514649688B005946A8
:10EAE000CA6C5146D3181A68A2460A601960D2E768
:10EAF000F8B54F464646C0B4071C181C0C1C08301D
:10EB000009219046994601F09DFE01283ADD012534
:10EB100000216D000131A842FBDC381CFFF762FFC9
:10EB2000089B011C4361012303614346092B25DD3A
:10EB3000261C0936351C44442B78381C303B0A22ED
:10EB4000FFF782FF0135011CA542F5D14346F418B9
:10EB5000083CC1450DDD4B46E5184346ED1A2378C8
:10EB6000381C303B0A22FFF76FFF0134011CAC4216
:10EB7000F5D1081C0CBC90469946F8BD09230A340F
:10EB80009846E6E70021C8E7031C010C0022002993
:10EB900001D103041022190E01D108321B02190FF2
:10EBA00001D104321B01990F01D102329B00002BCD
:10EBB00005DB2020590000D47047501CFCE7101CD6
:10EBC000FAE7C0460368011C580708D00020DA079E
:10EBD00004D4980720D49B080B60022070471804C7
:10EBE0000022002801D11B0C1022FF20184201D165
:10EBF00008321B0A180701D104321B09980701D1FA
:10EC000002329B08D80704D45B082020002BE5D0F3
:10EC100001320B60101CE1E75B080B600120DDE7AF
:10EC200010B50C1C0121FFF7DDFE012344610361D7
:10EC300010BDC046F0B55F4656464D464446F0B45A
:10EC40000F69146985B00E1C151CA74204DA3B1C21
:10EC5000161C271C0D1C1C1CB3683A1971689046C1
:10EC60009A4200DD0131FFF7BDFE14214246834682
:10EC70008B4493005B44191C039302905B46002273
:10EC80008B4503D2039904C39942FCD81435AA4694
:10EC9000A4001436BF0054440096F7190194A5420D
:10ECA0004CD251460D682C04240C1FD0009A5B46B0
:10ECB0000025196840CA0804010C3004000C6043A8
:10ECC000360C0818664340191D689946290C8919A5
:10ECD000050C491900040D0C000C0904014302C382
:10ECE0009742E6D849464D60524615682D0C1FD014
:10ECF0005B4619680026009A081C341C1688000C14
:10ED00006E433618361909043004090C01431960A2
:10ED100010CA5868240C6C430104090C6118360CA5
:10ED200089199C460C0C04339742E7D86546696004
:10ED30000421019A8A448B445245B2D84346002BA1
:10ED40000EDD039B043B1D68002D09D1424603E004
:10ED5000043B1968002902D1013A002AF8D19046F3
:10ED6000029B4246181C1A6105B03CBC904699466D
:10ED7000A246AB46F0BDC046F8B546464F46032313
:10ED8000C0B480460E1C141C134036D1A41023D0EE
:10ED900041468D6C002D39D000230127994627422A
:10EDA00007D1641018D0286800281AD0051C274203
:10EDB000F7D04046311C2A1CFFF73CFF002E1AD02A
:10EDC00071684246D26C8B00D318196864103160A8
:10EDD0001E60061C002CE6D1301C0CBC90469946E7
:10EDE000F8BD2A1C291C4046FFF724FF4A4628602C
:10EDF0000260051CDBE7061CD3E70B4A013B9B00C6
:10EE00009A580023FFF720FE061CBFE74046012169
:10EE1000FFF7E8FD054B42464361012303610023F0
:10EE20009064051C0360B7E73832020071020000ED
:10EE3000F0B54D46444656465F46F0B40E1C83B0CE
:10EE40000190306955114019041CB3680134914692
:10EE5000496880469C4203DD01315B009C42FBDC3B
:10EE60000198FFF7BFFD011C00901431002D08DD53
:10EE70000A1C00230027013380C2AB42FBD19B0058
:10EE8000C9183269331C950014331F224F465D198F
:10EE9000174027D02022D21B94460A1C0021186854
:10EEA0009246B840014302C202CB6046C1409D4237
:10EEB000F5D852465160002901D0444602340199E8
:10EEC0007068009BCA6C013C1C618300D3181A68EF
:10EED000009832601E6003B03CBC90469946A24642
:10EEE000AB46F0BD0A1C02CB02C29D42FBD8E6E74E
:10EEF00010B50B690469E21A11D19A00143014316B
:10EF00008318891801E098420BD2043B04391C682D
:10EF10000A689442F7D09442924101231A43101C8C
:10EF200010BD0022FBE7C046F8B54F464646C0B4C8
:10EF30000C1C071C081C111C161CFFF7D9FF051E12
:10EF40005DD0002856DB00256168381CFFF74AFDBC
:10EF50008446C5602069231C14338200D218904671
:10EF60003269351C143592005219644691461434A6
:10EF7000002104CB80CD1604360C71183E04360CEB
:10EF80008E1B120C3F0C3114D21B52183604360C57
:10EF90001114043412043243261F3260A945E8D804
:10EFA0009946984517D9271C40CB35042D0C6D1870
:10EFB0002A14360C92192D0411142D0C12042A4314
:10EFC00004C79845F0D84946CB4343449B080133D6
:10EFD0009B00E418261F331C002A04D1043B1A6846
:10EFE0000138002AFAD06346186160460CBC90468E
:10EFF0009946F8BD231C0125341C1E1CA4E7381CAF
:10F000000021FFF7EFFC012303614561EEE7C046F5
:10F010000E4B0F4A0B409B1810B5002B02DD191C3C
:10F02000002010BD5B421B1500200021132B07DDC3
:10F030000122322B02DC3324E31A9A40101CF0E741
:10F0400080221203111C19410020EAE70000F07F22
:10F050000000C0FCF8B546464F46C0B40769061C20
:10F060001436BF00F7193C1F25688846281CFFF797
:10F070008BFD20231B1A41460B600A281ADC0B2348
:10F080001B1A2A1CDA401D4991469C460B1C494616
:10F090000B430021A64203D2083F39686446E14091
:10F0A000153085400A1C2A43101C191C0CBC9046C4
:10F0B0009946F8BD0021A64202D23C1C083C2168BA
:10F0C000071C0B3F002F13D02B23181A0B4BBD40EE
:10F0D0002B439C460D1CC54063462B430025B44280
:10F0E00002D9043C2568C540B9402A1C0A43DBE725
:10F0F00002480A1C031C2B43D6E7C0460000F03F21
:10F10000F0B5012183B01D1C141CFFF76BFC2B0311
:10F110006A00061C1B0B570D02D0802252031343BA
:10F120000193002C1AD068460094FFF74BFD00288D
:10F1300031D1009B019C7361B4616342634102243D
:10F14000E41A3461002F14D0194A0899BB181B180F
:10F150000B60099A3523181A106019E001A8FFF70F
:10F1600031FD019901237161336120300124002FA9
:10F17000EAD1104B104AC018A31808999B00F31845
:10F1800008605869FFF700FD6401099B241A1C60A0
:10F19000301C03B0F0BD019C20231B1A211C994098
:10F1A000009A0B1C1343C44073610194C4E7C0462A
:10F1B000CDFBFFFFCEFBFFFFFFFFFF3FF0B5574644
:10F1C0004E464546E0B484B0894602A98046FFF722
:10F1D00041FF061C0F1C484603A9FFF73BFF021C1A
:10F1E0000B1C0298039900920193401A41468246F3
:10F1F00008698446484601696046411A49015144FC
:10F2000000290CDD0905CD192F1C301C391C01F01B
:10F210002BFF04B01CBC90469946A246F0BD019B52
:10F220000905591A0191009A019BEEE700000000C0
:10F2300010B5041E172C09DD08490748084A094B78
:10F24000013C02F07BFB002CF8D110BD064BC40042
:10F250001C1920686168F8E7000000000000F03F1A
:10F26000000000000000244048310200C046C046B3
:10F2700070B54E1E11697611131C013614338D00C2
:10F28000B6005D198619AB420AD2011C10CB10C121
:10F290009D42FBD8AB1A153B9B0801339B00C0185D
:10F2A0000023864202D908C08642FCD870BDC04601
:10F2B0000369021C10B51432481183420FDA9B0017
:10F2C000D3189A4221D2043B1868002804D01AE0CF
:10F2D000043B1968002916D19A42F9D310BD834224
:10F2E0000EDD1F2319408300D3180029E9D01C68C4
:10F2F000201CC8408840011C0120A142EED1E0E75B
:10F300008300D318DDE70120E8E70020E6E7C046E8
:10F310000B1C011C021C30B519430220002900D12E
:10F3200030BD802109068B4216D00D4904205C189F
:10F330000C498C42F4D90C4D5C198C42F0D90B4C21
:10F34000590049080320A142EAD9074C0020A142F4
:10F35000E6D150425041E3E7002AE1D0EFE7C04652
:10F360000000F0FFFFFFDF7F0000F07FFFFF0F00D6
:10F3700038B5074C0023051C081C236003F01CFD56
:10F38000431C00D038BD2368002BFBD02B60F9E76D
:10F39000902D002002780B7801300131002A01D035
:10F3A0009A42F7D0D01A7047F0B556464D464446BB
:10F3B0005F46F0B4936883B001900D1C90461668C8
:10F3C000002B00D17CE00868002400218946AB684E
:10F3D000002C45D01F1C9C424BD39022AB89D200FD
:10F3E000134249D029696A69401A8346500082183D
:10F3F000D00F821852109246621C5A44924554D241
:10F4000092468020C000034238D00198111CFFF7BB
:10F410001DF8071E57D05A462969FCF7B9FAAA8980
:10F420002B4B134080221343AB8151465B46F818A7
:10F43000CB1A2F6128606961271CAB60A246494640
:10F44000524600F051FF2A684146AB688968101C9B
:10F45000DB1B50440C1B4246AB602860946026D0F6
:10F460003168746889460836002CF9D01F1C9C420C
:10F47000B3D2271CA246E2E7BA46E0E7019800F0C3
:10F4800085FF071ED1D10198296900F065FE019A18
:10F490000C231360AA8940231343AB814046002309
:10F4A000836043600120404203E05246A9E7546074
:10F4B000002003B03CBC90469946A246AB46F0BD46
:10F4C00053600020F5E701990C230B60E2E7C0468A
:10F4D0007FFBFFFFF0B556464D465F464446F0B40D
:10F4E000AFB00C900B938B898A469146180604D5D1
:10F4F0000969002901D100F016FD1EA8002300248F
:10F5000000258346119013931293061C0D940895C1
:10F51000484603784C46002B1CD0252B02D119E01D
:10F52000252B3CD001342378002BF9D14946651AAC
:10F53000002D0FD013984B4633602B181393129B5A
:10F54000756001331293072B00DDD1E3083608996B
:10F55000491908912378002B01D100F09CFC3F252C
:10F56000621C00236D44012791462B707F4280224C
:10F57000637800250024102103970594904600200D
:10F58000019520248C4640274A460132191C203917
:10F59000582900D926E2CC4D890069588F464A4641
:10F5A000A51AC5E70B9D0B992D6804310595002D13
:10F5B00001DB00F00DFC059D0B916D420595019D51
:10F5C00004231D4301951378DFE713782B20DCE734
:10F5D000019D01231D4301951378D6E71378002878
:10F5E000D3D12020D1E73F256D442870B74C019D31
:10F5F00091460D94AD0600D4E6E00B9A0721073240
:10F600008A43141C08340B941468556806940795B3
:10F61000019DED0700D4A5E3069907980222014356
:10F620001AD010A830240470019C43701443019434
:10F6300012E0019D9146AD0600D47FE10B9B0722AD
:10F64000073393431C1C08340B941C685D680694B4
:10F650000795211C01222943039C3F200023684475
:10F66000049403700024039D002D03DB019D80237F
:10F670009D430195002900D083E2039D002D00D019
:10F680007FE25D46002A03D10198C00700D5A3E3BD
:10F69000049B03980293834200DA02900299631E4E
:10F6A0009C41091902913CE00B9C0B9F3F2025686F
:10F6B00000236844914604370370002D01D100F007
:10F6C00024FC039C281C002C01DA00F010FC002113
:10F6D000221CFFF741F9002801D100F036FC401B45
:10F6E0000490A04200DD04943F2068440021047887
:10F6F0000B970391CCE7019D25430195137844E7CF
:10F700000B9B0B9C1B68043414AD3F200B942B7097
:10F710000124002368449146037002940494002459
:10F720000394019C02231C40099402D0029C0234E1
:10F730000294019C84231C400A9400D072E1059835
:10F740000299441A002C00DC6CE1139A129B604F62
:10F75000102C24DD1020311C80465646AA460C9DF4
:10F7600003E0103C0831102C16DD40461032013306
:10F770000F60486013921293072BF2DD281C311C96
:10F7800011AAFFF711FE002800D020E2103C139AC6
:10F79000129B5946102CE8DC5546B2460E1CA218A6
:10F7A00001333760746013921293072B00DDCDE2B2
:10F7B000083639E19146474C3F22019D6A4410705A
:10F7C0000D94AD0600D518E7019DED0600D52FE399
:10F7D000019D6D0600D480E30B9C002524880795CD
:10F7E00006940B9C04340B9412E73F25019C6D4456
:10F7F00091462870A40600D5F6E2019DED0600D5DD
:10F8000033E3019C640600D42FE30B9D089C2D6814
:10F810002C800B9D04350B957AE61378111C6C2B0C
:10F8200000D11BE3019D61460D430195ADE6019DAD
:10F830003D4301951378A8E63F21019D6944914617
:10F840000870AD0653D50B9A072307329A43141C50
:10F850005368126808340B9406920793002B52DB0E
:10F860003F256D442C780699039D07980495012245
:10F870000143F8E60B9B0B9D1B68019C0693043526
:10F8800002231C43914610AB30220B950F4D0020F4
:10F890001A7078225A70079001940D9502220699E9
:10F8A000DAE6019D9146AD0663D50B9B072207332F
:10F8B00093431C1C08340B941C685D68211C06943F
:10F8C000079500222943C7E670320200FC3002008F
:10F8D000E4330200E8300200019C10233F251C4362
:10F8E0006D4401942870019D9146AD06ABD4019DF5
:10F8F000ED0600D48EE20B9C236804340693DB17DC
:10F9000007930B94ACD506980799002544428D4186
:10F910003F210694079569442D23039C0B7006999B
:10F92000049401222D2429439DE6019C10231C43AD
:10F930000194019D9146AD0600D57FE6019DED063F
:10F9400000D55BE2019D6D0600D4AEE20B9C002564
:10F950002488079506940B9C012204340B94069985
:10F960007AE6019C10231C430194019D9146AD064B
:10F970009BD4019DED0600D564E2019D6D0600D487
:10F980009FE20B9C00252488079506940B9C00227F
:10F9900004340B9406995FE6019D41460D430195A1
:10F9A0001378F2E51378551C2A2B00D1D7E2191CE5
:10F9B00030390022092900D9C2E2930001359A1892
:10F9C0006B1E1B7852008A18191C30390929F4D98A
:10F9D000002A00DA96E2191C203903922A1C5829C1
:10F9E00000D8D8E591463F226A441070002B00D120
:10F9F00051E214AD01242B7000231370029404947F
:10FA00008DE60025191C05953039AB0001325D19D2
:10FA1000531E1B786D006D18191C30390929F4D953
:10FA20000595B3E5139A129B3F246C442178002975
:10FA30000AD00121013201333460716013921293B4
:10FA4000072B00DD6AE10836099C002C0BD010A9B9
:10FA50003160023202210133716013921293072B3D
:10FA600000DD67E108360A9C802C00D1BEE0039CD3
:10FA70000498271A002F31DDBD4C102F24DD1021F2
:10FA80008846311C5646AA460C9D03E0103F0831BB
:10FA9000102F16DD4046103201330C60486013927F
:10FAA0001293072BF2DD281C311C11AAFFF77CFCF6
:10FAB000002800D08BE0103F139A129B5946102F5C
:10FAC000E8DC5546B2460E1CD2190133346077602B
:10FAD00013921293072B00DD14E10836049C0133C6
:10FAE00012193560746013921293072B00DDB5E094
:10FAF0000836019D6D0735D5059C0298251A002D05
:10FB000030DD129B9B4F102D23DD311CB846102495
:10FB10000C9E574603E0103D0831102D16DD954828
:10FB20001032013308604C6013921293072BF2DD00
:10FB3000301C391C11AAFFF737FC002800D09CE1CB
:10FB4000103D139A129B5946102DE8DCBA460E1C44
:10FB50004746521901333760756013921293072B91
:10FB600000DD2BE1029B059CA34200DA231C089DCB
:10FB7000ED180895002A00D07AE0002312935E4623
:10FB8000C6E4012A00D1A4E06B467733022A00D0F4
:10FB900077E0A4460D9C0F21B046181C069A079BDF
:10FBA000051C081C1040205C1E071709321C287019
:10FBB0003A431809031C171C681E1F43F0D1069214
:10FBC00007935B465B1B46466446049360E5B2467A
:10FBD00051468B8908985A0601D5012040422FB022
:10FBE0003CBC90469946A246AB46F0BD059C0298A7
:10FBF000271A002F00DC3AE75D4C102F23DD10217F
:10FC00008846311C5646AA460C9D03E0103F083139
:10FC1000102F15DD4046103201330C6048601392FE
:10FC20001293072BF2DD281C311C11AAFFF7BCFB35
:10FC30000028CCD1103F139A129B5946102FE9DCB3
:10FC40005546B2460E1CD2190133346077601392C8
:10FC50001293072B00DD12E1083608E70C98514695
:10FC600011AAFFF7A1FB0028B2D1139A5E4640E724
:10FC70000C98514611AAFFF797FB002800D17CE7AA
:10FC8000A6E70720B046A446191C069A079B071C46
:10FC900017405E07D4083037321C0D1C0F7022430A
:10FCA000D9080B1C141C691E1C43F0D10198069244
:10FCB000079346460B1C6446291CC00714D5302FF9
:10FCC00078D01D1C013930230B705B465B1B0493FD
:10FCD000DEE4079D002D4FD1069809284CD86D46CB
:10FCE000031C773530332B705946491B0491CFE400
:10FCF0000C98514611AAFFF757FB002800D067E780
:10FD00005E4624E40C98514611AAFFF74DFB0028EB
:10FD100000D05DE7139A129B5E46DFE60C985146D1
:10FD200011AAFFF741FB002800D051E7139A129B5C
:10FD30005E4689E60C98514611AAFFF735FB00286C
:10FD400000D045E7139A129B5E468CE60C9851460C
:10FD500011AAFFF729FB002800D039E7139A129B5C
:10FD60005E4661E60699079D0222294374E4C04677
:10FD7000D4330200E43302006B467733A046069C7E
:10FD8000079D1F1C201C291C0A22002300F0FAFDDD
:10FD900030323A70201C0A220023291C00F0F2FDA8
:10FDA000021C041C0D1C7B1E0A43EAD10694079515
:10FDB0003D1C44465A46521B049269E40C98514635
:10FDC00011AAFFF7F1FA002800D001E7139AC9E65B
:10FDD00013780B91FFF7D9FB6D46773559463023E1
:10FDE000491B2B70049153E40B9D089C2B68E21770
:10FDF00004351C605A600B95FFF78AFB0B980B9C2F
:10FE0000006800210434079106900B940122011C24
:10FE1000FFF722FC019D0B9C6D0600D46CE50023CE
:10FE2000E35E0B9D06930435DB1707930B9515E5F1
:10FE30000B980B9C006800210434069007910B94EA
:10FE4000FFF7E6FB0B980B9C006800210434079138
:10FE500006900B940022011CFFF7FEFB019D01326E
:10FE6000254301954B78FFF790FB0B9C089D236879
:10FE700004341D600B94FFF74BFBBA46A8E60C98C0
:10FE8000514611AAFFF790FA002800D0A0E6139A75
:10FE9000129B5E46EBE51398002800D198E60C987B
:10FEA000514611AAFFF780FA92E60B9D0B9C2D6834
:10FEB00000200434069507900B940122291CFFF7BB
:10FEC000CBFB0B9D0B9C2D680020043406950790FE
:10FED0000B940022291CFFF7BFFB0B9D0B9C2D6888
:10FEE00000200434069507900B94FFF791FBFBF775
:10FEF00045FE3F226A440023049014780B97039335
:10FF0000FFF7C6FB0122524265E5039B062B00D991
:10FF100006230493049CDB43DB171C4002940B97DD
:10FF20001C4DFFF7FCFB0C984021FEF78FFA524660
:10FF30001060106100281ED040235361FFF7DDFAE6
:10FF40002A1C00250395FFF721FB03993F206844F5
:10FF5000002204780B9704910392FFF799FB0B9B07
:10FF60000B991B6804310393002B0ADB53780B9128
:10FF70002A1CFFF70AFB0C9C0C2301202360404243
:10FF80002DE60B9101214942537803912A1CFFF77A
:10FF9000FCFAC04610310200F0B54F464646C0B4E8
:10FFA00098462B4BA4251B686D005C5983B0061C3A
:10FFB0000F1C91460193002C44D065681F2D1ADD5B
:10FFC000244B002B02D1012040421CE0C8204000FD
:10FFD00000E000BF041EF6D000254560A423019870
:10FFE0005B00C05801992060CC50C4235B00E550F1
:10FFF000C6235B00E550002E0AD16B1C0235AD0014
:020000022000DC
:10000000636000202F5103B00CBC90469946F0BDB0
:10001000AB00E318882248469850C42040002218BC
:1000200010680121A9400843106084225200404614
:100030009850022EE1D1C6225200A318186801433D
:100040001960DAE71C1C4D34FF345C51B5E7C0463B
:10005000602F02000000000010B55143FEF7F6F9D2
:10006000041E27D0031C083B5A6803239A43043A12
:10007000242A15D8031C132A05D800221A605A60B6
:100080009A60201C10BD00210160416008331B2ACA
:10009000F3D98160C160242A07D0031C1033ECE738
:1000A0000021FBF7B7FC201CECE7031C01611833AF
:1000B0004161E2E70020E5E7F8B50F1C041CFEF7FC
:1000C0008DFC204D204AAB685E6803239E43F71BDE
:1000D000BF183F0B1D4B013F3F039F4207DD201C14
:1000E0000021FFF745F9AA689319984204D0201C13
:1000F000FEF776FC0020F8BD7942201CFFF738F9A6
:1001000001300DD0AB68F61B012216435E60104B28
:10011000201C1A68D71B1F60FEF762FC0120EAE76B
:10012000201C0021FFF724F9AB68C21A0F2ADEDD7C
:1001300008490968401A0649086001210A435A60C3
:10014000D5E7C046B8240020EF0F0000FF0F0000E5
:10015000642D0020C4280020F0B5474680B4051C5B
:100160000C1E55D0FEF73AFC211C083948680127BF
:10017000031CBB43CA185468804603208443201CD8
:10018000534CA668964260D00026B446464650605E
:1001900037420AD10E68271C891B9B198E680837C5
:1001A000BE426BD0CF68F760BE6016187668012734
:1001B0003E4207D11B18604600282CD09068D268B8
:1001C000C26090600122181C104366464860CB5004
:1001D000002E1AD13F48834229D95A0A042A50D8FE
:1001E0009E093836700080002018826882424ED006
:1001F00003265468B443A34202D292689042F8D1D5
:10020000D368CB608A609960D160281CFEF7E8FB58
:1002100004BC9046F0BD90682F4EB042CFD11F4332
:10022000C1608160C86088604F60CB50EDE7DB083B
:10023000981082406068DB0002436260E418A368A3
:10024000CC608B60A160D960DFE7C31840460742ED
:1002500006D10A68891A88689B18CA68C2609060CB
:1002600001221A434A601D4AA16012689342CCD30E
:100270001B4B281C1968FFF71FFFC6E70126B44671
:1002800093E7142A0CD8161C5B367000ABE7B61047
:100290000123B3401E1C63681E436660131CB0E755
:1002A000542A03D81E0B6E3670009CE7AA2040002B
:1002B000824203D8DE0B7736700094E70948824209
:1002C00003D89E0C7C3670008DE7FC207E268AE7E2
:1002D000B8240020FF010000C0240020C028002016
:1002E000602D002054050000F0B588420ED98D180D
:1002F000A8420BD28618531E5142002A05D06A1814
:10030000D45C7218D454013BF9D2F0BD0F2A09D83D
:10031000051C002AF9D00023CC5CEC540133934235
:10032000FAD1F2E7031C0B439C072AD1171C103F9C
:100330003F093E01861910360C1C031C25681D6000
:1003400065685D60A5689D60E5681034DD60103308
:10035000B342F3D17D1C2D010F23491913404519D8
:10036000032B10D91E1FB6080136B6000023CC5847
:10037000EC500433B342FAD10324ED18C9182240DB
:10038000C7E7051CC7E71A1CC3E7C046F0B54D46D2
:1003900044465F465646F0B4804685B00D1C9146F3
:1003A00000D1DDE02E1C083EFEF718FB73684F46B7
:1003B00003221C1C0B37B3469443162F00D976E05A
:1003C000102001901027B94500D975E0019A944298
:1003D00056DAC548321980680390904200D1C3E0D4
:1003E0005168081C8A46012188438446944461462A
:1003F00048680121084264D000200022D90700D5B6
:1004000086E033680321F31A8C4659689A4663469E
:1004100099438C46002A00D1DFE003998A4200D13B
:10042000DEE061460B190199C018039088426ADB2F
:10043000D3689268D3609A605246D36892685646F1
:10044000D3609A60221F0836242A00D9BBE0331CEF
:10045000132A0AD92B68504683606968C1601B2A39
:1004600000D905E15346103308352A6851461A6011
:100470006868039C5860AD68D3469D604B68351C26
:10048000E21B0F2A2CD80122134023435846436015
:100490005C4461680A4362604046FEF7A1FA281C8A
:1004A00005B03CBC90469946A246AB46F0BD07223B
:1004B0009743019700D486E70C2341460B60002048
:1004C000EEE7032051468143081C09198C46019927
:1004D0008C4593DBD16892686446D1608A60CFE72F
:1004E0005846C119012003401F435B465F60131C3F
:1004F00003438A184B6053680831184350604046E4
:10050000FFF72AFEC8E7039303980199884293DA1C
:1005100049464046FDF79AFF8146002800D1D5E0C4
:100520007368021C0121181C8843083A3618B2422D
:1005300000D198E0221F242A40D8132A22D84B4603
:100540002A1C106818605168596092689A60404689
:10055000291CFFF701FE4046FEF742FA48469FE796
:10056000111CFDF773FF9BE7039A526802920298F1
:10057000032290433A1C011910328C4691420CDA46
:10058000039A3BE729684B461960686858601B2A44
:100590005ED82A1C08330832D3E7534BF219604661
:1005A0009A60C11B012319435160716840460B409A
:1005B0001F437760FEF714FA281C71E74846291C90
:1005C000FFF792FEC3E7291C301CFFF78DFE524651
:1005D0005368351C039CD34652E70B19039393E7EA
:1005E000624613193A1CC0181032039090428ADBFD
:1005F00050468268C3685646D3609A60221F083608
:10060000242A53D8331C132A08D9296881606B68BF
:10061000C3601B2A4FD8534610330835286818602A
:1006200069685960AD689D605346DA19039B2E488E
:10063000D91B0123194382605160504640685146DE
:1006400003401F4340464F60FEF7CAF9301C27E7BE
:10065000A9684B469960E868D860242A13D02A1C00
:10066000103310326DE7526803218A43A41807E75C
:10067000AB6850460361E9684161242A0DD05346B6
:1006800018331035F1E629692A1C196168694B464F
:10069000494618331832486153E72A695346826144
:1006A000686951462033C8611835DEE6301C291CC4
:1006B000FFF71AFEB8E7A86851460861EB684B617E
:1006C000242A08D0534618331035A7E74046FEF7D2
:1006D00087F90020E4E62869514688616A69534633
:1006E0002033CA61183599E7B824002038B50C1CAE
:1006F0000968051C002901D0FFF7F8FF281C211C00
:10070000FFF72AFD38BDC046264B70B51B68051E95
:100710009D423AD0C26C002A16D0002300269B00CE
:100720009958002901D107E0211C0C68281CFFF70B
:1007300013FD002CF8D1EA6C0136331E202BEED1CC
:10074000281C111CFFF708FD296C002902D0281C69
:10075000FFF702FDA4235B00E95800290CD0A62373
:100760005B00EE18B14201D106E0211C0C68281C88
:10077000FFF7F2FCA642F8D1696D002902D0281CCF
:10078000FFF7EAFCAB6B002B00D170BDEB6B281CB4
:100790009847B8239B00E9580029F6D0281CFFF79A
:1007A000A5FFF2E738240020002934D001230022DD
:1007B00010B488422CD301242407A14204D28142E0
:1007C00002D209011B01F8E7E400A14204D28142F0
:1007D00002D249005B00F8E7884201D3401A1A436D
:1007E0004C08A04202D3001B5C0822438C08A042A4
:1007F00002D3001B9C082243CC08A04202D3001B5A
:10080000DC082243002803D01B0901D00909E3E7D3
:10081000101C10BC7047002801D00020C04307B452
:10082000024802A14018029003BDC046D900000052
:100830000029F0D003B5FFF7B9FF0EBC4243891A77
:100840001847C046002941D010B4041C4C40A446AF
:1008500001230022002900D54942002800D540424A
:1008600088422CD301242407A14204D2814202D21F
:1008700009011B01F8E7E400A14204D2814202D23F
:1008800049005B00F8E7884201D3401A1A434C083C
:10089000A04202D3001B5C0822438C08A04202D372
:1008A000001B9C082243CC08A04202D3001BDC089A
:1008B0002243002803D01B0901D00909E3E7101CDB
:1008C0006446002C00D5404210BC7047002806D07A
:1008D00003DB0020C043400801E08020000607B48D
:1008E000024802A14018029003BDC0461900000052
:1008F0000029EBD003B5FFF7A7FF0EBC4243891ACE
:100900001847C0467047C0468446101C62468C4655
:10091000191C634600E0C0461FB500F091FF002897
:1009200001D40021C8421FBD10B500F0C1FE4042F5
:10093000013010BD10B500F083FF002801DB00205E
:1009400010BD012010BDC04610B500F079FF002891
:1009500001DD002010BD012010BDC04610B500F023
:10096000F1FE002801DC002010BD012010BDC046B2
:1009700010B500F0E7FE002801DA002010BD0120CC
:1009800010BDC046002B11D1002A0FD1002900D183
:10099000002802D00021C943081C07B4024802A164
:1009A0004018029003BDC0465DFFFFFF03B46846D8
:1009B00001B5029800F022F8019B9E4602B00CBCE3
:1009C0007047C046F0B583B0161C1F1C0090019103
:1009D00001F054FE041C0D1C221C2B1C301C391C65
:1009E00001F02AFE009A019B121A8B410899201CE3
:1009F0000A604B60291C03B0F0BDC046F0B583B05F
:100A0000141C1D1C0090019102F014F8221C2B1CD8
:100A1000061C0F1C01F010FE009A019B121A8B415C
:100A20000899301C0A604B60391C03B0F0BDC04609
:100A3000F8B55F46564644464D46F0B40C034D00AB
:100A4000CE0F610A440F2143C400180380465800AA
:100A5000400D8246D80F84464046400A530F034358
:100A6000D0006D0D371C83465246664500D19DE08F
:100A7000AF1A002F00DC03E1002A38D1184300D060
:100A8000E4E0630709D00F232340042B05D0231D86
:100A9000A342A441644209191C1C080200D478E056
:100AA000CE4B6A1C9A4200D105E1CD4BE4081940B7
:100AB00048075205490204430B0B520D371C002016
:100AC00000211B03201C1C0B0B0D1B05C54D2343D4
:100AD000520552081D4015436D006D08FF07291C83
:100AE00039433CBC90469946A246AB46F8BDBB484C
:100AF0008542C6D0802000040343382F00DDECE09F
:100B00001F2F00DD20E12020C01B1A1C81468240DF
:100B10005846F8400243944658464A469040421E82
:100B20009041FB40624602431F1CA21A9442A4411A
:100B30006442C91B091B141C0B02A2D549024F0AAF
:100B4000002F00D1C4E0381C01F058FD021C083A07
:100B50001F2A00DDB7E02821091A201C9740C84051
:100B600007439440954200DDA9E0551B691C1F29ED
:100B700000DDD8E01F22551B3B1C221CAB40CA40A5
:100B8000AC40651EAC411343CF401C43391C0025CB
:100B900077E74807E4086A05C908520D371C044383
:100BA0008E4B9D4248D009030B0B88E7AA1A944646
:100BB000002A00DC98E05046002853D08748854240
:100BC00000D15EE78020000403436246382A00DD3E
:100BD000FDE01F2A00DD4BE120226046101A1A1C9E
:100BE00082408246914658466246D0404A46024379
:100BF0009046584652469040421E9041424602431B
:100C00006046C3401219A242A4416442591809190E
:100C1000141C080200D434E7704B01359D4200D10A
:100C200024E16F4B60081940012323401C1C04433E
:100C3000CB071C43490824E70B1C234300D1C7E121
:100C400080231B030B431B031B0B38E7013F002FC3
:100C500064D15846221A9442A4416442C91A091B1D
:100C6000141C69E75846184300D10AE70122524292
:100C700094446046002800D0C5E058460219C2E7F7
:100C8000002F72D1681C4005400D012800DCDEE019
:100C90005A46A21A9442BF41C81A7F42C71B380263
:100CA00000D488E05A46141BA3459241591A524277
:100CB0008F1A664644E7371C00230024FFE64849A4
:100CC000AD1A3940DDE6271C28388740002449E763
:100CD000201C01F093FC203038E75A461A43531E7B
:100CE0009A41D2B2002720E7002A00D0DDE0681C3C
:100CF0004205520D012A00DC8EE0384DA84200D199
:100D0000B3E05D462A19A242A44164425918091968
:100D1000CC07520814434908051CB2E62F48854207
:100D200000D0EAE6ADE62B1C1F3B3A1CDA40131C50
:100D300020296DD03F22551BAF403C43601E8441AB
:100D40001C43002100259CE6381C20381A1CC24098
:100D5000101C202F5ED04022D71BBB405A461A439E
:100D6000531E9A4102430027DFE6002D3CD01B4D65
:100D7000AA4500D194E080252D047F422943382FD5
:100D800000DDADE01F2F00DD2CE12025ED1B081C50
:100D9000261CA840FE40AC400643651EAC413443CF
:100DA000F9405D462C1BA34592415B1A5242991AA9
:100DB00055466646C0E6131C3B43141C002B00D06E
:100DC000BEE600270022002500210024E8E65A465E
:100DD0001A43531E9A41D2B2002313E7FF070000C3
:100DE000FFFF7FFFFFFF0F800D1C254358D0FF43FF
:100DF000002F51D1041BA3459241591A5242891A1E
:100E00005546664698E69648854200D0DDE638E6C7
:100E1000002792E70023A1E7081C2043002D00D003
:100E2000C0E0002800D1FBE05846184300D128E676
:100E300058460219A242A441644259180919141CC7
:100E40000A0200D41DE6874B0125194019E6081C4B
:100E50002043002D39D100286DD15946194300D1C6
:100E6000BDE0191C5C4666460BE6051C2A1CABE778
:100E7000604620381A1CC24060469146202800D1A6
:100E8000ABE04022121A93405A461A43531E9A412D
:100E90004B461A430023B5E6714DAA4500D06EE7D4
:100EA000191C5C4655466646EBE5002D1ED10D1C0F
:100EB000254373D0D543002D6DD15C445C459241F0
:100EC0005918524289185546A3E6002849D1594677
:100ED000194300D196E0191C5C466646604DD0E58A
:100EE0000C43611E8C41E4B200215AE75C4DAA45D7
:100EF00054D05542802210040143382D00DD85E096
:100F00001F2D00DD95E02022501B0A1C84468240E4
:100F1000201CE8400243904662469440601E844193
:100F200042461443E9405C445C459241CB1852422E
:100F3000991855466DE65846184300D1A1E5584624
:100F4000271ABC429241C81A5242801A02026AD53C
:100F50005846041BA3459241591A5242891A6646C3
:100F60008FE55846184336D04807E40804438020EC
:100F7000C9080003014208D0DD08054205D15946E1
:100F8000CA085C071443291C6646630FC90019434D
:100F9000E400334D75E5324A9245AED1191C5C46EA
:100FA00055466EE5002837D05846184313D08025A3
:100FB0004807E408C9082D0304432942E5D0D808AE
:100FC0002842E2D15D46EA085C071443011CDCE7D5
:100FD0000023002473E5224D53E5002354E7002746
:100FE0000022F1E63D1C203D0A1CEA40151C202F82
:100FF00031D04026F71BB9400C43611E8C412C4375
:101000000021CEE6164A0027151CDDE60C43611EC2
:101010008C41E4B2002186E7191C5C46104D30E596
:10102000191C5C462DE5031C3B43D8D0011C3C1C1D
:1010300027E52020404240190A1CC2409046202D3E
:101040000BD04020451BA9400C43611E8C414546F6
:101050002C43002167E70021CEE70021F4E7C046DA
:10106000FF070000FFFF7FFFF0B5564644465F468E
:101070004D46F0B41F1C0B031B0B98464B0087B06A
:10108000041C81465B0DC80F161C9A460090002B6D
:1010900051D06A4B9A4531D08022414652030A43CF
:1010A000630FD2001A43664B90460025E20091463A
:1010B0009A44002402953B031B0B9B46FD0F7B00CB
:1010C000311C5B0D019560D05C4A934254D0802165
:1010D000584649030143720FC9001143584A8B46D1
:1010E0009B18F1000020009A04436A4003920F2CE1
:1010F00000D9ADE0534EA4003459A74640460443FE
:101100006ED1002102250824884689460295D2E73F
:10111000009C0298C34649460194022864D00328E3
:1011200000D1ABE2012800D038E2019A002402404D
:101130000025A14660E0434623434AD040460028AC
:1011400000D1C0E101F05AFA031E272B00DDB3E104
:1011500028210D1A211C083B4246E9409A400D1CEB
:101160001543221C9A40A8469146374B00251B1A6E
:101170009A46002402959EE75A4616430320002E05
:10118000B1D1B34600210220ADE75A4632431BD00D
:101190005B46002B00D18AE1584601F02FFA272840
:1011A00000DD7DE12822171A011C321C08395B463C
:1011B000FA408B40171C1F43331C8B40BB46191C45
:1011C000214B1B1A00208EE70027BB46002101207F
:1011D00089E70020012504248046814602956AE7BC
:1011E00003250C24029566E7019C0394039D0122CC
:1011F0002A400024114DA146002000212403260B83
:101200000C0D2405114B34432D0523402B435B006B
:101210005B08D207191C4846114307B03CBC9046F6
:101220009946A246AB46F0BD002280242403914695
:10123000024DE1E700240025A146DDE7FF0700009D
:1012400001FCFFFFF43302000DFCFFFFFFFF0F80E6
:101250005546ED1A0495D84500D953E100D14EE129
:10126000049C0025013C4E4604944746A946584636
:1012700003020C0E1C430902250C23041B0C0091D5
:10128000381C291C0193FFF78FFA019983464143CB
:10129000381C8A46291CFFF7CBFA330C0904194382
:1012A0008A450CD95B460919013B8C4200D947E1BC
:1012B0008A4500D844E10222524293440919534618
:1012C000CB1A181C291C9846FFF76EFA071C0198C8
:1012D000291C784382464046FFF7AAFA36040B04DD
:1012E000360C33439A4509D91B197A1E9C4200D902
:1012F00024E19A4500D821E1023F1B195E463204E1
:101300001743380CBB46009E009F51463F0C3204E9
:101310005B1A5946BA46120C0F043F0C90465146D0
:101320007A434F434146414356467043CF19160C0A
:10133000BE19B14202D980277F02C019310C1204B4
:101340003604120C4018B618834200D2C4E000D113
:10135000BEE0191A4846861BB145BF417F42CF1BEC
:10136000A74200D113E1291C381CFFF71DFA01998F
:1013700002904143381C8946291CFFF759FA330C67
:101380000904194389450CD9029B0919013B8C4278
:1013900000D9FFE0894500D8FCE0029F0919023F0F
:1013A00002974F46CF1B381C291C0597FFF7FCF905
:1013B000071C0198291C784381460598FFF738FAE5
:1013C00036040904360C0E43B14509D936197B1E83
:1013D000B44200D9E0E0B14500D8DDE0023F361963
:1013E000029D4946761A290439430B0457460A0CD4
:1013F0001B0C40464546584355437B437A43EB1804
:10140000070CDB199D4202D980256D0252191D0C73
:1014100000041B04000C52191B18964235D300D14E
:10142000FCE001231943049E994FF519002D00DCBF
:10143000A1E0480709D00F230B40042B05D00B1D5A
:101440008B42894149428B44191C5A46D20107D527
:10145000904B5C46049E80271C40FF00A346F51974
:101460008D4B9D427ADD039C0122224000248B4D4E
:10147000A146C1E680242403474627424CD13C4381
:101480002403240B009A854DB6E63619481EB44253
:101490005ED9011C9642C4D1009E9E42C1D1C2E7D2
:1014A000031C283B311C99408B46002188E6301CE8
:1014B00001F0A4F8203072E6283B211C994000225C
:1014C0008846914651E6201C01F098F820303BE612
:1014D0000021B14500D33DE7009F5A46B944B945C4
:1014E000BF417F423F19FB18013A9C421ED29842ED
:1014F00000D97EE000D1B5E0191A93462AE7894564
:1015000000D8ADE64846464642467708D307460827
:10151000C0071E438146AAE65846204212D1044322
:1015200024032A1C240B89465C4D65E6A342E3D1C3
:10153000009F4F45DBD9211A93460BE7171CDDE6C8
:101540009B46BCE63C432403240B009A534D53E6D0
:10155000B24259D800D18AE0011C62E75F46C9084F
:101560007B07039E0B437C026D0501229946240BE9
:101570006D0D324040E64A4B049FDB1B382B10DDDB
:10158000039C0122224000240025A14634E60121CB
:10159000494248E7029304E71F1C21E7019C03949A
:1015A00041E71F2B40DC3F48049F0C1C3A1858466B
:1015B0009140DC40904020430A1C511E8A41011C8E
:1015C00011435A46DA40131C480709D00F220A403B
:1015D000042A05D00A1D8A42894149425B18111C20
:1015E0001A0234D5039C0122224000240125A14681
:1015F00002E6009F02214942B9448B44B945894122
:1016000049420919CB18A4E6009D881E6900A94229
:10161000AD416D422C19361900913AE7002B00D0EC
:1016200033E70024009437E71F4A049C5D46121BF1
:10163000D5402A1C202B1FD01C4E5F46A3199F406B
:101640003B1C19434B1E994111430023BCE75A0729
:10165000C9080A43039F91465B0201221C0B3A40D2
:101660000025C9E54E45C4D89346002172E6009F87
:101670009F42C9D3011C0FE70023E2E78024240323
:101680005F463C432403240B019A8946034DB3E58E
:10169000FF030000FFFFFFFEFE070000FF07000042
:1016A00002FCFFFF1E040000E2FBFFFF3E040000FF
:1016B000F0B55F4656464D464446F0B40D1C041C3A
:1016C0008046E80F814618030F03000B3F0B83B0E1
:1016D00084461B48009749005E00DF0F490D924683
:1016E000760DBB4681420CD01548864210D00120B1
:1016F000B14215D003B03CBC90469946A246AB46D9
:10170000F0BD009F01202743F4D10D488642EED161
:10171000604602430120002AECD10120B142E9D108
:10172000009B6345E6D1D045E4D1D94506D00029D8
:10173000E0D11C43201C441EA041DBE70020D9E778
:10174000FF070000F0B55F4656464D464446F0B4EC
:10175000CD0FDE0FAC461D032D0BB146374E0F03E8
:101760004C00AB465D0080463F0B640D92466D0D0C
:10177000B44232D0314EB54235D0002C0ED1384370
:1017800041424141081C002D0BD0002919D1CC4504
:101790002DD0654668420123184318E0002DF6D18C
:1017A000281C59460A4353425341002806D1002BB6
:1017B000EDD0634658420123184308E00020002B77
:1017C00005D14A46504250414042012318433CBC97
:1017D00090469946A246AB46F0BD3E1C0643C9D092
:1017E00002204042F3E75E461643C6D0F8E7AC421B
:1017F00007DC0BDA61464842484140420123184366
:10180000E5E76646704201231843E0E75F450AD8E2
:101810000ED000205F45DAD26546684268414042FA
:1018200001231843D3E76246504201231843CEE711
:10183000D045F8D80020D045EED3C8E7FF07000018
:10184000F0B556464D4644465F46F0B40D1C83B095
:10185000041C0190E80F814618030F03000B3F0B97
:1018600084463548009749005E00DF0F490D9246D7
:10187000760DB846814234D02F48864236D00029B2
:1018800018D0002E1FD1341C67463A4353425341AF
:10189000002C1FD00020002B05D142465042504161
:1018A00040420123184303B03CBC90469946A246EF
:1018B000AB46F0BD0098044360426041041C002E1A
:1018C000E2D00028E9D1C14515D04F467842012326
:1018D0001843E8E7002BF6D04B4658420123184343
:1018E000E1E7009F02202743DDD1C5E767460220DC
:1018F0001743D8D1C3E7B14204DD4A465042012321
:101900001843D0E7B14207DB00986045E4D80AD01D
:10191000009F00206745C6D24F467842784140423A
:1019200001231843BFE7019A5245D5D8019A0020F8
:101930005245F1D3B7E7C046FF070000F0B5564661
:1019400044465F464D46F0B41F1C0B031B0B9A46E2
:101950004B0087B0041C80465B0DC80F161C029319
:101960008146002B68D0694B0299994232D080227F
:10197000534652031A43D200630F1A439246644AF5
:10198000E000891880460291002400253B031B0BD0
:101990009B467800FB0F321C400D039300D175E08D
:1019A0005A4B984269D08022594652030A43730F1A
:1019B000D2001A43564B9346C018F20000230399F5
:1019C0004E4671401C430F2C00D9A9E0514EA40093
:1019D0003459A74653461C4300D087E00025AA4649
:1019E000A84608240225D1E74946022D6CD0032DD4
:1019F00000D117E2012D00D058E10D40EDB20024D6
:101A0000A9460023A0460020002125030A0D1C053D
:101A10002D0B1205404B2A43134023435B004C46D9
:101A20005B08E207191C4046114307B03CBC9046D6
:101A30009946A246AB46F0BD5346234350D0534689
:101A4000002B00D184E1504600F0D8FD031E272B67
:101A500000DD76E128210D1A211C083B5246E940A1
:101A60009A400D1C1543221C9A40AA4690462B4BC7
:101A700000241B1A0293002588E75B461E430323BC
:101A8000002E9CD1B3460022022398E75B463343E5
:101A900021D05846002800D14EE100F0AFFD2728A4
:101AA00000DD42E128210F1A021C311C083A5B4676
:101AB000F94093400F1C1F43331C9340BB461A1C34
:101AC000164B181A00237AE701230B40002499468D
:101AD000A0460E4B97E70027BB46002201236EE786
:101AE000002104248A46884601254FE70C2403255B
:101AF0004CE700258024A9462403A846034B82E72F
:101B0000DA46904603991D1C6FE7C046FF070000A8
:101B100001FCFFFF34340200FFFF0F800DFCFFFFCC
:101B2000029F160C381804904046070C0004000C65
:101B30001204120C031C5343041C3D1C74435543F4
:101B400098463B1C73436419A44644460293230CF5
:101B500063449D4204D9029D802464022D1902959C
:101B60001D0C039545462C041B04240C1C190594DC
:101B70005C46230C051C58432404240C8446381C62
:101B8000604365435F438146CC44280C6044BB46B8
:101B9000814502D980277F02BB442D04070C2D0C00
:101BA000000440195546BC462F04E3448446280CE3
:101BB0003D0C2F1C5743B8462F1C77434243B94670
:101BC00047463F0C9144BA46D14446434A4502D960
:101BD00080225202B6184F463A0CB6183A044746CD
:101BE0003F043F0CB8462F1C67435D4344435843B2
:101BF00065190190380C2D184244B846AC4204D9FE
:101C0000019880235B02C0180190039C029F201C56
:101C10006044C0196045A44147466442A4462B0471
:101C20003C049946240C4C44A046D8448018C24633
:101C3000E24490429241574652429146F219E2459F
:101C4000BF417F424B46BC46D845BF41D4187F4276
:101C500063461F432D0C7F19B24292414C45AD4162
:101C600052426D421543019E7D19AB19E20D5B0294
:101C7000059F134342023A439A46531E9A41C30DAD
:101C8000101C18436402204380465046C0010DD505
:101C9000454601225646049C6B082A401A43F30726
:101CA00001341A43760804949046B246049E634F6A
:101CB000F319002B61DD404640070BD00F2244464C
:101CC0002240042A06D04246043242458041404226
:101CD000824490465546ED0107D5594B5646049F20
:101CE00080201E40C000B2463B18564A934200DD99
:101CF000EAE644465546E2086807104301226C02B2
:101D00005B050A408046240B5B0D91467BE6DA4674
:101D100090461D1C69E680242403574627421CD1A7
:101D20003C432403240B484B6DE6031C283B311C29
:101D300099408B460022C3E6301C00F05FFC203047
:101D4000ADE6283B211C994000228A4690468EE64B
:101D5000201C00F053FC203078E65846204207D182
:101D6000044303992403240B89469046364B4AE6E4
:101D70003C432403240B344B45E6344B049E9B1B0D
:101D8000382B06DD01230B4000249946A046002392
:101D900039E61F2B25DC049C2D4D46466019524622
:101DA00044468640DC4082405746301C2243DF4098
:101DB000441EA04102433B1C540709D00F20104091
:101DC000042805D0101D9042924152429B18021CDB
:101DD0001D021AD501230B4000249946A046012379
:101DE00011E61C48049C5546001BC540281C202BAE
:101DF00016D0194E5746A21997403A1C43461A432B
:101E0000531E9A4102430023D6E758075B02D208CB
:101E10001C0B01230B401043994680460023F2E53A
:101E20000022EBE780242403504601230443194099
:101E30002403240B8946044BE5E5C046FF0300005C
:101E4000FFFFFFFEFE070000FF07000002FCFFFF90
:101E50001E040000E2FBFFFF3E040000F8B55F46F1
:101E6000564644464D46F0B40C034D00CF0F610A70
:101E7000440F2143C4001803DE0F8046B446464693
:101E80005800760A530F3343D600C94A6D0DBA463F
:101E9000400DB346904200D1EBE06246012672400D
:101EA0009446674500D1A1E02F1A002F00DC08E11D
:101EB00000283BD15846184300D0E8E0600709D01D
:101EC0000F232340042B05D0231DA342A4416442C9
:101ED00009191C1C0A0200D479E0B54B6A1C9A420D
:101EE00000D109E1B34BE408194048070443490213
:101EF0005205012750460B0B520D074000200021D0
:101F00001B03201C1C0B0B0D1B05AB4D2343520563
:101F100052081D4015436D006D08FF07291C394309
:101F20003CBC90469946A246AB46F8BDA0488542C7
:101F3000C4D0802000040343382F00DDF0E01F2FC1
:101F400000DD24E12020C01B1A1C5E468240FE40BA
:101F5000324394465A468240101C421E9041FB4038
:101F6000624602431F1CA21A9442A4416442C91B48
:101F7000091B141C0A02A1D549024F0A002F00D1E7
:101F8000C9E0381C00F03AFB021C083A1F2A00DDA9
:101F9000BCE02821231C091A9740CB401F439440E2
:101FA000954200DDAEE0551B691C1F2900DDDDE018
:101FB0001F22551B3B1C221CAB40CA40AC40651E77
:101FC000AC411343CF401C43391C002576E748073A
:101FD000E4086A0501275646C908520D37400443F4
:101FE000734B9D4249D009030B0B87E72A1A94468D
:101FF000002A00DC9BE0002855D06D48854200D1C6
:102000005CE78020000403436046382800DD09E1D6
:102010001F2800DD50E162462020801A1E1C8640E9
:10202000B1465E46D6404A4632435E4686409046BA
:10203000301C421E9041424602436046C340121982
:10204000A242A441644259180919141C080200D480
:1020500034E7574B01359D4200D142E1554B6008B2
:102060001940012323401C1C0443CB071C4349088F
:1020700024E71E4300D014E70FE70B1C234300D1D5
:10208000CFE180231B030B431B031B0B36E7013FF0
:10209000002F66D15E46A21B9442A4416442C91A35
:1020A000091B141C66E75846184300D106E70126B1
:1020B0007642B4446046002800D0CAE05E46321939
:1020C000BEE7002F7AD1681C4005400D012800DCD6
:1020D000E3E05A46A21A9442BF41C81A7F42C71B86
:1020E0003E0200D492E05846041BA3459241591A7F
:1020F00052428F1AE24641E7534601271F4000240F
:102100000023FBE62B49AD1A3940D7E6271C2838B7
:102110008740002444E7201C00F070FA203033E7A9
:102120005A461A43531E9A41D2B200271BE7002A8F
:1021300000D0E1E0681C4605760D012E00DC91E040
:102140001B4DA84200D1F7E05E463219A242A441DD
:10215000644259180919CC07520814434908051C50
:10216000ACE61348854200D0E6E6A7E62B1C1F3BF1
:102170003E1CDE40331C202970D03F22551BAF404F
:102180003C43601E84411C430021002596E6381C18
:1021900020381E1CC640301C202F61D04022D71B87
:1021A000BB405A461A43531E9A4102430027DAE6BF
:1021B000FF070000FFFF7FFFFFFF0F80002D38D0DB
:1021C000B94DA84200D192E080252D047F422943D9
:1021D000382F00DDAAE01F2F00DD2CE12025ED1BAC
:1021E0000E1CAE40B046261CFE404246AC40164394
:1021F000651EAC413443F9405A46141BA345924135
:102200005B1A5242991A051CE246B3E6131C3B4383
:10221000141C002B00D0B1E600270022002500216D
:102220000024DDE65A461A43531E9A41D2B20023D7
:1022300005E70D1C25435AD0FF43002F53D15A46C2
:10224000141BA3459241591A5242891A051CE246B1
:1022500090E69548854200D0D6E62FE600278FE726
:1022600000239EE7081C2043002D00D0C3E0002877
:1022700000D1F6E05846184300D11FE6584602192F
:10228000A242A441644259180919141C0A0200D43C
:1022900014E6864B0125194010E6081C2043002D4A
:1022A0003AD1002800D089E05946194300D1BFE057
:1022B000191C5C46E24601E6604620381A1CC24002
:1022C0006646101C202E00D1B0E04022921B9340A5
:1022D0005A461A43531E9A4102430023AFE6724DF9
:1022E00000272A1C9BE7704DA84200D070E7191CFC
:1022F0005C46051CE246E1E5002D20D10D1C25437E
:1023000075D0D543002D6FD15C445C45924159187E
:1023100052428918051C99E6002835D159461943BF
:10232000DDD0191C5C46E2465F4DC7E50C43611EDB
:102330008C41E4B200215FE7051C021C6FE75A4D97
:10234000A84254D05542802216043143382D00DD76
:1023500081E01F2D00DD91E02022561B0A1CB446AF
:10236000B240261CEE403243904662469440661EC0
:10237000B44142461443E9405C445C459241CB1869
:1023800052429918051C61E6584618434CD048073C
:10239000E40804438020C9080003014208D0DD0896
:1023A000054205D15946CA085C071443291CE24678
:1023B000630FC9001943E4003B4D7FE558461843BD
:1023C00000D17BE55E46A71BBC429241C81A52422F
:1023D000801A06024CD55846041BA3459241591A4F
:1023E0005242891AE24669E52F4A9042AED1191C41
:1023F0005C46051C62E5002836D05846184313D0C9
:1024000080254807E408C9082D0304432942CFD09A
:10241000D8082842CCD15D46EA085C071443011C69
:10242000C6E70023002469E51F4D47E500234FE779
:1024300000270022F3E63D1C203D0E1CEE40351C1B
:10244000202F2DD04026F71BB9400C43611E8C4134
:102450002C430021D0E60C43611E8C41E4B20021E4
:102460008AE7191C5C4629E5191C5C460E4D25E5DA
:10247000031C3B43DCD0011C3C1C1FE5202676429C
:1024800076190A1CF2409046202D0BD04026751B71
:10249000A9400C43611E8C4145462C4300216BE74B
:1024A0000021D2E70021F4E7FF070000FFFF7FFFD4
:1024B00070B50B1C124C09030E0B5900021C490D80
:1024C000DD0F0020A14211DD0E4881420FDC80208B
:1024D000400306430C48401A1F280BDD0B4A521AD2
:1024E000D640321C5042002D00D1101C70BD084B4C
:1024F000E818FBE7074BC240C9188E403243F1E7AA
:10250000FE0300001D04000033040000130400005B
:10251000FFFFFF7FEDFBFFFFF8B5041E31D0C70FB3
:1025200000D04442201C00F069F8184D2D1A0A28EA
:1025300019DD0B38844024036D05240B6D0D3A1C06
:102540000026002000210B0D2403240B1B05234330
:102550000F4C2D051C402C4364006408D307211C3C
:10256000301C1943F8BD061C1536231CB3401E1C35
:102570000B23181AC44024036D05240B6D0D3A1C5F
:10258000DFE70022002500240026DAE71E04000011
:10259000FFFF0F8010B5041E28D000F02FF8154A59
:1025A000121A0A2815DD0B38844024035205240B27
:1025B000520D0023002000212403181C0B0D240BB6
:1025C0001B0523430C4C12051C4014436400610896
:1025D00010BD031C1533211C99400B1C0B21081A3C
:1025E000C44024035205240B520DE3E700220024CB
:1025F0000023DFE71E040000FFFF0F801C210123E2
:102600001B04984201D3000C10391B0A984201D3D5
:10261000000A08391B09984201D30009043902A2B3
:10262000105C40187047C04604030202010101011A
:1026300000000000000000009C460304F0B51B0CE5
:1026400017043F0C150C1E1C041C000C7E436B432E
:1026500047434543FB18300C1818874202D98023A2
:102660005B02ED18030CED1863465C434A433604E5
:10267000360CA118000480194919F0BDF0B5444684
:102680005F4656464D46F0B41C1C85B0002900DA62
:10269000DBE00F1C0021061C8A46101C191C002CB4
:1026A00000DAC9E00196009089468046002951D1A0
:1026B000B84200D871E0FFF7A1FF002809D020231D
:1026C0004546311C1B1A85408740D940A8460F4318
:1026D00086404246150C13041B0C291C381C9B46D3
:1026E000FEF762F85B464343041C291C381C9946DC
:1026F000FEF79EF8330C08041843814509D940447D
:10270000631E804500D978E1814500D875E1023C1F
:1027100040444946411A8946081C291CFEF744F8E2
:102720005A464243071C291C48469346FEF780F848
:1027300036040904360C0E43B34507D946447B1EC4
:10274000B04502D8023FB34500D81F1C24042743DC
:10275000002403E0B94211D9002400275246381C56
:10276000211C002A03D03B1C00215842A14105B086
:102770003CBC90469946A246AB46F0BD081CFFF70C
:102780003DFF041E00D0BFE0B94500D242E1019DEB
:102790000099071C8D424741E0E7002804D1012041
:1027A0000021FEF701F880464046FFF727FF00288A
:1027B00052D1414644460B043C1B1B0CA3460D0C56
:1027C00000930124291C5846FDF7EEFF009F814627
:1027D0004743291C5846FEF72BF8330C09041943CC
:1027E0008F4208D94B464144013B884502D88F426D
:1027F00000D91AE19946C91B8B46081C291CFDF714
:10280000D3FF009B291C4343071C58460093FEF747
:102810000FF83604009D0904360C0E43B54207D963
:1028200046447B1EB04502D8023FB54200D81F1C6B
:1028300049460E04374391E75246D243031C0C1C11
:10284000924600215842A1412CE7002746428F4181
:10285000012149428A4620E720231B1A4246351CA3
:1028600082403C1CDD40DC4087402B1C150C3B4368
:10287000291C8640201C009317049046FDF794FF06
:102880003F0C011C794381468B46201C291CFDF717
:10289000CFFF009C0904230C19438B450CD94B46F0
:1028A0004144013B884500D9BDE08B4500D8BAE0E2
:1028B00002225242914441445C460C1B201C291CBC
:1028C0000194FDF771FF391C4143041C8B460198AC
:1028D000291CFDF7ADFF009A090413041B0C1943D2
:1028E0008B4509D94144631E884500D997E08B4543
:1028F00000D894E0023C41445B46CB1A49469B46D3
:102900000B041C4300975DE7009D20231B1A4A46D9
:102910008240DD401543391C009AD94082408846E8
:10292000311C0092D9403A1C82400B1C1343019386
:102930002F0C2B041B0C391C40460293FDF734FF6F
:10294000029A81464243391C40469346FDF770FF88
:10295000019A0904130C19438B450AD94B464919AE
:10296000013B8D425DD88B455BD902235B42994484
:1029700049195A468A1A101C391C0392FDF714FF94
:10298000029B80464343391C03989B46FDF750FF4A
:10299000019A090413041B0C19438B450AD94346B9
:1029A0004919013B8D4238D88B4536D902235B4209
:1029B000984449195D464D1BAB464946009D0F049E
:1029C000424617432A04120C3B042D0C1B0C380CF6
:1029D000111C594342436B436843D3180D0C5B19D8
:1029E0008C469A4202D98022520280181D0C40194E
:1029F00083450CD303D00024B0E61C1C89E6654651
:102A00002A041B04120C9B18A6409E42F3D2013FDD
:102A10000024A3E600240127A0E69846CAE71C1C70
:102A20006AE79946A5E7994646E702225242914451
:102A30004144E0E6F0B55F4656464D464446F0B4A4
:102A40000D1C85B0061C9246984602900191039297
:102A50001F1C141C8346A946002B59D1AA4269D9D0
:102A6000101CFFF7CBFD00280AD020231B1A311CB5
:102A7000D94085400B1C2B43864084409946B34681
:102A8000250C23041B0C291C48469846FDF78CFE98
:102A90004646071C4643291C4846FDF7C9FE5A46D0
:102AA0000904130C19438E4209D909197B1E8C4263
:102AB00000D957E18E4200D854E1023F0919891B21
:102AC0008946081C291CFDF76FFE43464343061C3C
:102AD000291C48469846FDF7ABFE5A4613040904E4
:102AE0001B0C1943884508D90919731E8C4200D95B
:102AF00036E1023E884500D832E1380430430027F1
:102B0000391C05B03CBC90469946A246AB46F0BD88
:102B1000019A934262D8181CFFF770FD041E60D121
:102B2000019B9F4200D22CE1029F03998F4260419A
:102B30000027E5E7002A04D101200021FDF734FE3B
:102B4000041C201CFFF75AFD002800D0B9E0230424
:102B50002D1B1B0CA946260C98460127311C484604
:102B6000FDF722FE41464143051C8A464846311C7A
:102B7000FDF75EFE5A460804130C1843824507D938
:102B800000196B1E844202D8824500D910E11D1C39
:102B90005346C31A181C311C9A46FDF705FE4146E0
:102BA0004143814688465046311CFDF741FE5A4656
:102BB000130409041B0C194388450BD94B4609190A
:102BC000013B8C4200D9CFE0884500D8CCE00223FD
:102BD0005B42994428044946084391E700270020B6
:102BE0008EE720231B1A424657468240DF40174398
:102BF000524682400192321CDA40291CD94085405D
:102C0000131C2B4302933D0C3B041B0C8846081CF1
:102C1000291C9A46FDF7C8FD534643438146291CAB
:102C200040469B46FDF704FE029A0904130C194323
:102C30008B4506D94B46C919013B8F4200D8ABE002
:102C400099465A468A1A101C291C9346FDF7ACFD7A
:102C500053464343291C804658469A46FDF7E8FDF3
:102C6000029A090415042D0C29438A4506D94346C6
:102C7000C919013B8F4200D886E098465746CF1BC2
:102C8000BA464946019F0804424610433D042D0CB4
:102C900003043F0C1B0C020C291C594355437B4376
:102CA0007A43EB180F0CDB198C469D4202D9802722
:102CB0007F02D2191D0C521992455FD356D00027BE
:102CC0001EE720231B1A311C2F1CD940DF408540F2
:102CD0000B1C84402B4386400193B3462304260CEF
:102CE0001B0C381C311C9846FDF75EFD42464243E2
:102CF000051C311C381C9146FDF79AFD019F090403
:102D00003B0C1943894507D909196B1E8C424DD8D4
:102D100089454BD9023D09194A468A1A101C311CB3
:102D20009246FDF741FD43464343071C311C504684
:102D30009946FDF77DFD019A090413041B0C194304
:102D4000894507D909197B1E8C422DD889452BD975
:102D5000023F09194B46CB1A2D0499462F43FDE635
:102D60001E1CCAE61F1CAAE6994633E761460A0400
:102D70001B04120C9B18A6409E42A0D201380027CB
:102D8000BEE600270120BBE68A4500D875E702238E
:102D90005B429844C91971E78B4500D850E702237C
:102DA0005B429944C9194CE71F1CD3E71D1CB3E7CC
:102DB000023D0019ECE6C046094A1368002B0CD00E
:102DC00018186946884202D81060181C7047054BD5
:102DD0000C2201201A604042F8E7034B1360EFE732
:102DE0008C2D0020902D0020982D0020FEE7C0465D
:102DF000F8B5C046F8BC08BC9E467047F8B5C0465A
:102E0000F8BC08BC9E4670470B09080A0100000088
:102E1000005027002E2E2F6D61696E2E630000007A
:102E20004D595F5541525400657272203A20257504
:102E30000A000000010002006F6E5F626C655F6552
:102E400076740A0048656C6C6F0A000053746172F6
:102E5000742E2E2E0A0000005374617274204C6F81
:102E60006F700A002F55736572732F70672F636F31
:102E700064652F626C656E616E6F2F6E72663531A0
:102E80003832322F2F536F757263652F626C652F46
:102E9000626C655F73657276696365732F626C65DA
:102EA0005F7372765F636F6D6D6F6E2E63000000EF
:102EB0009ECADC240EE5A9E093F3A3B50000406EA2
:102EC0002F55736572732F70672F636F64652F6260
:102ED0006C656E616E6F2F6E726635313832322FCF
:102EE000536F757263652F73645F636F6D6D6F6E83
:102EF0002F736F66746465766963655F68616E647D
:102F00006C65722E630000002F55736572732F700D
:102F1000672F636F64652F626C656E616E6F2F6ED5
:102F2000726635313832322F536F757263652F6197
:102F300070705F636F6D6D6F6E2F6170705F74691D
:102F40006D65722E63000000D2A80100D8A80100B0
:102F5000E4A80100DEA80100EAA801004300000087
:102F6000102000200CC2010070C2010070C20100DC
:102F7000EAC1010070C2010070C2010070C201000C
:102F800070C2010070C2010070C20100F6C10100F0
:102F90003ABD010070C20100F0BC010040BD01005B
:102FA00070C201008CBD010046BF010046BF010098
:102FB00046BF010046BF010046BF010046BF0100F9
:102FC00046BF010046BF010046BF010070C20100BC
:102FD00070C2010070C2010070C2010070C2010025
:102FE00070C2010070C2010070C2010070C2010015
:102FF00070C2010098BD0100D2BE010070C2010084
:10300000D2BE010070C2010070C2010070C2010096
:1030100070C2010070BF010070C2010070C20100E7
:103020007CBF010070C2010070C2010070C20100CB
:1030300070C2010070C20100B8BF010070C201007F
:1030400070C2010004C0010070C2010070C2010022
:1030500070C2010070C2010070C2010070C20100A4
:1030600070C2010070C2010070C2010070C2010094
:1030700056C0010082C00100D2BE0100D2BE0100D4
:10308000D2BE010026C1010082C0010070C2010051
:1030900070C2010032C1010070C20100D0C0010045
:1030A00044C20100F4C001007AC1010070C20100F5
:1030B00084C1010070C2010018C2010070C2010089
:1030C00070C2010048C10100303030303030303043
:1030D0003030303030303030494E4600696E660056
:1030E0004E414E006E616E0030313233343536372A
:1030F0003839414243444546000000003031323304
:103100003435363738396162636465660000000023
:10311000286E756C6C2900003000000020202020F3
:10312000202020202020202020202020496E666999
:103130006E697479000000004E614E00504F534993
:10314000580000002E000000000000000000F03FCA
:103150000000000000002440000000000000594072
:103160000000000000408F40000000000088C340C5
:1031700000000000006AF8400000000080842E413A
:1031800000000000D01263410000000084D7974186
:103190000000000065CDCD41000000205FA002428C
:1031A000000000E876483742000000A2941A6D4201
:1031B000000040E59C30A2420000901EC4BCD642F4
:1031C00000003426F56B0C430080E03779C341439F
:1031D00000A0D8855734764300C84E676DC1AB4315
:1031E000003D9160E458E143408CB5781DAF154433
:1031F00050EFE2D6E41A4B4492D54D06CFF080440E
:10320000F64AE1C7022DB544B49DD9794378EA4422
:103210000080E03779C34143176E05B5B5B89346D2
:10322000F5F93FE9034F384D321D30F94877825A9E
:103230003CBF737FDD4F15750500000019000000CD
:103240007D00000000000000BC89D897B2D29C3CF1
:1032500033A7A8D523F649393DA7F444FD0FA5327D
:103260009D978CCF08BA5B25436FAC642806C80ACB
:10327000DCF50100E4F90100E4F90100D0F50100FA
:10328000E4F90100E4F90100E4F90100E4F90100C6
:10329000E4F90100E4F90100A4F50100CAF5010018
:1032A000E4F90100BEF50100A4F90100E4F9010010
:1032B00098F9010002FA010002FA010002FA010085
:1032C00002FA010002FA010002FA010002FA01000A
:1032D00002FA010002FA0100E4F90100E4F9010038
:1032E000E4F90100E4F90100E4F90100E4F9010066
:1032F000E4F90100E4F90100E4F90100E4F9010056
:10330000D8F80100E4F90100E4F90100E4F9010052
:10331000E4F90100E4F90100E4F90100E4F9010035
:10332000E4F90100E4F90100E4F9010062F90100A7
:10333000E4F90100E4F90100E4F90100E4F9010015
:10334000E4F901002AF90100E4F90100E4F90100BF
:10335000B4F70100E4F90100E4F90100E4F9010027
:10336000E4F90100E4F90100E4F90100E4F90100E5
:10337000E4F90100E4F90100E4F9010000F70100BB
:1033800038F80100E4F90100E4F90100E4F9010072
:103390002EF8010038F80100E4F90100E4F9010019
:1033A0001AF80100E4F90100EAF70100A2F80100AF
:1033B00074F80100F6F60100E4F90100A8F6010036
:1033C000E4F9010032F60100E4F90100E4F901003A
:1033D000E6F50100303030303030303030303030D1
:1033E000303030302020202020202020202020209D
:1033F0002020202050120200EC11020034120200A2
:103400001A110200341202002812020034120200C3
:103410001A110200EC110200EC1102002812020045
:103420001A11020010110200101102001011020006
:1034300074140200201B02000E1D02000E1D02006B
:10344000001B0200EA190200EA190200F21A020047
:10345000001B0200EA190200F21A0200EA19020037
:10346000001B0200E8190200E8190200E819020036
:08347000161D0200000000001F
:08347800A82CFF7F01000000F9
:1034800000000000FFFF0100010000000024F40024
:1034900000000000FC22002064230020CC23002038
:1034A000000000000000000000000000000000001C
:1034B000000000000000000000000000000000000C
:1034C000000000005C2F020000000000000000006F
:1034D00000000000000000000000000000000000EC
:1034E00000000000000000000000000000000000DC
:1034F00000000000000000000000000000000000CC
:1035000000000000000000000000000000000000BB
:1035100000000000000000000000000000000000AB
:10352000000000000000000000000000000000009B
:10353000000000000000000001000000000000008A
:103540000E33CDAB34126DE6ECDE05000B0000004F
:10355000000000000000000000000000000000006B
:10356000000000000000000000000000000000005B
:10357000000000000000000000000000000000004B
:10358000000000000000000000000000000000003B
:1038B0000000000000000000102000204153434998
:1038C00049000000000000000000000000000000AF
:1038D0000000000000000000000000004431020071
:1038E000F8300200F8300200F8300200F830020030
:1038F000F8300200F8300200F8300200F830020020
:10390000F8300200FFFFFFFFFFFFFFFFFFFFFFFF99
:10391000FFFF000041534349490000000000000040
:103920000000000000000000000000000000000097
:103930000000000001000000000000000000000086
:10394000B8240020B8240020C0240020C024002077
:10395000C8240020C8240020D0240020D024002027
:10396000D8240020D8240020E0240020E0240020D7
:10397000E8240020E8240020F0240020F024002087
:10398000F8240020F8240020002500200025002035
:1039900008250020082500201025002010250020E3
:1039A0001825002018250020202500202025002093
:1039B0002825002028250020302500203025002043
:1039C00038250020382500204025002040250020F3
:1039D00048250020482500205025002050250020A3
:1039E0005825002058250020602500206025002053
:1039F0006825002068250020702500207025002003
:103A000078250020782500208025002080250020B2
:103A10008825002088250020902500209025002062
:103A20009825002098250020A0250020A025002012
:103A3000A8250020A8250020B0250020B0250020C2
:103A4000B8250020B8250020C0250020C025002072
:103A5000C8250020C8250020D0250020D025002022
:103A6000D8250020D8250020E0250020E0250020D2
:103A7000E8250020E8250020F0250020F025002082
:103A8000F8250020F8250020002600200026002030
:103A900008260020082600201026002010260020DE
:103AA000182600201826002020260020202600208E
:103AB000282600202826002030260020302600203E
:103AC00038260020382600204026002040260020EE
:103AD000482600204826002050260020502600209E
:103AE000582600205826002060260020602600204E
:103AF00068260020682600207026002070260020FE
:103B000078260020782600208026002080260020AD
:103B1000882600208826002090260020902600205D
:103B20009826002098260020A0260020A02600200D
:103B3000A8260020A8260020B0260020B0260020BD
:103B4000B8260020B8260020C0260020C02600206D
:103B5000C8260020C8260020D0260020D02600201D
:103B6000D8260020D8260020E0260020E0260020CD
:103B7000E8260020E8260020F0260020F02600207D
:103B8000F8260020F826002000270020002700202B
:103B900008270020082700201027002010270020D9
:103BA0001827002018270020202700202027002089
:103BB0002827002028270020302700203027002039
:103BC00038270020382700204027002040270020E9
:103BD0004827002048270020502700205027002099
:103BE0005827002058270020602700206027002049
:103BF00068270020682700207027002070270020F9
:103C000078270020782700208027002080270020A8
:103C10008827002088270020902700209027002058
:103C20009827002098270020A0270020A027002008
:103C3000A8270020A8270020B0270020B0270020B8
:103C4000B8270020B8270020C0270020C027002068
:103C5000C8270020C8270020D0270020D027002018
:103C6000D8270020D8270020E0270020E0270020C8
:103C7000E8270020E8270020F0270020F027002078
:103C8000F8270020F8270020002800200028002026
:103C900008280020082800201028002010280020D4
:103CA0001828002018280020202800202028002084
:103CB0002828002028280020302800203028002034
:103CC00038280020382800204028002040280020E4
:103CD0004828002048280020502800205028002094
:103CE0005828002058280020602800206028002044
:103CF00068280020682800207028002070280020F4
:103D000078280020782800208028002080280020A3
:103D10008828002088280020902800209028002053
:103D20009828002098280020A0280020A028002003
:103D3000A8280020A8280020B0280020B0280020B3
:103D400000000200FFFFFFFFC9D10100E960010090
:083D5000C16001000000000049
:040000031000B8D55C
:00000001FF
